:020000040000FA
:10000000203800208D2000008B650000612000005A
:10001000612000006120000061200000000000005D
:10002000000000000000000000000000E11B0000D4
:10003000612000000000000061200000612000003D
:10004000611C0000611C0000611C0000611C0000BC
:10005000611C0000611C0000611C0000611C0000AC
:10006000611C0000611C0000611C0000611C00009C
:10007000611C0000611C0000611C0000611C00008C
:10008000611C0000611C0000611C0000611C00007C
:10009000611C0000611C0000611C0000611C00006C
:1000A000611C0000611C0000611C0000611C00005C
:1000B000611C0000611C0000611C0000611C00004C
:1000C000611C0000611C0000611C0000611C00003C
:1000D000611C0000611C0000611C0000611C00002C
:1000E000611C0000611C0000611C0000611C00001C
:1000F000611C0000611C0000611C0000611C00000C
:1001000053B94AB9002908BF00281CBF4FF0FF317E
:100110004FF0FF3000F00CB8ADF1080C6DE904CEE3
:1001200000F008F8DDF804E0DDE9022304B07047D0
:10013000704700BF2DE9F04F099E88468E46154650
:1001400004461946002B40F0C7804245B2FA82F7B8
:1001500046D94FB1C7F1200C08FA07F320FA0CFC7E
:10016000BD404CEA030EBC404FEA15481FFA85FC1F
:10017000BEFBF8F9220C08FB19E309FB0CFA42EA72
:1001800003439A4528D9EB1809F1FF3004D29A4568
:1001900002D9A9F102002B44A3EB0A03A4B2B3FBDA
:1001A000F8F208FB123302FB0CFC44EA0344A445BA
:1001B00014D92C1902F1FF3303D2A44501D9931E9F
:1001C0002C44A4EB0C0443EA00401EB1FC40002385
:1001D00034607360BDE8F08F4846DDE71346F0E712
:1001E00002B9FFDE8FBBA8EB020301214FEA154ED7
:1001F000AAB2B3FBFEFC200C0EFB1C330CFB02F876
:1002000040EA0343984563D9EB180CF1FF3004D260
:10021000984502D9ACF102002B44A3EB0803A4B229
:10022000B3FBFEFC0EFB1C330CFB02F244EA03445E
:10023000A2424FD92C190CF1FF3304D2A24202D9A9
:10024000ACF102032C44A41ABDE7C7F1200C28FA34
:100250000CF908FA07F320FA0CFCBD404CEA030243
:100260004FEA154EABB2B9FBFEFC110C0EFB1C9015
:100270000CFB03F841EA0040804504FA07F423D957
:1002800028180CF1FF3104D2804502D9ACF10201EB
:100290002844A0EB080092B2B0FBFEFC0EFB1C0051
:1002A0000CFB03F842EA004398450FD9EB180CF118
:1002B000FF3204D2984502D9ACF102022B44A3EBE1
:1002C000080342EA014191E76146E2E76246F6E748
:1002D0006046A2E76346B6E7434505D90EB1C6E9D5
:1002E00000080021084675E7B3FA83FCBCF1000F53
:1002F00010D1434501D382420AD8841A68EB030324
:1003000001209E46002E68D0C6E9004E002161E71C
:100310006046F7E7CCF1200E03FA0CF322FA0EF454
:100320001C4320FA0EF108FA0CF328FA0EFB1943CD
:100330004FEA144902FA0CF5BBFBF9F8A3B209FB2A
:1003400018BB0A0C08FB03FA42EA0B42924500FA7A
:100350000CF73ED9A21808F1FF3004D2924502D919
:10036000A8F102002244A2EB0A0289B2B2FBF9F81A
:1003700009FB182208FB03F341EA024293422AD9FF
:10038000A21808F1FF3104D2934202D9A8F1020168
:10039000224441EA0040A0FB0598D21A42454B4650
:1003A000414602D306D14F4504D2B9EB050368EBB1
:1003B000040101388EB1FC1A62EB010707FA0EFE48
:1003C00024FA0CF34EEA030327FA0CF7C6E90037C8
:1003D0009CE74046C7E74146DBE73146FAE60000C6
:1003E0007FB5304B304AC3F800263048C3F80426A6
:1003F0004921C3F80826C3F80C26C3F81026C3F811
:100400001426C3F81826C3F81C2606F024F805F0B5
:10041000DBFB274800F05CF828B9254A2548452130
:1004200006F019F8FEE701A800F06AFC224B1B68F1
:10043000834204D02148452106F00DF8FEE7039AD7
:100440001F48492106F007F81E48492106F003F825
:100450004FF44041002006F096FB20B11A48452198
:1004600005F0F9FFFEE769469DF8080000F03CF84A
:10047000009B039C1C44019B1D8900F039FF6619F9
:100480004FF02002EFF3118382F31288BFF36F8FD6
:10049000635983F30888736898470C48452105F031
:1004A000DAFFFEE7000001403546526E6875000035
:1004B0008175000094750000DC010020B375000018
:1004C000D6750000057600002A7600005D760000F3
:1004D00010B5044C236813B903F03EFE2060206879
:1004E00010BD00BFD801002008B540B1024600236E
:1004F0000448452105F0AFFF6FF0150008BD086006
:10050000FCE700BF807600002DE9F04F1D46DBB010
:10051000824BDDF890B11E68DDE96648174600F0B1
:10052000B5FE7F4B0122C3F800253AA804F080FAFB
:100530003CB1B8F1000F04DD424621463AA805F06F
:1005400095FE7B89B7F808809844FB684FF0000956
:100550009844C8454ED80DA93AA804F0DBFA704B70
:100560000022C3F80025C3F80025689B23B1202290
:100570000DA9184606F034F8002300932A464FF6DA
:10058000FF73394607A805F020FB0446002844D134
:10059000DFF898A1DFF8888102904FF0FF370DF166
:1005A000160305AA06A907A805F05BFB041E34DBA9
:1005B00040F0A480BDF81690B9F1100F38D1BDF805
:1005C0001490B9F1200F40F0A38006994B463AAA47
:1005D000284605F04EFF0446F8B94A463AA90DA848
:1005E00005F0B6FB04464F4B1B68834215D101232F
:1005F0000293D4E7659AA8EB09039A4228BF1A46EA
:100600001346924649465A46284605F032FF0446AC
:1006100038B1434B0022C3F8002520465BB0BDE84B
:10062000F08F524659463AA805F020FED14490E793
:10063000B9F1010F3ED1BDF81430202B68D80699CE
:100640003AAA284605F015FF04460028E5D19DF892
:1006500014B0BBF1200F09D8DAF80030324F039301
:10066000039B9C4205DB0023C8F800354FF0FF34A4
:100670001CE000F00BFEC8F800951DA804F0D8F9A6
:100680007A6857F8081B12681DA805F0EFFD15A938
:100690001DA804F03FFA0022C8F800253AA95A46DE
:1006A00015A805F08CFF18B9C8F80005274676E7AD
:1006B0000134D5E7B9F1220F7FF471AF7B1C3FF411
:1006C0006EAFDAF80030BB4215DDBDF81430802B78
:1006D0001ED806993AAA284605F0CBFE0446002803
:1006E0009BD1FFB2BDF8143000973AAA20210DA883
:1006F00000F01EF806464FF0FF3750E7029B53B15B
:10070000084B1B68B34201D0044B1E68344684E793
:100710004FF0FF3481E701247FE700BF0000002095
:1007200000A00250DC010020FC710000F871000004
:100730002DE9F04196B017461D469DF87020354BC7
:100740000E4653F83210019103EBC20380465B68FA
:10075000186802AA0144302301A805F014FD10B165
:100760004FF0FF3053E0DDE901431C4403AA06AB20
:10077000214601A805F02FFD0028F1D1049A072A8F
:10078000EED12549059805F01AFF0028E8D1079A0F
:10079000082AE5D12149089805F011FF0028DFD18A
:1007A00002AA214601A805F002FD0028D8D1DDE902
:1007B000013213449C42D3D1412AD1D13D4430234C
:1007C00003AA294602A8029705F0DDFC0028C7D13C
:1007D000DDE9023213449D42C2D32A4602A906A88B
:1007E00005F08AFA0028BBD12A4602A90EA805F016
:1007F00083FA0028B4D1202EB2D101990B78042BB2
:10080000AED1334606AA0131404600F057FD16B07E
:10081000BDE8F081FC710000A6760000AE76000015
:100820002DE9F04186B00223DFF86C80ADF800308E
:100830000D466F46002617F8010B01A901F0C4F818
:100840000446A0B901988168102302AA103905F066
:1008500010FE0446019805F00BFE44B910224146F3
:1008600002A805F0ACFE40B12EB14FF0FF34204697
:1008700006B0BDE8F0810126DDE7019806F0A2F997
:100880000423A0F108012A46019805F0F2FD044670
:10089000019805F0EDFDEAE7587500002DE9F041FB
:1008A000384B88B0064600200D461C6805F081F9DB
:1008B00006A9C0B201F088F8002857D1294605F0F2
:1008C00078F92C2407A9C0B204FB056401F07CF878
:1008D000002836D04FF02C0808FB05F806EB080777
:1008E000396911F0100137D14FF480730193264B11
:1008F00000932246CDE90311069B02910846FFF7BB
:1009000003FE0446214B56F8082006989A420CD163
:100910003A89FB68D1438B4207D8134482689342DB
:1009200003D21B4B1B68A3421DD045B38268002134
:1009300005F0D7FD174A1848452105F08CFD012424
:1009400011E0079805F0EDFD0746079805F090FDCA
:10095000631EE21C93420DD1002DF0D00699304663
:1009600005F0F1FA2C46069805F082FD204608B005
:10097000BDE8F08113F8011FB942EBD0AAE7074A9E
:10098000D9E700BF00000020040F00203DB8F39617
:10099000DC010020B7760000C9760000C1760000B7
:1009A00073B50D46044600212846CDE9001105F037
:1009B00089FA30B3164E2368B34203D101AA204608
:1009C00005F015FAE36AB34204D16A4601212046D4
:1009D00005F00DFADDE90032934288BF0193019BD7
:1009E000AB60019A2946204600F034FB094B1A6897
:1009F000002A03DD0848572105F02DFD002002B034
:100A000070BD05F10801FFF70BFFAB680193E8E744
:100A10003DB8F396400E0020F17600002DE9F84F26
:100A2000DFF878B01B4C1C4D8A469046994600264C
:100A30000B9B9E4201D300200FE00B9B174A9F1B8C
:100A4000B7F5806F28BF4FF480673B4606EB09017E
:100A5000504605F00EFD10B10120BDE8F88F0A994F
:100A60003B465A467118404605F01FFD0028F3D159
:100A7000C4F800563E44C4F80456C4F80856C4F8F6
:100A80000C56C4F81056C4F81456C4F81856C4F8D6
:100A90001C56CDE7000001403546526E4002002052
:100AA0002DE9F0438E4B1E688E4B43620F468E4BF2
:100AB0000365002185B00446084605F07AF804F184
:100AC0002001C0B200F080FF0121002005F071F884
:100AD00004F14C01C0B200F077FF0546204605F056
:100AE000C7F9804668B900221146204605F066F92C
:100AF000804600B37D480022572105F0ACFC01235D
:100B000091E07B488022572105F0A5FC0123984500
:100B100084F85830E7D194F858308DF80730042B1A
:100B200000F28480012B00F2888000F09F80FF2378
:100B300084F858309AE0204600F0A4F90028DED06E
:100B4000684605F0B6F96946204605F051FA18B135
:100B5000684842465721D0E7684605F0B3F980F06F
:100B600001006A46C1B2204605F028F90246002875
:100B7000C0D1684605F0A6F9804660BB69462046AC
:100B8000FFF70EFF9DF8073084F85830033B012B28
:100B900006D8404605F07AFA10B1FF2384F85830A1
:100BA0009DF80730023B022B0BD8002005F05CFAC1
:100BB00038B1FF2384F858304F48452105F04BFCED
:100BC000FEE794F85830FF2BF6D06A460021204605
:100BD00005F0F4F893E79DF80790B9F1010F17D1EC
:100BE000104602F095FC831E022B80460DD8494624
:100BF0002046FFF753FE414B1B68984205D0012861
:100C00000CBF4FF001084FF0050884F8588082E7C8
:100C100001212046FFF742FE384B1B6898420CBF6B
:100C20009DF80730052384F8583074E7052B7FF4CE
:100C30007EAF002005F02AFA13E069462046FFF750
:100C4000AFFE94F85830DA1E012A05460CD8002071
:100C500005F01CFA054600287FF469AF002005F076
:100C600003FA054610B162E7022BF7D094F858302A
:100C7000FF2B04D12048452105F0EDFBFEE7012BB9
:100C800006D06A460021204605F098F80546D0B9FE
:100C900000212046FFF702FE0646DFF86080D8F804
:100CA000003098420FD110220021684605F0A3FCC5
:100CB000206A04F087FF3871236AD8F800605B6807
:100CC000BB603C600025E06C05F0D2FB206A05F0BB
:100CD000CFFB002D14BF2846304605B0BDE8F08399
:100CE0000000002040060020400A0020627700003B
:100CF000207700008E770000B8770000DC0100202C
:100D000038B5064D044660220021284605F073FCE4
:100D100021462846FFF7C4FE38BD00BFE001002091
:100D200073B516461C4633B3436A5D686379012B7D
:100D300015D101BB1F4B22681B689A4298BF002542
:100D4000002004F036FF01A9C0B200F03DFEF0B172
:100D50000125019805F08CFB284602B070BD022BDE
:100D600009D12368012B08D9124A1268934202D88C
:100D7000B1FA81F149090025E2E7FCD10029DFD071
:100D80000129F8D12179023918BF0121F3E7294659
:100D900001982023324605F06CFB05460028D7D188
:100DA000002CD6D0356804482D1A18BF4FF0FF35F7
:100DB000CFE700BF040000203DB8F3962DE9F04FC7
:100DC000074685B00C4601460020164604F0C7FFD2
:100DD000051E51DB3846E46D04F0CEFF5FFA84F95E
:100DE00005F1FF3809FB08084FF0000A4FF0010B2E
:100DF0004FF0FF349DB9BAF1010F03DD20484521C2
:100E000005F029FB631C06D07F2C2ADC013440F25C
:100E100001133460B380284605B0BDE8F08F6B1E27
:100E200000930DF10F0201234146384605F021FBE6
:100E3000031E019322DB01220DF10F01384605F05C
:100E4000D5FE019B40B15B4501D00AF1010A009D2E
:100E5000A8EB09089B46CDE7B4F1FF3F08BF2C463D
:100E6000F5E70223803C7371631004F00104013341
:100E7000013433603471CEE70725CCE70125CAE79A
:100E8000C4770000816A426D914238B508D0531C86
:100E90008B4205D01348572105F0DDFA002038BDFC
:100EA00080291CD910485721F6E7446A056D04EBE8
:100EB000C30405EBC30564686D68AC4202D00B48FF
:100EC0005721E9E701339A42EFD1914205D9436AAC
:100ED00003EBC2025368A342F1D10120DFE70023F4
:100EE0001C46F0E7E77700001F7800004E7800000E
:100EF00000B589B004A9022005F0DEFE9DF810209F
:100F0000012A41D0254B2649032A18BF0B469DF8DC
:100F1000132002929DF8122001929DF81120214881
:100F200000924921204A05F096FA06A9052005F00D
:100F3000C3FE9DF81820012A28D0184B1849032A0F
:100F400018BF0B469DF81B2002929DF81A200192B3
:100F50009DF8192000921348144A492105F07BFAA4
:100F60009DF81030012B13D19DF81230032B0FD1B7
:100F70009DF81830012B0BD00D48492105F06BFA74
:100F8000022009B05DF804FB0A4BC0E7094BD9E722
:100F90000948492105F05FFA0020F2E77F78000058
:100FA000857800009778000089780000D8780000E4
:100FB000E87800007A7800000779000070B54B6887
:100FC00014461E4A03F0FF23934286B006460D46A0
:100FD0002FD10B68012B2CD104A9204602F044FA32
:100FE0009DF81020012A26D0154B1649032A18BF58
:100FF0000B469DF8132002929DF8122001929DF855
:10100000112000921048114A492105F024FA9DF858
:101010001030032B0DD12146304604F094FF2046BA
:1010200005F03DFEA968204604F0B9FE204602F016
:10103000FBF906B070BD064BDBE700BF0001000402
:101040007F7800008578000097780000D87800004D
:101050007A7800002DE9F04F2DED028B054689B01E
:1010600085480C464921174605F0F5F96B6A0122BF
:101070005E68002333449F42114602F10102F9D811
:10108000DFF800B22046CBF8001004F01BFF18B3C5
:10109000E86D04F05FFEAF6A0023013F33448342F2
:1010A00001D2013FFAE7DBF80030BB4214D37348AA
:1010B000572105F0D0F9DBF80020714807FB06F353
:1010C00002FB0662572105F0C6F90123E37109B05E
:1010D000BDEC028BBDE8F08F06A9022000F074FC85
:1010E00007A9052000F070FC079A21462846FFF763
:1010F00065FF6379012B08D1DBF80070DFF888A168
:10110000DBF80030A7B9012323604FF00203DFF8BA
:10111000788163710127DBF80030DDF818909F4279
:101120004DD9484605F0A4F9079805F0A1F9CEE796
:10113000226801339B1A9F423FD86B6ADDF8188002
:10114000196853F8370003EBC703012A53F8083C2A
:10115000A3EB010308EE103AA0EB010912D1E268FB
:10116000079B022A0AD041462846029304F0EBFE70
:1011700022464146284604F01CFF029B1946284699
:1011800004F0E1FE32464946404604F0DAFE18EE2D
:10119000103A42464146CDE900962846FFF73EFC0C
:1011A0002146284604F09BFE23680133236020B1CA
:1011B000DAF800300133CAF80030013FA0E72368B5
:1011C0009F4257D3696A286D51F837300393FA006C
:1011D000083A0B6850F802C0029303682079DDF8E2
:1011E0001CA00128ACEB030342D189580593029B54
:1011F0003246C91A4846049104F0A3FE0499059B9F
:1012000000914A465146019628460493FFF706FC92
:101210002146284604F063FE4FF002032371049B2D
:1012200020B1D8F800200132C8F800201946324613
:101230005046049304F085FE049B0093DDE90223ED
:1012400049469B1A019652462846FFF7E7FB21467E
:10125000284604F044FE2368013323604FF0010365
:10126000237138B1D8F800300133C8F8003001E0FC
:101270000228DBD001374EE71E79000047790000D5
:101280007679000004000020400E002070B5094D62
:101290002B7853B9084C0126C4F8006503F06AFCAA
:1012A00028B92E70C4F8000570BD0020FCE74FF08F
:1012B000FF30F9E70410002000A0025070B50B4E7B
:1012C000AEB01D46CDE902210446FFF7DFFF012342
:1012D000C6F80035DDE902212346009505A805F092
:1012E000E6FD0023C6F800352EB070BD00A0025008
:1012F000164A4FF0FF3301215160C2F84833C2F85B
:10130000083302F5C0425160C2F84833C2F80833CE
:1013100002F598325160C2F84833C2F80833A2F59A
:1013200008320021C2F80015C2F8083302F518325D
:10133000C2F80015C2F80833A2F51042C2F8083509
:101340004FF08042C2F80833704700BF00B0004041
:101350000B6801330B60014B1B6818470800002025
:1013600007B50B46002102460191034801A900F090
:10137000E9F803B05DF804FB511300002DE9F74FC5
:10138000B0F8189019F00808044693460ED00129C9
:101390000CBF49F0100949F02009A0F818908BF310
:1013A0001188BFF36F8F03B0BDE8F08FDFF890A115
:1013B00009F00709022907D1204604F09FFF002801
:1013C000EDD00128238B4BD16769218B002F15DAD3
:1013D000256821F00701C4E9008841F0010121835B
:1013E0000026218B01F007024A4502D0A368002B9A
:1013F00057D10DB9002E6FD0002353E001F0070341
:101400005A1F012A1DD821F00701062B256889B231
:10141000C4E900880AD13DB1638B2A4612680133C2
:101420009BB2002AFAD1638341F002012183204656
:1014300004F064FF0028D3D0238B43F020032383E0
:10144000CEE7042B0AD121F0070189B2218320467F
:1014500004F054FF10B141F0200121830025BFE7C3
:10146000032809D1226923F00703166843F0060315
:10147000238300252F46B4E7042806D1226923F0F0
:101480000703566843F00403F2E7052806D12269F2
:1014900023F00703966843F00503E9E700252E468D
:1014A000E8E7012341F0080121838BF31188BFF3A2
:1014B0006F8F03BB002D31D116B151462046B04786
:1014C0004FF02003EFF3118B83F31288BFF36F8F7C
:1014D000238B23F008032383238BDA0627D523F0FD
:1014E000100323830121B4F8189009F0070900299B
:1014F0007FF460AF53E7A1680029DBD0D1F80090FA
:10150000D1F804B001923B462046D847019AB9F180
:10151000000FCFD04946D9F80090F1E729463B4665
:10152000204601922D6804F005FF019AC2E713F0EE
:1015300020011EBF23F0200323830221D3E700BF35
:10154000616300002DE9F04F8FB01D46531E0190DE
:101550008A4602934FF00009029B5878252803F130
:10156000010421D14FF0000C18464FF0FF37023034
:101570006146CDF80CC03C460A2602780290392A12
:1015800000F1010058D81F2A18D8002A00F0F6816F
:10159000019B514625209847029B51461878019B94
:1015A000984709F10209D7E7002800F0E781019B7D
:1015B0005146984709F101090294CDE7A2F12003B1
:1015C000192BE5D80FF2040E5EF823F03516000053
:1015D00091150000911500003516000091150000CE
:1015E000B91600009115000091150000911500003A
:1015F00091150000FB160000351600009115000043
:101600000F170000C716000091150000D316000048
:10161000EF160000EF160000EF160000EF160000B6
:10162000EF160000EF160000EF160000EF160000A6
:10163000EF1600009446A0E7582A00F01B81A2F1A3
:1016400063035FFA83FEBEF1170FA1D8172B9FD853
:101650000FF2040E5EF823F0D718000035170000D3
:10166000911500009115000091150000151700005C
:1016700035170000911500009115000015170000A6
:101680009115000091150000911500001F18000031
:101690009115000091150000B71800009115000089
:1016A0003517000091150000911500001F1800006B
:1016B0009115000015170000019B51462520984701
:1016C00009F1010948E7039B03F0FE030393002798
:1016D00053E7002C0BDA002F0BDA039B002B00F0F2
:1016E000498124EAE47406FB0424303C45E7002FDA
:1016F000F7DB06FB0727303F3FE7002F55F8043B99
:1017000001DB1F4639E71C1EBFF637AF64420223D8
:10171000039332E7682A03D1682906D148212CE7D0
:101720006C2A02D16C2900F0278100297FF430AFA8
:10173000114622E77A2907D1752A05F104062D689A
:1017400062D14FF000080DE06C29F5D04C29F3D19F
:10175000EB1D23F007031E46752AF6E8020107D1A8
:10176000D3E90058BCF1200F51D1864B013C09E070
:1017700005468846B8F1000FF4DA6D42824B68EBFB
:101780004808013C00930DAB05934FF0000B284631
:1017900041460A220023CDF810B0FEF7B1FC059BAC
:1017A000CDF81C80303203F801292846CDE90535F3
:1017B000414600230A22FEF7A3FC069B0A2B079B47
:1017C00073F100030BF1FF3B05468846DFD2049B13
:1017D000049AC3F1010B0EAB9D18002FA5F104056F
:1017E00004DA039B13F0010F18BF2746039BA7EBF6
:1017F0000B08B8F1000FD4BFA4EB0B04E41B9B074C
:1018000000F18180274677E04FEAE578B2E7BCF146
:101810002B0F0ABF5D4B5E4B04F1FF34B2E7702A19
:1018200028D12E46002356F8041B00295CD05948C5
:101830000090023C02F06002A2F139080DF1340E72
:10184000002501F00F02092A88BF424430320EF809
:10185000012910294FEA111242EA03724FEA1310CC
:1018600073F1000305F1FF3C21D20EABC5F1010B72
:101870001D44B2E76C2904D12E46002356F8041B00
:1018800008E04C29F8D1073525F007052E466B688E
:1018900056F8081BBCF1230F06D13F4D3D4812F00E
:1018A000200F08BF2846C3E739480090C2E76546C5
:1018B00011460346C5E72E4656F8045B284604F059
:1018C0006BFE002F834602DBB842A8BFBB46304BFD
:1018D000009300278AE72E464FF0010B56F8043B91
:1018E0008DF8203008ADF2E72C4D4FF0050BEEE7F8
:1018F000019B514620209847013FF9D524EAE47323
:10190000013C9944E41A009BA9EB030904E000930D
:101910005146019B9847009B09EB030713F8010B05
:101920000028F4D1C146B9F1010913D528EAE878B5
:10193000D946B9F1010912D5BBF1000FA8BFD844AF
:101940002546013D11D5002CA8BFA04408EB07098E
:10195000354601E6019B514630209847E3E715F8EC
:10196000010B019B51469847E3E7019B514620201C
:101970009847E6E70123CBE64C21FEE548460FB049
:10198000BDE8F08FA77D0000027A0000047A000015
:1019900013810000097A0000067A00000C7A00002A
:1019A00008B54FF02002EFF3118382F31288BFF3E2
:1019B0006F8F00F097FC034804F093FC00F062F88E
:1019C000FCE700BF127A00000C4B1B6870B573B1C6
:1019D0000B4A15680022AA4202DB6FF0010070BDBD
:1019E0001C4613F8106B864204D00132F3E76FF007
:1019F0000C00F4E70C600020F1E700BF0C000020B1
:101A00006872000070B588B005460C46C0B26946E1
:101A10001646FFF7D9FF00281FDB009BEBB15A6881
:101A200002929A682168D8680195CDE903260022C0
:101A3000CDE90612059202F08FFB0546009804F0EE
:101A400017FD6DB12846084901AA04F0D1FE079898
:101A500008B9059B236008B070BD6FF01500FAE768
:101A60006FF01200F7E700BF35650000014802F093
:101A700037BD00BF6C720000014910220A60704738
:101A800010ED00E072B6404080F31188BFF36F8F15
:101A9000BFF34F8F30BF62B6BFF36F8F704700BF89
:101AA00072B6494081F3118820BF80F3118862B675
:101AB000704700BF37B505460C46C9B18B68009327
:101AC000D1E900230E48452104F0C5FC6369009369
:101AD000D4E903230B48452104F0BDFCE2690A4820
:101AE000452104F0B8FCA2690848452104F0B3FC84
:101AF0002146284603B0BDE8304002F057BB00BF86
:101B00003B7A00006F7A0000A37A0000B77A0000E9
:101B100043B2002B08DB012200F01F0002FA00F0A4
:101B20005B09024A42F82300704700BF00E100E071
:101B3000054B420900F01F0053F82220012303FA4D
:101B400000F01040704700BF00E100E043B2002BFE
:101B5000A8BF03F1604301F10101B8BF064B4FEA92
:101B60004111ACBF03F5614300F00F00C9B2B4BF2F
:101B7000195483F80013704714ED00E030BFFFF7ED
:101B8000FDBF00BF144A08B5144B22F07F029A60D3
:101B9000BFF34F8FBFF36F8FD3F8882022F470020A
:101BA000C3F88820D3F8882042F4A002C3F8882024
:101BB0004FF04042C3F83422BFF34F8FBFF36F8F13
:101BC0000023E1EE103A02F047FB02F08BFB00F03D
:101BD00051FA02F04DFB00BF0000000000ED00E0F4
:101BE0001EF0040F0CBFEFF30880EFF3098081694A
:101BF00011F8021C0229FFD001B504F0BEFC01BDA2
:101C000010F1160F074B08D0984208D320338342B7
:101C100005D98B4203D9044870472033F9E70020E7
:101C2000704700BF201000204010002004460846E6
:101C300011461A460023E1EE103A084B202583F3A3
:101C4000098863B64FF0000383F31188BFF36F8FE9
:101C5000A04785F31188BFF36F8FFEE7403800205F
:101C600001B5EFF30580A0F110004FEAC000044970
:101C7000014409C99847BDE80140024908470000EE
:101C8000F46F0000891C0000704700BF2DE9F0418F
:101C9000324C0746884632484521154604F0DBFBA6
:101CA000A36ADE0603D52F48452104F0D4FBA36ABE
:101CB0001C0703D52C48452104F0CDFB274CA36A13
:101CC000980728D46FF01506244CA36ADA0703D5C9
:101CD0002648452104F0BFFBA36A9B0603D5244890
:101CE000452104F0B8FB1D4B9A6AD40628D49A6AA1
:101CF000900725D40020194B9A6A920642BF5A6A6F
:101D000022F400525A629A6A42F0FF029A62002359
:101D10002B70BDE8F0814521164804F09CFB666BF2
:101D2000A36A1906CED514483246452104F093FB28
:101D3000B8F1000FC8D0A36A23F08003A362C3E701
:101D40005B681905D6D539463046FFF759FF00289C
:101D5000D0D080F309880220CDE700BF00ED00E07D
:101D6000EA7A0000057B00003D7B00008D7B0000CF
:101D7000B17B0000557B0000727B000010B51D4C4C
:101D80001D48452104F067FBA36A9B0103D51B484E
:101D9000452104F060FBA36ADC0103D51848452106
:101DA00004F059FB134CA36A180303D515484521C9
:101DB00004F051FBA36A590303D51348452104F0ED
:101DC0004AFB0C4CA36A9A0303D51048452104F042
:101DD00042FBA36ADB0303D50D48452104F03BFB1E
:101DE000044A936A6FEA03436FEA13439362002045
:101DF00010BD00BF00ED00E0E57B0000027C0000AC
:101E00001A7C0000397C00005C7C0000867C0000AD
:101E1000A57C000070B5234C06460D46224845219E
:101E200004F019FBA36AD90403D52048452104F026
:101E300012FBA36A1A0503D51D48452104F00BFBCC
:101E4000184CA36A9B0510D51A48452104F003FBE2
:101E5000A26BA36A180408D51748452104F0FBFAC1
:101E60001EB1A36A23F40043A3620E4CA36A590572
:101E700003D51248452104F0EEFAA36ADA050BD522
:101E80000F48452104F0E7FA064A936A002043F41C
:101E90007F439362287070BDA36A9B04F4D5094800
:101EA0004521EFE700ED00E0D57C0000F07C00006C
:101EB0003D7B0000067D0000247D00003E7D00008B
:101EC0005E7D0000B17B00002DE9F041554B5F685D
:101ED0008AB0C7F30804002686F31188BFF36F8F1A
:101EE00002F07F43B3F17F4F07D102F00C03082BC0
:101EF00005D14D48452104F0AEFA354604E01207FD
:101F00004EBF0D46054601264FF00008E31E8DF832
:101F10000780092B73D8DFE803F005676B647272E2
:101F20007272726F3F4F4148452104F094FAFC6A87
:101F30008DF8078014F0020405D03D48452104F0D7
:101F40008AFA002406E0FB6A002B1DDA3948452195
:101F500004F081FA9DF807309BB92022294602A897
:101F600004F03EFB099B002E56D0C3F3080222B9B1
:101F70006FEA53236FEA4323099302A92046FFF730
:101F800099FD0AB0BDE8F081FB6A5B00E2D52A4802
:101F9000452104F060FAAB6933F8022C4DF6027368
:101FA0009A420AD097F8283073B10DF10702012147
:101FB0002846FFF76BFE0446CCE72A681F484521F8
:101FC00004F049FA2C68C5E797F829302BB10DF1D8
:101FD00007010120FFF71EFFEDE77B8D9BB2002B71
:101FE000B8D0FFF7CBFEE6E70DF107020021DFE7EF
:101FF0000DF107010020EDE7114845219FE7114948
:10200000114A124817F4F87F08BF0A46A4F11003DA
:10201000452104F020FA94E723F4FF7323F0010331
:10202000AAE700BF00ED00E0A97D0000D97D000017
:10203000F57D00001B7E00002E7E0000527E000019
:10204000737E00007B7D0000907D00009C7E000080
:10205000024A536943F010035361704700ED00E0FA
:10206000EFF30880EFF3098101B57246FFF72CFF0B
:1020700001BD00BF044800232021C2180133302BCA
:1020800082F80013F9D1704700E100E0002080F3EE
:102090001488BFF36F8F04F037FF00200D490860EC
:1020A000BFF34F8F0C4880F3088800F02BF82020F6
:1020B00080F3118809484FF40261401880F30988C1
:1020C000EFF314800221084380F31488BFF36F8F6D
:1020D000FFF758FD94ED00E0203800204038002044
:1020E0000749D1F890200023C2F3072218469342F3
:1020F00000D17047C1F89830C1F8A0000133F6E76D
:1021000000ED00E008B572B6002383F31388FFF7F3
:10211000E7FF144B4FF0FF32C3F88020C3F8842050
:10212000C3F88820C3F88C20C3F89020C3F894200B
:10213000C3F89820C3F89C20C3F88021C3F88421F9
:10214000C3F88821C3F88C21C3F89021C3F89421E7
:10215000C3F89821C3F89C2162B6BFF34F8FBFF339
:102160006F8F08BD00E100E0024B034A03480221E3
:1021700000F06AB800000420000000207472000023
:10218000F8B5234F00268E420FDA4468002C3CD06D
:102190009BB104F1FF3C14EA0C0F08D01D483246F5
:1021A000452104F058F96FF015021046F8BD1F2CB8
:1021B000F4D905681CEA050FF0D1202C0568D0F889
:1021C00008C0D2B20FD9B4F1004F0ED8013CB4FA16
:1021D00084F4C4F11F046400072A4CEA040406D9FD
:1021E0000D484521DDE70824F6E73E24F4E725F015
:1021F0001F05154345F0100544F00104C7F8982069
:10220000C7F89C500132C7F8A04001360C30BAE73D
:1022100000ED00E0B87E0000E07E0000044B0522E7
:10222000C3F89420BFF34F8FBFF36F8F704700BF89
:1022300000ED00E0BFF35F8F024B0022C3F8942053
:10224000704700BF00ED00E010B5034C0123227879
:10225000FFF796FF207010BD051000201449086894
:10226000082810B521D8FFF7E5FF124C4968002275
:10227000904201F10C0105D10F4B1870FFF7CEFF12
:10228000002010BDC4F8982051F80C3C23F01F0327
:10229000134343F01003C4F89C3051F8043C43F05E
:1022A0000103C4F8A0300132E2E74FF0FF30E8E765
:1022B0008C72000000ED00E0051000204FF02002BD
:1022C000EFF3118382F31288BFF36F8F044A012169
:1022D000C2F8401583F31188BFF36F8F0020704759
:1022E00000E001404FF08043C0B2C3F81C05BFF3CB
:1022F0004F8F0549054BCA6802F4E0621343CB6077
:10230000BFF34F8F00BFFDE700ED00E00400FA05CA
:1023100020B1034B800143F001031847704700BF11
:10232000F0710000084B70B5C31A0D4607499B10A9
:10233000044659430648402204F082F92B460146E0
:102340002046BDE870401847540E0020B76DDBB63C
:10235000646F000073B50C4C0C4A4023041B0093BF
:102360000D460B460A49A41061430646094804F08D
:1023700094F9011E05DA30462B4602B0BDE87040E4
:10238000184702B070BD00BF540E00200D6700005A
:10239000B76DDBB6646F0000002270B50121044602
:1023A0001046FFF7D3FB0F4801F0D6FA0E4B9842C8
:1023B00015D104F0B2FC26690C49304603F0EEFF5B
:1023C00000280BDB246909490125356404F11C0050
:1023D00003F0E4FF002801DBE564002070BD6FF02E
:1023E0000400FBE72D2400000000AD0BDC720000B0
:1023F00073B50C2301460B484B43C418D4E90E5265
:1024000000264033A6631844019204F006F935B162
:10241000019A05482B4602B0BDE87040184702B04B
:1024200070BD00BF540E0020646F000010B1012881
:1024300004D07047034B1B6C5B0701D1FFF7D8BF7B
:10244000704700BF540E002008B54FF02003EFF393
:10245000118183F31288BFF36F8F124A136843F020
:10246000020013F0010310600CD04FF08042D2F84C
:102470000C34D2F80C2413F0010303D00A4804F002
:10248000CCF8012381F31188BFF36F8F23B1BDE82E
:1024900008400020FFF7ACBFBDE80840012004F071
:1024A00049BC00BFA40E0020940E0020094BBFF3CE
:1024B0005B8F53E8002F22F0020143E80010002850
:1024C000F7D1BFF35B8FD30702D4012004F06FBCB8
:1024D000704700BFA40E00202DE9F8433749BFF331
:1024E0005B8F0746012251E8003F41E800200028A9
:1024F000F9D1BFF35B8F33B9314932484B60CB60C0
:102500008A6003F05EFF7B1E012B31D8012F07D1BB
:102510004FF08043D3F81C3403F00303012B27D082
:1025200004F0BAFC044618B9274B1B78002B3DD1A8
:102530004FF02003EFF3118683F31288BFF36F8F00
:102540000124DFF888904FF080454FF00108D5F85E
:102550001834D5F81824D2030CD503F00303012B4B
:1025600001D0012F06D1DCB186F31188BFF36F8F44
:10257000BDE8F8833046FFF793FAD5F81835002BFD
:10258000E5D1D5F80421002AE1D0C5F80431D5F809
:102590000431C5F81885C9F88081C5F80880D6E7E8
:1025A0004FF080430222C3F80423E1E74FF0804359
:1025B0000222C3F808230646C3E700BFA80E002086
:1025C000440E0020700E00200710002000E100E003
:1025D00030B54068047B01F01F05B2F5001F45EAE5
:1025E000441585B04FF0000404D1284601F038FCB2
:1025F000002032E0B2F5800FCDE902442FD1B3F1D3
:10260000007F0CBF042305238DF80830836823FA6C
:1026100001F1C9072FD4B2F1A07F2CD16A09012A98
:1026200005F01F031C4A03F5E07318BF4FF0A042EA
:1026300052F82330DB071ED40DF10704214628464B
:1026400001F072FB154B984214D1204601F0BAFB01
:10265000134B98420ED06FF00B0005B030BDB3F1B4
:10266000C06F05D0B3F1007F0CBF02230123CBE77D
:102670000323C9E703940023194602AA284601F060
:102680002DFA074B984204D10121284601F0A0FB06
:10269000AEE76FF00400E0E7000300500400AD0B6C
:1026A0000000AD0B10B501F07DFB044668B901F0E8
:1026B00051FB084B98420AD10748214601F02EFBF6
:1026C000224605210620FFF741FA002010BD6FF0D9
:1026D0000400FBE70000AD0BDD260000430970B5E8
:1026E00002D0012B15D070BD0B4E336959680029FB
:1026F000F9D000F01F0301250C689D408A682A402C
:1027000002D04B6830469847002CECD02146246814
:10271000F4E7024EE9E700BF7C6F0000946F000011
:102720002DE9F04347683B7B01F01F0585B00E465D
:1027300045EA43151446CAB902A9284601F0F4FA3D
:102740000446284601F0B4FB4A4B984204D06FF08F
:10275000040005B0BDE8F083844205D19DF808006F
:1027600001F02AFBA042F2D10020F2E74FF000096D
:102770000DF103013046CDE9029901F0D5FA4B463F
:10278000804602AA4946284601F0A8F9394B9842EA
:1027900002D06FF01500DCE7804503D19DF80300FF
:1027A00001F00AFBA30351D540F20663234040F237
:1027B000062293423BD00CD8062B15D004D89BB1EF
:1027C000022BE6D104230FE0B3F5007FE1D1012312
:1027D0000AE040F2024293422BD0B3F5C06F2AD0F8
:1027E000B3F5806FD5D102238DF8043084F48033A3
:1027F000C3F30043E0068DF8053054BFC4F3401323
:10280000032321038DF8063017D57B68012101FAD7
:1028100006F6C3F80865002201A9284601F00CFA63
:10282000144B984214BF6FF01500002091E7072366
:10283000DAE70523D8E70323D6E7620341BF7B68C5
:10284000012101FA06F6C3F80C65E4E7E3064FF050
:10285000000354BFC4F3401403241A4601A92846B8
:102860008DF8044001F03AF9024B98423FF47CAFF6
:102870008FE700BF0000AD0B024B0B60012313601C
:10288000704700BFC40E002000487047407300002E
:1028900010B504F0EEFA034C206004F0E6FA606034
:1028A000002010BDC40E002037B50C462046194646
:1028B0000193154603F08BFF019B40B9094822465E
:1028C000452103F0C8FD6FF0150003B030BD33B1F2
:1028D0001A462146284603F083FE0020F5E71846F5
:1028E000F3E700BF4C7F00004FF08042D2F8101594
:1028F000D2F8103501F01E0123F01F030B4343F003
:102900000103C2F81035024B00221A70704700BF55
:10291000061000204FF08053D3F83031082B22D11D
:102920004FF08042D2F8101511F001001CD0D2F8FF
:10293000100501F01E0120F01F000843C2F8100529
:10294000D2F8080158B1D2F8103523F01F030B4319
:1029500043F00103C2F810356FF08B007047034B52
:1029600001221A7070470020704700BF0610002037
:102970002DE9F8430E463046194617461C4603F02B
:1029800026FF48B91B4823463246452103F063FD24
:102990006FF01500BDE8F88344EA060515F003055D
:1029A00004D01548234632464521EFE7FCB1DFF855
:1029B000509024F00304AC4205EB060806D10F4A00
:1029C000D2F80034DB07FBD50020E3E7FFF7A2FFD6
:1029D00050B97959404601F091FB99F800300BB19C
:1029E000FFF782FF0435E6E76FF08B00D2E7204661
:1029F000D0E700BF4C7F00006E7F000000E0014088
:102A0000061000202DE9F0410F46154604F02DFA7E
:102A100029460646384603F0DAFEB84660B3B7FBEF
:102A2000F6F306FB137323B9B5FBF6F406FB145457
:102A300044B114482B463A46452103F00CFD6FF093
:102A4000150413E0AE4211D804F00FFA0E4F0646FB
:102A5000FFF760FF044660B9404601F02FFB3B786A
:102A60000BB1FFF741FFAD1BB044F1D12046BDE8EB
:102A7000F0816FF08B04F9E704482B463A46452174
:102A8000DBE700BF917F0000061000204C7F0000B4
:102A9000074BD3F8082142B10020C3F80801D3F84E
:102AA0000821D3F818350B7070474FF0FF3070478E
:102AB00000200040024BD3F88004C3F88004704724
:102AC00000200040F8B50E4604F0E6F91A4D78BB38
:102AD00064240127BFF35B8F55E8003F002B03D12F
:102AE00045E80072002AF7D1BFF35B8F07D04FF49F
:102AF0007A70013C04F0D6F914F0FF04EAD10F4CCF
:102B00000023C4F81C31D4F81C310123A360C4F89D
:102B10001C654FF47A76D4F81C3123B9012004F0F7
:102B2000FAF8013EF7D10123E36000232B60F8BDE2
:102B300001232B60E3E700BFCC0E00200020004003
:102B400030B54B79012B22D0032B1DD110258B7969
:102B5000032B19D1CB79BBB90A7912B1022A13D14F
:102B60000E220B68B3F5164F61D02DD8B3F5165F62
:102B70005FD016D8B3F5966F5DD00AD8B3F5967FBF
:102B80005CD0B3F5167F5CD06FF085004EE0002579
:102B9000DDE7B3F5166F57D0B3F5965FF4D1344B3C
:102BA00039E0B3F5E14F52D007D8B3F5615F50D0AB
:102BB000B3F5964FE8D12F4B2DE047F61224A342F0
:102BC000E2D14FF4000326E0B3F5613F44D011D8C1
:102BD000B3F5963F42D008D84DF6C024A3423FD06B
:102BE000B3F5614FD0D1244B15E0B3F5E13FCBD124
:102BF000224B10E0B3F5612F35D007D8204CA3420B
:102C000033D0B3F5E12FBFD11E4B04E01E4CA342DD
:102C1000BAD14FF0805304691C482A43C0F82435C8
:102C2000C0F86C2503C984E80300002030BD184BB0
:102C3000F1E7184BEFE74FF49E23ECE74FF4A03396
:102C4000E9E74FF41C33E6E74FF41D23E3E7124BAB
:102C5000E1E74FF46C13DEE7104BDCE7104BDAE7EB
:102C60004FF46503D7E70F4BD5E74FF08063D2E70A
:102C700000B0130000A04E0000F0EB0000E0D70110
:102C800090D0030000705F0740420F00002000401A
:102C900000509D000050270000F0750000B0AF0309
:102CA00000903A0100D0BE0EF7B54368124C1E6882
:102CB000076900210546C4F8001501AA304603F053
:102CC00089FE002815DB019B32681979186803F02A
:102CD000B8FE00280DDB39462846FFF731FF40B922
:102CE0000423C4F80035C4F80801D4F808310123DE
:102CF000236003B0F0BD00BF00200040F8B50669B6
:102D000005460F4604F0C8F810B9294B1B78A3B943
:102D10004FF02003EFF3118483F31288BFF36F8F1A
:102D2000686803F0BBFD00BB84F31188BFF36F8FAD
:102D3000EEE784F31188BFF36F8F6424686803F0B3
:102D4000ADFD28B9012003F0E6FF013CF6D1F4E720
:102D50004FF02003EFF3118483F31288BFF36F8FDA
:102D6000686803F09BFD0028E3D006F8107F6968CF
:102D70000B680122C3F84465C3F848250022C3F854
:102D80002021D3F82001C3F85821D3F858214A68EC
:102D9000D20641BF0822C3F800254FF48002C3F8D1
:102DA000042301229A6084F31188BFF36F8FF8BD6A
:102DB00007100020F0B54B79012B26D0032B21D131
:102DC00010268B79032B1DD1CC790CB1012C19D194
:102DD0000A7912B1022A15D10E220B684568B3F5A3
:102DE000164F2D6865D02DD8B3F5165F64D016D870
:102DF000B3F5966F62D00AD8B3F5967F61D0B3F57C
:102E0000167F61D06FF0850052E00026D9E7B3F558
:102E1000166F5CD0B3F5965FF4D1374B3CE0B3F559
:102E2000E14F57D007D8B3F5615F55D0B3F5964F52
:102E3000E8D1324B30E047F61227BB42E2D14FF4E3
:102E4000000329E0B3F5613F48D013D8B3F5963FAE
:102E500047D009D84DF6C027BB4244D0B3F5614FE7
:102E6000D0D14FF46B0317E0B3F5E13FCAD14FF077
:102E7000EB7311E0B3F5612F38D008D8204FBB4277
:102E800037D0B3F5E12FBDD14FF0E86304E01D4F1B
:102E9000BB42B7D14FF080530069C5F82435031DFC
:102EA00003C934432243C5F86C2583E8030000209E
:102EB000F0BD4FF41D03EFE7134BEDE74FF49E23F6
:102EC000EAE74FF4A033E7E74FF41C33E4E74FF4AD
:102ED0001D23E1E70D4BDFE70D4BDDE74FF06C7392
:102EE000DAE70C4BD8E74FF46503D5E74FF0706392
:102EF000D2E74FF08063CFE700B0130000A04E0090
:102F000090D0030040420F000050270000C0750021
:102F100000F03A0000903A0110B501238340114AB5
:102F2000BFF35B8FDC4352E8001F01EA040C42E868
:102F300000CEBEF1000FF6D1BFF35B8F4FF48032AD
:102F400002FA00F002F1804202F58052C2F8080352
:102F5000BFF35F8FBFF36F8F0B4214BF01200020C0
:102F600010BD00BFD40E00201949F8B5044622F068
:102F70007F450868C1E90023A5F50013101AB3F5D1
:102F8000400F22D2134B1B681A0A1B065E19124B04
:102F900042F10007C3E90067012601F0FFF9A30031
:102FA00003F1804303F58833D3F84025AA420BD1BF
:102FB0001EB94FF40002C3F84025084B4FF480308F
:102FC00000FA04F4C3F84443F8BD0026E5E700BF67
:102FD00048010020D80E00203001002000100140E0
:102FE00019B3BFF35B8F0123104A834052E8001FDF
:102FF000194342E8001CBCF1000FF7D1BFF35B8F0F
:103000000B4A4FF480338340C2F80433094BBFF3BB
:103010005B8F1B68BFF35B8F23FA00F0C30742BFCF
:10302000054B4FF40032C3F800217047D40E002046
:1030300000100140D00E002000E100E00D4B1868A8
:10304000010A0006BFF35F8F0B4BD3F80435181845
:1030500041F10001B3F5801F0AD2084BD3E90023E8
:10306000904271EB030303D210F1807041F1000133
:10307000704700BFD80E0020001001403001002032
:103080002DE9F04F2DED028B85B01646984605468A
:10309000FFF742FF08EE100AFFF7D0FFB04271EBD6
:1030A00008037BD2474B301A68EB0101984271F15B
:1030B000000380F08480444B03EB0513D3E902AB9B
:1030C000D84508BF564551D04FEA850909F18049D6
:1030D00005F1500709F58839BF004FF4803101FA36
:1030E00005F3BFB226F07F4207F180470193D9F87C
:1030F0004005364B07F588371446D3F80415401AB7
:1031000020F07F4021F07F4C0128C9F840C507D14D
:10311000CDE90221132003F0C5FEDDE902212B4B8E
:1031200001F1020CA4EB0C0020F07F40B0F5000F81
:1031300088BF64460020386038680198C3F84403AB
:1031400024F07F40C9F84005D3F80405814206D039
:10315000201A023820F07F40B0F5000F1CD8A41AC6
:1031600024F07F4414EB060A48F1000B164910982E
:103170002B0101EB0512C2E902ABC850119B536051
:103180000024284618EE101AFFF72AFF204605B043
:10319000BDEC028BBDE8F08F2046AEE701230C4A60
:1031A000BFF35B8FAB4052E8001F194342E80010A9
:1031B0000028F8D1BFF35B8FB246C346D6E76FF065
:1031C0001504DEE701000001380100200010014075
:1031D000D00E002073B5194B194D00244FF0FF306D
:1031E0004FF0FF31C5F80845C3E902014FF48033C1
:1031F000C5F80433134B02264FF400320121C5F801
:1032000004631120C3F880212246FEF79FFC1120A1
:10321000FEF77EFC0C4A0123AB602B6013600B4B66
:103220000B4A0093019400232046FFF729FF304604
:10323000FFF752F9204602B070BD00BF38010020F0
:103240000010014000E100E0D40E0020692F0000D2
:10325000FFFF7F002DE9F743364CD4F804339A077B
:103260000BD5D4F8043143B1334A0023C4F80431F8
:10327000D4F804311368013313604FF02003EFF3E7
:10328000118283F31288BFF36F8FD4F80433DB030A
:1032900012D5BFF35B8F294B53E8001F21F00100CB
:1032A00043E80006002EF7D1BFF35B8F002939D128
:1032B000D4F84031002B35D1002382F31188BFF3BD
:1032C0006F8F63B3FFF7BAFE4FF02003EFF3118C5B
:1032D00083F31288BFF36F8F194BD3E90267B042B3
:1032E00071EB070228BF4FF0FF384FF0000221BFFB
:1032F0004FF0FF39D3E90015C3E902891A6026BFF0
:103300004FF48033C4F8483311468CF31188BFF36F
:103310006F8F21B1009532463B460020884703B0AD
:10332000BDE8F0830023C4F84031D4F840310123D4
:10333000C3E700BF00100140D80E0020D00E0020CF
:1033400038010020431C13B521D0012821DDB0F540
:10335000000F20DA441EFFF771FE104BD3E9001373
:10336000401AB0F5000F28BF0024013002190C48A4
:10337000824228BF024652184FF0000009490190CE
:10338000009143F10003FFF77BFE02B010BD04483B
:10339000E0E70024DFE7024CDDE700BF4801002042
:1033A000FFFF7F00692F000008B5FFF747FE024BC3
:1033B0001B68C01A08BD00BF48010020036803F065
:1033C0001F025B09012B0260024818BF4FF0A040AA
:1033D000704700BF000300500C4A30B513680C4D15
:1033E000002405EB0311D1F80818C9B221B904B1C2
:1033F00013600360002008E00133072B4FF0010445
:10340000EFD9036013606FF01B0030BDDC0E0020AD
:1034100000E00140034808B5452103F01CF80020F6
:10342000FEF760FFDD7F000030B5816885B01039A0
:1034300021F00704054603F074F81022014668469F
:1034400003F0D9F807491022684603F0C9F81023A1
:103450006A462146284603F028F8003818BF0120A4
:1034600005B030BD5875000030B50C46816887B096
:10347000102302AA1039054602F0FBFF002802DAE9
:10348000012007B030BD102202A9284603F089FBB5
:1034900090B303232370284603F094FB01230146D5
:1034A0000DF10702284602F0E4FF0028E8DB9DF852
:1034B000073003F00F021B096270237101220DF126
:1034C0000701284603F06DFB10B96378042B03D97C
:1034D0000123637000232371AA68183A22F00702BF
:1034E000083AA11C284603F087FB0028C8D1E11C3C
:1034F000284603F0DBFBC4E70449102202A803F0CE
:103500005EF8002814BF02230123C3E758750000AA
:103510002DE9F04385B006466946022003F0CCFB56
:10352000054618B1FF2005B0BDE8F08302A90520CB
:1035300003F0C2FB012804463FD12D483246492101
:1035400002F089FF03238DF808308DF809408DF8CB
:103550000A308DF80B308DF80C509DF800509DF816
:1035600008609DF803709DF80B809DF80290214C37
:1035700000222078294603F02BFB18B360783146EF
:1035800003F026FBF0B1A378042B01D0BB4219D184
:10359000E378042B01D0434514D12379042B0FD1B8
:1035A0006379022B19D1144A1448492102F053FFC0
:1035B0006079831E022BB6D9B4E70028CDD0B1E7DD
:1035C0004B45EDD00132032A04F10604D1D10C4859
:1035D000492102F040FF0120A5E7032B05D0094A4D
:1035E0000949042B18BF0A46DEE7084ADCE700BF9A
:1035F0002280000095800000068000006D800000A1
:1036000080800000FF7F0000108000000B80000021
:103610004FF08053D3F83021082A06D1D3F8343143
:10362000052B02D8024AD05C70470020704700BFCB
:10363000AD800000024AD2F80034002BFBD0704766
:1036400000E0014008B503F05CFB40B14FF080435F
:103650000022C3F80C21C3F81021C3F8382503F069
:1036600050FB002846D04FF08052624BD2F8041431
:10367000C3F82015D2F80814C3F82415D2F80C1496
:10368000C3F82815D2F81014C3F82C15D2F8141466
:10369000C3F83015D2F81814C3F83415D2F81C1436
:1036A000C3F84015D2F82014C3F84415D2F82414F6
:1036B000C3F84815D2F82814C3F84C15D2F82C14C6
:1036C000C3F85015D2F83014C3F85415D2F8341496
:1036D000C3F86015D2F83814C3F86415D2F83C1456
:1036E000C3F86815D2F84014C3F86C15D2F8442416
:1036F000C3F87025FFF78CFF18B13F4B3F4AC3F862
:103700008C26FFF785FF18B13D4BFB22C3F8182527
:10371000FFF77EFF70B14FF080414FF08053D1F83A
:10372000E42ED3F8583222F00F0203F00F031343B4
:10373000C1F8E43EFFF76CFF20B1324B4FF400724A
:10374000C3F8402603F0DDFA48B14FF08043D3F8C8
:103750000024D20744BF6FF00102C3F800242A4AB4
:10376000D2F8883043F47003C2F88830BFF34F8F2B
:10377000BFF36F8F4FF08053D3F83021082A0ED15A
:10378000D3F83431052B02D8204AD35C3BB14FF03B
:103790001023D3F808224FF08043C3F858254FF088
:1037A0001021D1F80C32DB071FD519480123C0F8CE
:1037B0000435FFF73FFFD1F80C3223F00103C1F8C5
:1037C0000C32FFF737FF0023C0F80435FFF732FF54
:1037D000BFF34F8F0C490F4BCA6802F4E0621343EA
:1037E000CB60BFF34F8F00BFFDE70B4B0B4A1A6056
:1037F00008BD00BF00C000400050004048810300E9
:1038000000F000400090024000ED00E0A7800000C2
:1038100000E001400400FA052C0000200090D003D5
:1038200070B501250268B2FA82F3C3F11F035E1C72
:10383000DCB214D0BFF35B8F05FA03F322EA030373
:1038400050E8006F964204D140E8003CBCF1000F04
:10385000F6D1BFF35B8FE5D102480C7070BD024812
:10386000FCE700BF0000AD0B0200AD0B0368CB40CE
:10387000DB0710B515D4012303FA01F10368BFF388
:103880005B8F41EA030250E8004F9C4204D140E8BC
:10389000002CBCF1000FF6D1BFF35B8FEED10248D4
:1038A00010BD0248FCE700BF0000AD0B0400AD0BEB
:1038B000F7B5044618B1012829D003B0F0BD4FF088
:1038C00080430222C3F80823C3F80401D3F804217B
:1038D0000122DA6001239C428DF8073014BF0025D5
:1038E0000DF1070542F210774FF08046D4B1012C5C
:1038F000E3D125B1D6F80C3403F001032B70D6F8D0
:103900000C34DB0318D4134B00225A71D5E74FF067
:1039100080430022C3F80803C3F80021D3F8002134
:103920005860D7E725B1D6F8183403F003032B60AD
:10393000D6F81834DA03C0D52DB9012003F0EBF91D
:10394000013FD3D103E09DF80730012BF5D0012CC6
:10395000D9D0B2E7E00E0020044B1A7922B9012237
:1039600018609A800248704702487047E00E0020B5
:103970000000AD0B0C00AD0B4FF0804310B5D3F839
:1039800000216AB10022C3F80021D3F800210122EE
:10399000C3F80823114B587910B95A711B6898471E
:1039A0004FF08043D3F8042172B10022C3F8042100
:1039B000D3F80421D3F81824D3F81814920704D1AB
:1039C0000122C3F818259A6010BD0222C3F808230B
:1039D000024BBDE810401B6801201847E00E002094
:1039E000036803F01F025B09012B0260024818BF45
:1039F0004FF0A040704700BF00030050034B083059
:103A000033F81000C0F34010704700BF30000020B2
:103A100070B500F108030C4C34F81330DA05054694
:103A20000E4607D5C3F3432304EBC30254F83330E7
:103A300052689847A3682BB1E26831462846BDE832
:103A40007040184770BD00BF30000020134A083096
:103A500010B432F81030D9051CD5C3F3432123F438
:103A6000F85322F8103002F11004002034F8023B21
:103A700013F4807F03D0C3F3432399420AD001306B
:103A80003028F3D1002342F8313005485DF8044B6B
:103A9000FFF7ECBE5DF8044B704700BF300000201C
:103AA000A400002038B50246FFF7A8FF094C02F138
:103AB000080540B134F8153007495B0B03F5A273D4
:103AC000002041F823001046FFF7C0FF002324F830
:103AD000153038BD30000020006000402DE9FF4166
:103AE000044617461D4621B34E4E00F1080836F82D
:103AF00018309B0706D5FFF781FF18B14A4804B07C
:103B0000BDE8F0810023CDE900338DF80E308DF84B
:103B10000F300DF10F020B4620460DF10E0103F0A0
:103B200048F936F8183023F0020343F0010326F871
:103B3000183097B13B4B3E787A6804F1080033F8AF
:103B400010108F070CD5002AD8D133F8102022F09E
:103B50001C0242EA860223F81020CDBB3348CEE790
:103B600021F02001C904C90C23F81010002AECD060
:103B7000032EC3D817782EB92D4A07F5A27142F843
:103B80002160E2E7BA0002F1804202F5C04241EA58
:103B90004731D2F810C52CF0030CC2F810C5D2F88A
:103BA00010C52CF44F3C2CF4407CC2F810C5D2F860
:103BB00010E54FEA042C0CF47C5C4EEA064E4CEA0D
:103BC0000E0C41F0200123F81010C2F810C5BCE71C
:103BD000D5E900672046FFF739FF002EBED0114D12
:103BE0002B689E4204D16B689F4201D100220AE0FB
:103BF00010480DF10F01FFF713FE0C4B98427FF4B4
:103C00007EAF9DF80F2045F8326005EBC203083403
:103C10005F6035F8143043EA422343F4807325F89B
:103C200014309BE7300000200400AD0B0000AD0B0A
:103C300000600040A4000020F0B5044685B01546A1
:103C400019B3334E00F1080736F81720930703D451
:103C5000FFF7D4FE002858D112F01C0F02D04B7889
:103C6000012B52D001238DF80F300023CDE9001332
:103C70004A1C8B1C20460DF10F0103F09AF836F810
:103C8000173043F0030326F8173015B9214805B063
:103C9000F0BD1F4E04F1080736F81700830734D52E
:103CA00095F800C06146890020F0200001F18041B4
:103CB000C00401F5C041C00C26F817000023C1F86C
:103CC00010356A78002AE1D0D1F81035AD7823F4A8
:103CD000991323F4F853C1F81035D1F810E52302F5
:103CE00003F47C53120402F4403243EA0E031343FC
:103CF0002A0502F4801240EA4C30134340F02000C1
:103D000026F81700C1F81035C0E70348BFE700BF29
:103D1000300000200000AD0B0400AD0B014BC3E9E7
:103D2000020170473000002008B50246FFF766FE2A
:103D300038B1054B0548083233F812305B0B0B7075
:103D400008BD0348FCE700BF300000200000AD0BB9
:103D50000400AD0B38B50F4C94F87850BDB9602213
:103D6000294604F1100002F046FC0620FDF7D0FEC3
:103D7000094B0A48C3F87C51D3F87C214FF000422C
:103D8000C3F80423012384F87830636738BD0448FE
:103D9000FCE700BF30000020006000400000AD0BD9
:103DA0000500AD0B034B93F87800003818BF0120D5
:103DB000704700BF3000002001460148FFF756BDA4
:103DC000A000002001460148FFF72ABDA000002006
:103DD00037B50446FFF712FE04F108021E4B33F814
:103DE0001230E8B113F002051AD15B0B9A0002F110
:103DF000804000F5C24002F1804202F5C0420560F9
:103E00000068D2F8100540F00100C2F8100529B191
:103E1000012202FA03F3114AC2F8043303B030BDA1
:103E2000C3F38203042B12D0052B12D001A80194F6
:103E3000FFF7D6FD019BD0F81015D94001F0010124
:103E40000231204603B0BDE8304002F0F9BF032143
:103E5000F7E70221F5E700BF3000002000600040D6
:103E600008B50246FFF7CAFDC0B102F108010E4BCA
:103E700033F81130990711D45B0B01229A409B0053
:103E80000A4903F1804303F5C043C1F80823D3F87E
:103E9000102522F00302C3F8102508BDBDE8084034
:103EA0000021104602F0CCBF30000020006000402E
:103EB0000E4B00F1080213B533F81230DB0704464D
:103EC00011D5FFF7CDFF2046FFF7ECFD01A80194C7
:103ED000FFF786FD019B03F5E073022240F82320E3
:103EE000034802B010BD0348FBE700BF30000020CC
:103EF0000000AD0B0400AD0B2DE9F04F644B65489D
:103F00006549002687B0012234461D6835B1D0F8D6
:103F1000045315421EBF1C601D68164304338B42B8
:103F20004FEA4202F1D1DFF86C81D8F87C31002BE6
:103F300000F091804FF0A043D3F820250492C3F8FD
:103F40002025D3F820280592C3F8202800270DF15A
:103F500010097B0100934FF0010A49E0009B4F4A92
:103F600094FAA4F4B4FA84F41C4404F10803E008BD
:103F700032F81330039404F007020AFA02FC19F82D
:103F8000002022EA0C0209F8002003A8C3F38205EE
:103F90009908FFF725FD039A02F5E0724B0750F8E8
:103FA0002220AB46C2F3014229D520465946D5B25C
:103FB000FFF72EFD03A80394FFF712FD039B03F503
:103FC000E07350F82330C3F301439D4207D1002131
:103FD000204602F035FF2946204602F031FF03A8B3
:103FE0000394FFF7FDFC039B0AFA03F3C0F82035A6
:103FF00059F82740002CB1D1CFB90127A9E7022AEF
:104000000CBF032102212046019202F019FF032D6B
:1040100004D0019A022A06D1012DE0D1594620464A
:10402000FFF7F6FCDBE7032AD9D1022DF5E7C8F844
:104030007C41D8F87C311A494FF0A043D3F82025B1
:104040000492C3F82025D1F820350593C1F8203516
:1040500013437FF47BAF012416B907B0BDE8F08F9E
:1040600096FAA6F3B3FA83F304FA03F29B0003F182
:10407000804303F5C04326EA0206D3F81005D3F8BF
:104080001015C0F30520C1F30141FFF7C1FCE3E7C0
:1040900000610040006000402061004030000020CE
:1040A00000030050044AD2F80034DB07FBD501605E
:1040B000BFF35F8F704700BF00E001404FF08053B7
:1040C0001A69B0FBF2F302FB130373B9084B022227
:1040D000C3F80425C3F80805D3F80024D207FBD59C
:1040E00000220448C3F8042570470348704700BF06
:1040F00000E001400000AD0B0A00AD0B10B5054C0F
:104100000123C4F80435FFF7CDFF0023C4F80435BC
:1041100010BD00BF00E001400E4B70B553F82040C9
:10412000013053F82060A64200D870BDD4E90035B4
:104130002846984765B1EB6830B10028B8BF4042C7
:10414000FF28A8BFFF2018705A7842F001025A7069
:104150000834E8E7BC73000070B5054610B90024C8
:10416000204670BD0378002BF9D00E4C0E4EB442A1
:1041700008D10C4CB442F2D0204602F07FFE50B978
:104180001834F7E7204602F079FE10B12368AB42FD
:10419000E6D01834EBE72168284602F004FA00283C
:1041A000EED1DDE7646F0000F46F000073B50446E4
:1041B0000D464FF02003EFF3118683F31288BFF30F
:1041C0006F8F042896BF124B124B53F820300022F9
:1041D000009245210246104802F03DF93DB1EB69DD
:1041E000C3F308031BB10D48452102F034F90C4B11
:1041F0000C480022452102F02EF929462046FFF7FF
:1042000009F986F31188BFF36F8F02B070BD00BF4C
:10421000D0730000B3800000C1800000EE80000079
:10422000148100001C81000008B5094B0122022006
:104230001A70FFF771FF02F039FE0320FFF76CFFE1
:10424000FCF7CEF8034A137B23F00103137308BD78
:10425000071000205001002008B50348034A002140
:10426000121A02F015FE08BD3001002008100020CF
:1042700008B5194B83F30888184C636943F400733D
:1042800063610025E02384F82230E57725766576A2
:10429000A57684F82050636A43F4E023636284F8CF
:1042A0002350FDF7D5FEFDF7E7FB4FF0FF33A36288
:1042B000E362FDF7D3FFFDF757FF02F0DEFD28466E
:1042C000FFF72AFF0120FFF727FF05482B462A4664
:1042D0002946FDF7ABFC00BF6040002000ED00E088
:1042E0002942000008B50648064A0749121A02F09A
:1042F000D1FDBDE80840054A0549064802F0CABD9F
:10430000000000202C010020888100000000000037
:104310008881000000000020034B1B680BB9FFF7E9
:1043200043B80020704700BFE80E00200D4B10B5C9
:104330001C689C4208BF0024FFF7EEFF74B1D4E96B
:1043400004321B1A62EBE070B3F1004F70F100020F
:1043500004DA0028ACBF1846002010BD6FF0004002
:10436000FBE700BFAC00002030B5036868B10A4A23
:104370005268904209D043B1D3E90421D0E9044501
:10438000121941EB0501C3E90421426813605A6028
:104390000023C0E9003330BDAC0000202DE9F84314
:1043A0004FF02003EFF3118483F31288BFF36F8F74
:1043B000234EDFF89480234D3060D8F80000326837
:1043C0004045D5E9001E4FEAE2770BD050B1D0E965
:1043D000043C9A4277EB0C0916DA9B1A6CEB070C3B
:1043E000C0E9043C52184EEB0707C5E90027002539
:1043F0003560FFF79BFF2946FEF7A4FF84F3118881
:10440000BFF36F8FBDE8F88359184EEBE377D31AEB
:10441000336000220023C0E90423C5E90017FFF739
:10442000A3FF84F31188BFF36F8F836898474FF021
:104430002003EFF3118483F31288BFF36F8FBCE77F
:10444000E80E0020D0010020AC00002010B50A4C7E
:1044500023681BB101232360002010BD00F052F837
:104460000028F7D00138062803D8044B53F8200061
:1044700010BD034810BD00BFEC0E0020E473000027
:10448000FE8FFFFFBFF34F8F0549064BCA6802F44A
:10449000E0621343CB60BFF34F8F00BFFDE700BF67
:1044A00000ED00E00400FA0510B40A4B0A490B4C79
:1044B0004FF0FE32C3F800244968C3F80424C3F85F
:1044C0000824C3F80C240023C4F800355DF8044B1D
:1044D000084700BF00B00250B400002000A0025006
:1044E000D0E90012014BC3E900127047B40000206C
:1044F00038B131B1014400220346013088421A70BC
:10450000FAD1704738B500F02FF820B1032400F03D
:1045100063F8204638BD00F031F898B900F0ACF8E7
:1045200098B90F4DD5F828391B0EF02B08D1D5F8C6
:10453000242A0C4B9A420AD0072400F017F8E6E729
:104540000624FAE70424204638BD0024F5E70120BC
:1045500000F092F804460028F7D1C5F80C0AD8E715
:1045600000B002500000E02000207047002070479B
:10457000014BC3F8040A704700B0025010B511484F
:1045800000F048F800B110BD0F4800F043F80028D3
:10459000F9D10E4C204600F03DF80028F3D10C4B29
:1045A0000C481C6000F036F801460028EBD100F002
:1045B0002DF8044608B1204610BD00F03FF8204613
:1045C000FAE700BFC8000020BC000020C4000020A3
:1045D000CC000020C000002008B5084800F024F8F6
:1045E000074800F021F8074800F01EF8064800F0E0
:1045F0001BF8BDE8084000F00BB800BFC800002061
:10460000BC000020C4000020C00000200020704733
:10461000704700BF08B5034B02681B6810689847D5
:10462000002008BDD800002008B5034B02685B6875
:1046300010689847002008BDD800002070B5094CCC
:10464000094D2069AB68984718B1084B08485B686A
:104650009847084AEB68206900211160BDE8704066
:10466000184700BFE8000020D8000020B400002058
:1046700000740000F00E002070B51B4D1B4E044668
:10468000B26828699047F8B95CB1194C2368B3B196
:10469000012B1BD0013B23602869F3689847002059
:1046A00070BD134C216841B9124B0122C3F800259B
:1046B000114AD2F81039002BFBD101312160F36887
:1046C00028699847002070BD0C4870BD0A4AD2F88E
:1046D0001039002BFBD1074A6FF07E40C2F800353D
:1046E000FFF746FF2368D5E7E8000020D800002048
:1046F000F00E002000A0025000B00250E98FFFFF32
:1047000010B5044630B16368DB0602D50023236090
:10471000636010BD024B03485B689847F3E700BF36
:10472000B400002020740000B0B1436893B1DB06F0
:104730000ED5012350E8002F194640E8001C9CF0DC
:10474000000FF7D1012AF5D0BFF35F8F002070472B
:1047500003487047034870476FF4E040704700BF5C
:10476000E98FFFFFEA8FFFFF68B143683BB1DB06CB
:1047700007D5BFF35F8F00230360184670470348D7
:104780007047034870476FF4E0407047EA8FFFFFBF
:10479000E98FFFFF10B5044620B1002211232260EB
:1047A000636010BD0148FFF77FFEF6E74874000024
:1047B00030B10268034B04489A4208BF002070479A
:1047C00002487047DD55AABB8208F0007108F0006E
:1047D00038B50D460446B0B1A0220021043002F0E5
:1047E0007FFB95B10822294604F1640002F07EFBAC
:1047F000082205F1200104F1840002F077FB044B4C
:104800002360002038BD0348FCE70348FAE700BFF7
:10481000DD55AABB7108F0008308F0002DE9F743CD
:1048200005460E4699461146FFF7C2FF044600288A
:1048300040F08480002E00F08580002900F0848004
:10484000B9F1200F40F0828005F14404082205F1FF
:104850000408204602F04AFB05F1240708223146ED
:10486000404602F043FB06F120010822384602F0E0
:104870003DFB02A94FF4807041F8049D02F02AFB31
:10488000002865D1334A4FF480731360012193608F
:104890000823314A00F02EFB0121084605232F4A48
:1048A00000F028FB0823424601211C2000F022FBD7
:1048B00008233A460121032000F01CFB224608236E
:1048C0000121022000F016FB0823254A01211A20AD
:1048D00000F010FB0523234A01211B2000F00AFBF6
:1048E0000823214A0121142000F004FB08231F4A59
:1048F0000121152000F0FEFA082305F164020121D0
:10490000162000F0F7FA082305F184020121172090
:1049100000F0F0FA0823164A01210B2000F0EAFA11
:1049200000F044FB0446019800F0D2FA114B002C31
:1049300018BF1C46A421284602F0D4FA204603B032
:10494000BDE8F0830C4CF9E70C4CF7E70C4CF5E7AD
:10495000084CEFE790B00250AC74000024750000E2
:104960006C74000010750000D0740000F07400003A
:104970008C7400008408F0007608F0008008F000D5
:104980008108F0000C4BC2691A60826943F8042C5C
:10499000426943F8082C026943F80C2CC26843F8BA
:1049A000102C826843F8142C426843F8182C0268D3
:1049B00043F81C2C704700BF5CB602500C4B1B68C0
:1049C000C3610C4B1B6883610B4B1B6843610B4B32
:1049D0001B6803610A4B1B68C3600A4B1B6883603A
:1049E000094B1B684360094B1B680360704700BF9D
:1049F0005CB6025058B6025054B6025050B602503F
:104A00004CB6025048B6025044B6025040B602506E
:104A100030B10268034B04489A4208BF0020704737
:104A200002487047DD55AABB0202F0000002F00008
:104A300038B5044668B1051D7021284602F052FAC7
:104A400028462022044902F049FA044B2360002042
:104A500038BD0348FCE700BF38750000DD55AABB30
:104A60000002F0002DE9F043284B04460E4615469F
:104A70000FCB85B06F4687E80F002DB94FF00009C6
:104A8000484605B0BDE8F0832046FFF7C1FF8146E8
:104A90000028F5D1231D0193636AA3BB236F8BB15B
:104AA000C3F14008A84528BFA84604F130003146AC
:104AB0001844424602F012FA236F434446442367E7
:104AC000A5EB0805226F402A06D104F130013846D3
:104AD00000F0AEFB0023236705F03F0835F03F05EB
:104AE00005D031462A46384600F0A2FB2E44B8F1E4
:104AF000000FC3D04246314604F1300002F0EEF917
:104B0000C4F87080BCE7DFF80890B9E7E0710000F6
:104B10000C02F0002DE9FF41144B04460E460FCB6A
:104B20006F4687E80F002046FFF772FF8046B0B956
:104B3000CEB1636A251D01953BB901236362226FE3
:104B400004F13001384600F073FB2B46043E243458
:104B500053F8042B12BAA34246F8042FF8D140466A
:104B600004B0BDE8F081DFF80880F8E7E0710000EC
:104B70000502F000084B1B681B0EF02B08D1074BF9
:104B80001A68074B9A4205D1064B002018607047FF
:104B9000052070470620704728B9025024BA0250F9
:104BA0000000E0200CBA0250002230B54900134644
:104BB000023840F6FC7502F1A05404F52C44A40020
:104BC000904202F10102CABF236025605B181E2AD1
:104BD000F1D1044A13600B445360034B034A1A603B
:104BE00030BD00BF78B0025084B0025020F80F00F2
:104BF00030B51E4B85B01A46196800910099CC0754
:104C0000FAD500F1A05000F52C408000016813682F
:104C10000193019BD807FAD5154B164C1868164D11
:104C20001F30202390FBF3F00138002810DA002316
:104C30000130400153B1A0F120014FF00042134276
:104C400004D1013888424FEA5202F8D105B030BD94
:104C500013680393039BDB07FAD5431823602B6883
:104C60000293029B002BE3D10138DEE7B4B002507F
:104C7000ACB00250E4B00250DCB00250F0B51D6898
:104C800085B001F01F040DB91F2C25D1154D2E46FE
:104C90002F680197019FFF07FAD500F1A05000F59A
:104CA0002C408000006835680395039DED07FAD518
:104CB0000D4D00EB611028600C48006802901F2C1D
:104CC00018BFC94302980FBF106001F01F0100FA1E
:104CD00001F111600021196010684300C00F1360DA
:104CE00005B0F0BDB4B00250E4B00250DCB00250E8
:104CF0000C4B18603F3020F03F0089014030586075
:104D00009960D9601961596199611C33064819602D
:104D100082B002680192019AD207FAD5196002B0F6
:104D2000704700BF90B00250B4B0025038B5A0F147
:104D30002003B3F5426F05462CD88F2826D800F102
:104D4000470300F16604DB064FEA541400D0013437
:104D500064013F34A409013411B1A1421AD30C46B5
:104D6000E3004FF48050B0FBF3F0202828BF202050
:104D700002B11060084B01221A602146FFF714FFB0
:104D800028462146FFF7B4FF002038BD00F11F047C
:104D90006409DDE70148F8E71CB802502221F00061
:104DA000F0B5454B89B01D461C680194019CE40791
:104DB000FAD5424BDFF80CE1DFF80CC113449B003D
:104DC00000241A680B181E2B88BFC0F11E011F3269
:104DD0000B1852095343B3F5806F82BF4FF48061C3
:104DE000B1FBF2F1091A00F1A05000F52C40274662
:104DF000A14233DC2B680493049BDB07FAD5304BCC
:104E00001B68296805910599CF07FAD52D4C2E49C5
:104E1000236000231E46934203F1010040D120F09D
:104E200001022948194600268A423CD82968069181
:104E30000699CE07FAD5254909682868079007988A
:104E4000C007FAD52160204800210C468B422DD1A5
:104E50001D4900209A422CD809B0F0BD2B6802935E
:104E6000029BDB07FAD503199B001B682E6803968B
:104E7000039EF607FAD5CEF800300023934203F1E3
:104E8000010306D1164623F00103B34204D80134CE
:104E9000AEE7CCF80070F1E7CCF800700136F4E72B
:104EA0000E600346B7E706600131BDE704600131DB
:104EB000CCE708600133CDE7B4B0025024AC001455
:104EC0007CB00250D4B00250D8B0025078B002503A
:104ED00008B540B1202801464FF0070228BF202125
:104EE0000020FFF75DFF024B00221A6008BD00BFE3
:104EF0001CB80250F0B5294D85B02C462E6800969E
:104F0000009EF607FAD500F1A05000F52C40800075
:104F10000568206801900198C707FAD52048214FFD
:104F2000056002EB8306B24229D15A1C1D4E22F0C5
:104F3000010200279A4227D823680293029BDE07CA
:104F4000FAD5194B0B449B001B681F335B099A422F
:104F500013D2216803910399C907FAD5154400219A
:104F60009B1A104A056008468B4210D85A1C0D49FE
:104F700022F0010200209A420CD805B0F0BD52F890
:104F800004CBC7F800C0CEE737600133D2E710602A
:104F90000131E9E708600133EDE700BFB4B002502A
:104FA000D4B00250D8B0025024AC00142DE9F04126
:104FB000814B1D6898682033A0B01E461A68019284
:104FC000019AD707FAD57D4B7D4A1A603268029262
:104FD000029AD407FAD57B4A1A607B4A14461168B4
:104FE00003910399C907FAD5784A1168C1F34021A2
:104FF00037680497049FFF07FAD5754F1F6027682D
:105000000597059FFF07FAD51768002900F0CF80A4
:10501000B90540F1CC80316806910699CF07FAD5E1
:105020006C491960216807910799C907FAD5116879
:10503000C1F3402137680897089FFF07FAD5664FEC
:105040001F6027680997099FFF07FAD51268002992
:1050500000F0AF80910540F1AC8032680A920A9A64
:10506000D207FAD5564A1A6032680B920B9AD707C4
:10507000FAD55A4A1A6031680C910C99CC07FAD5C6
:105080005749196031680D910D99C907FAD55549ED
:10509000196031680E910E99CF07FAD552491960FF
:1050A00031680F910F99CC07FAD550491960504BD0
:1050B0001E46196810911099C907FAD53F4C4D4BFF
:1050C000236033681193119BDB07FAD54A4B2360A9
:1050D00033681293129BDF07FAD5484B23603A4B93
:1050E0009846196813911399C907FAD5324F386059
:1050F00033681493149BDB07FAD522603368159349
:10510000159BD807FAD53E4B236033681693169B40
:10511000D907FAD53B4B236033681793179BDA07FF
:10512000FAD5394B236033681893189BDB07FAD5FF
:10513000364B236033681993199BD807FAD5344B43
:10514000236033681A931A9BD907FAD5314B236031
:1051500033681B931B9BDA07FAD52F4B236000F0B3
:105160001DFC08BBD8F800301C931C9BDB07F9D54D
:105170003D6033681D931D9BD907FAD5274B2360EB
:1051800033681E931E9BDA07FAD5254B2360D8F8A7
:1051900000301F931F9BDB07F9D50C4B1B6813F4E2
:1051A000805F204B08BF184620B0BDE8F0811E4844
:1051B000FAE71E48F8E700BF90B0025080B00250F6
:1051C00000100251C01F7229B4B0025088B00250C2
:1051D000C0CF0129C01F0E29C03F0029400102494C
:1051E000003184A800001649400108A180440888C5
:1051F000B0B00250C044708880077A41C0077E4139
:1052000000006A498006164940006E4900020021EC
:1052100000822021408220218082242140A161A19E
:1052200000C861510308F1000108F1000208F10013
:105230002DE9F74F314B44688046924699461A68EB
:10524000002AFCD12E4B9B461A68002AFCD14FF055
:10525000FF30019100F094FC802000F097FC294D74
:10526000294A2A4F2A4E012307202B60A2F59E725D
:10527000C2F83C011360636A3B60A36A3360D8F8EC
:10528000003042F8043CD8F808302046984701998D
:10529000D9F80030002BFBD1BAF1000F20D11D4B03
:1052A00004221A60D9F80030002BFBD1DBF800A0F3
:1052B000BAF1000FFAD1D8F80C30204698473B6875
:1052C00063623368A362144BC3F800A0C3F844A11F
:1052D000D9F80030002BFBD12B6003B0BDE8F08F74
:1052E000236A012B04BF0C4A13600C4B4020196049
:1052F000C3F804A000F050FCD4E700BF10B902507E
:1053000020BC025018B8025000B90250CCB702506D
:10531000D0B70250C8B7025084B6025028BC025021
:1053200010B5544B98B019461A680192019AD207E9
:10533000FAD5514B514A1A600A680292029AD40770
:10534000FAD54F4A1A600A680392039AD007FAD531
:105350004C4818600A680492049AD207FAD54A4A5F
:105360001A600A680592059AD407FAD5474A1A6066
:105370000A680692069AD207FAD5454A1A600A6860
:105380000792079AD407FAD5424A1A600A68089227
:10539000089AD207FAD5404A1A600A680992099A0F
:1053A000D407FAD53D4A1A600A680A920A9AD207C7
:1053B000FAD53B4A1A600A680B920B9AD407FAD5C1
:1053C000384A1A600A680C920C9AD207FAD5364A03
:1053D0001A600A680D920D9AD407FAD5334A1A60FA
:1053E0000A680E920E9AD207FAD5314A1A600A68F4
:1053F0000F920F9AD407FAD52E4A1A600A681092B3
:10540000109AD207FAD52C4A1A601A4B19461C6812
:105410001194119CE407FAD5174B18600868129094
:105420001298C407FAD51A600A681392139AD00723
:10543000FAD5124A1A600A681492149AD207FAD559
:105440001E4A1A600A681592159AD407FAD51C4AA2
:105450001A600A681692169AD007FAD5194A1A6085
:105460000A681792179AD207FAD5174A1A6018B025
:1054700010BD00BFB0B0025080B002500093652153
:1054800000043190409665900083612100C3302173
:1054900000C36490008161900046102100811121B9
:1054A0000041442100C320290C4610C80086312148
:1054B00000C3602140C12829409665210013319026
:1054C00040962529594614C84004324910B5494B25
:1054D00094B019461A680092009AD207FAD5464B42
:1054E000464A1A600A680192019AD407FAD5444ADA
:1054F0001A600A680292029AD007FAD541481860E9
:105500000A680392039AD207FAD53F4A1A600A68DA
:105510000492049AD407FAD53C4A1A600A680592A4
:10552000059AD207FAD53A4A1A600A680692069A8C
:10553000D407FAD5374A1A600A680792079AD20741
:10554000FAD5354A1A600A680892089AD407FAD53B
:10555000324A1A600A680992099AD207FAD5304A83
:105560001A600A680A920A9AD407FAD52D4A1A6074
:105570000A680B920B9AD207FAD52B4A1A600A686E
:105580000C920C9AD407FAD5284A1A600A680D9230
:105590000D9AD207FAD5264A1A600A680E920E9A18
:1055A000D407FAD5234A1A600A680F920F9AD207D5
:1055B000FAD5214A1A600F4B19461C681094109CAA
:1055C000E407FAD50C4B1860086811901198C407CD
:1055D000FAD51A600A681292129AD007FAD5174AB9
:1055E0001A600A681392139AD207FAD5144A1A60FD
:1055F00014B010BDB0B0025080B002508090652150
:1056000000040990409665908080612180200821E7
:10561000802064900081619000461021008111215A
:105620000041442180202029024610C8008609211B
:105630008020602140212829409665214096252917
:10564000594614C810B5504B96B01C461A680192C2
:10565000019AD207FAD54D4B4D4A1A602268029240
:10566000029AD207FAD54B4A1A604B4A42EA804066
:1056700022680392039AD207FAD51860226804922E
:10568000049AD007FAD5454A1A60A2F5800242EA88
:10569000814122680592059AD207FAD519602268DD
:1056A0000692069AD007FAD53D4A1A6022680792F8
:1056B000079AD107FAD53B4A1A6022680892089ADD
:1056C000D207FAD5384A1A6022680992099AD00797
:1056D000FAD5364A1A6022680A920A9AD107FAD590
:1056E000334A1A6022680B920B9AD207FAD5314AD4
:1056F0001A6022680C920C9AD007FAD52E4A1A60CA
:1057000022680D920D9AD107FAD52C4A1A602268A8
:105710000E920E9AD207FAD5294A1A6022680F9281
:105720000F9AD007FAD5274A1A602168109110996C
:10573000C907FAD51A60144B1A46196811911199C4
:10574000C807FAD5114B20491960116812911299B6
:10575000C907FAD51D491960116813911399CC072F
:10576000FAD50B491960116814911499C807FAD534
:1057700017491960116815911599C907FAD5154A85
:105780001A6016B010BD00BFB0B0025080B0025019
:105790004004419000862929D81001C84014419046
:1057A00040142129401465210034409000310C90B0
:1057B000C0400C90C030202940960D900041609070
:1057C000031645C80086112100416021594644C88E
:1057D0004014459040142D9070B5264888B0054679
:1057E00004680094009CE607FAD52348234C046023
:1057F000234C44EA83432C680194019CE407FAD5C6
:105800000360930143EA824242F0104444F4C044EE
:105810002B680293029BDE07FAD504602B68039382
:10582000039BDB07FAD5174B03608B0143EA8141E9
:1058300041F0104343F4C0432E680496049EF607DB
:10584000FAD503602B680593059BDE07FAD5046043
:1058500041F058412B680693069BDC07FAD501609E
:1058600042F058422B680793079BDB07FAD502608A
:1058700008B070BDB0B0025080B00250C021022903
:105880008071009880611890354B8EB019461A6867
:105890000092009AD207FAD5324B334A1A600A684E
:1058A0000192019AD007FAD5304A1A600A6802922A
:1058B000029AD207FAD52E4A1A600A680392039A0E
:1058C000D007FAD52B4A1A600A680492049AD207C4
:1058D000FAD5294A1A600A680592059AD007FAD5BE
:1058E000264A1A600A680692069AD207FAD5244A0E
:1058F0001A600A680792079AD007FAD5214A1A60F7
:105900000A680892089AD207FAD51F4A1A600A68EC
:105910000992099AD007FAD51C4A1A600A680A92B5
:105920000A9AD207FAD51A4A1A6008680B900B989F
:10593000C007FAD51A600A680C920C9AD007FAD5FB
:10594000144A1A600A680D920D9AD207FAD5124AC3
:105950001A600E210D230F2200200EB0FFF73CBF6E
:10596000B0B0025080B00250804301294063392119
:10597000807001298020542100D13490C04034909F
:10598000C0302029C0530D9000413890832308C8AF
:1059900080E3102100413821CF4308C82DE9F041B0
:1059A000012392B0CDE90333624B1D461A6805927C
:1059B000059AD207FAD5604C604B2360604B1946BC
:1059C0001A680692069AD707FAD55E4B1A68D6046B
:1059D00000F1A8802A680792079AD007FAD55A4A98
:1059E00022600A680892089AD207FAD51E68C6F3A0
:1059F0000036002E40F098801220FFF7F9F8074695
:105A00001320FFF7F5F887428CBF12201320FFF711
:105A1000EFF8471EFFF738FF03AB01AA3946122003
:105A2000FFF72CF904AB804602AA39461320FFF792
:105A300025F900EB4800022832D003283ED0012887
:105A400074D12B680993099BDB07FAD53F4B236080
:105A50002B680A930A9BD807FAD53D4B23602B6825
:105A60000F930F9BD907FAD53A4B23602B681093FD
:105A7000109BDA07FAD5384B23602B681193119BE2
:105A8000DB07FAD5354B2360013F25D510231922BA
:105A900018210020FFF7A0FE304612B0BDE8F081CB
:105AA0002B680B930B9BD907FAD52D4B23602B68E2
:105AB0000C930C9BDA07FAD52A4BCFE72B680D9392
:105AC0000D9BDB07FAD5284B23602B680E930E9BAA
:105AD000D807FAD5254BC1E703AB01AA39461220F6
:105AE000FFF7CCF804AB044602AA39461320FFF7AF
:105AF000C5F810EB440402D1FFF712FCC4E7FFF72E
:105B0000E5FC022C08D0032C09D0012C10D1172160
:105B10001620FFF797FDB7E715211420F9E70F21AD
:105B20000E20F6E7124EB7E7124EB5E7124EB3E776
:105B3000124EB1E7B0B0025080B0025000084A5196
:105B4000B4B0025088B0025000084E5100065A49C5
:105B500040065E49000442410014424940042E4977
:105B6000000652494006564900063A4940063E4959
:105B70000608F1000708F1000408F1000508F1002B
:105B8000014B1860704700BF08BA0250014B186003
:105B9000704700BF04BA0250034A13681842FCD091
:105BA000024A10601846704700BA025008BA025004
:105BB000704729B1012914BF6FF015000520704707
:105BC000022070470020704770472DE9F7430E46CA
:105BD00017469946044628B94FF0FF38404603B0AF
:105BE000BDE8F0830029F7D0002AF5D0CB680D89F5
:105BF0001D4404230DEB03022946384600F039FC0E
:105C000080460028E8D1BDF80410738946F60812D2
:105C1000914223D1BDF806109942DDD104230DEB4A
:105C200003022944384600F024FC0028D4D1BDF8F2
:105C3000042046F607139A42CED19DF82830A3726D
:105C40007389BDF80620A4F808902B44E36004355E
:105C50001344C4E9006763612561BFE7002BE6D008
:105C6000BAE72DE9F7430F4690461E46044620B991
:105C70004FF0FF3003B0BDE8F0830368002BF7D08E
:105C80004368002BF4D04FF6FF79D4E904239A42FD
:105C900016D223685B8923B1E368934204BF0433BF
:105CA00023610423216960680DEB030200F0E1FB2E
:105CB0000028DDD1A37A256923B1E368AB4201D87E
:105CC0000120D7E72189BDF80620494502F10403E8
:105CD00003D0BDF804C08C450BD116B1BDF804103B
:105CE000318004353D60A8F8002022691344236107
:105CF000C0E72B442361C8E773B50C46064611463E
:105D0000022301AA204600F03EFA0546E8B9019AAE
:105D10001F2A0ED92368A2F12001194420223046FF
:105D200000F05EFC2368019A13442360284602B009
:105D300070BD0146C2F12002304600F05CFC019AC1
:105D40002168C2F120003044EAE76FF00205EDE778
:105D500000F035BC4FF4C0735843303070470B78B7
:105D6000022B06D0052B0CBF4FF4C0704FF0FF3054
:105D700070474FF4C070704710B5044600F0C8FB80
:105D8000A3684FF4C072303B02FB103010BD816835
:105D9000183921F007010122083900F076BF13B548
:105DA0000446019100F00EFF0423A0F108010DEB61
:105DB0000302204600F03DFF02B010BD73B513464C
:105DC00001920E46024600210546FAF7A9FF044655
:105DD00050B9019B05F12C0201212846FAF7A0FFDA
:105DE00010B1002E18BF0446204602B070BD73B536
:105DF000054600200C461646FFF7DBFE6946C0B29A
:105E0000FBF7E2FD30BB2C2101FB045400982189F3
:105E1000E368CD1804230DEB0302294600F029FBAB
:105E2000C0B9BDF80420648946F608139A4216D119
:105E3000BDF806309C420DD1042300980DEB0302FF
:105E4000611900F016FB28B9BDF8042046F60713C7
:105E50009A4207D0009800F00BFB02B070BD002CF6
:105E6000F2D0F7E7BDF80610214429443160F1E78C
:105E700037B5426A0446802501A902200195FBF747
:105E8000C1FD58B9019B226DA36201A905200195AE
:105E9000FBF7B8FD054628B1092500E00125284695
:105EA00003B030BD019B206A636500F031FBE06503
:105EB000F5E70123036003F1012343600023C0E9F8
:105EC000023370474379012B07D10368012B04D1BA
:105ED0000079431E5842584170470020704770B502
:105EE00086B006460D46022003A9FBF76DFD30BBC8
:105EF0000398FFF741FFF16D0446284600F0E4F8EF
:105F00000444039800F004FB0190039800F009FB9F
:105F10000822014604A800F06EFB2A798DF81020B3
:105F20002146019B039804AA00F0BFFA041E0398BF
:105F300018BF012400F09CFA204606B070BD012471
:105F4000FAE700F0CEBA2DE9F8430E4600210746E5
:105F50000846FFF72EFE012104460020FFF729FE28
:105F600033789C4221D0984221D101252C2303FB78
:105F70000575F86DAC6AFFF7EDFE013C07464FF082
:105F800000086B6A03EBC40253F83410D2F8049093
:105F90001B684A46C91A3046C844FFF7D2FFB845C5
:105FA00004F1FF34EDD3BDE8F8830025DEE70120DE
:105FB000F9E737B515460C460520694600F07CFE2A
:105FC000E979012903D00022204600F089FE9DF8DE
:105FD0000330012B02D1204600F061FEA968204663
:105FE000FFF7DDFE2046FDF71FFA002003B030BDAD
:105FF00073B50D460646FAF77BFF0446E86050B3DA
:1060000002282DD101A9FBF7DFFC58BB01982A46D5
:106010003146FAF7D3FE0446D0B9019800F0D2FD1C
:10602000012301460DF10302019800F022FA044613
:10603000A0B9019801220DF1030100F0D7FD10B1C4
:1060400001238DF803309DF8033003F00F03EB714B
:10605000019800F00DFA204602B070BD0124F7E768
:106060000724F8E70124F6E713B5022001A9FBF79E
:10607000ABFC48B90198FFF78AFE0446019800F08E
:10608000F7F9204602B010BD0124FAE71FB502203F
:1060900001A9FBF799FCA8B9019802A9FDF7E4F959
:1060A000044668B99DF80B30032B03D1019800F02A
:1060B000F6FD0446019800F0DBF9204604B010BD5F
:1060C0000124F7E70124F8E730B543790279012B81
:1060D0000CBF0123022301FB03F4036803F1FF3328
:1060E00002F1FF3204FB03F314BFCD01002501FBD5
:1060F0000231481930BD036870B5CD1A002D0DDD91
:1061000093F900601C78002E0BDB5C1C04601B788C
:1061100013600368C91A13688B4232D96FF05F00AD
:1061200070BD04F07F04013C032C27D8DFE804F0A5
:106130000209121E012DF1D05C7814600233036055
:10614000E7E7022DEADDB3F8014064BAA4B21460B7
:106150000333F4E7032DE1DD9C785D78240244EA03
:106160000544DD782C4314600433E8E7042DD5DDC5
:10617000D3F8014024BA14600533E0E76FF0630000
:10618000CEE70020CCE770B404680E1B002E07DDBC
:1061900026789E4208D10134046070BCFFF7ABBF83
:1061A0006FF05F0070BC70476FF06100FAE738B5C0
:1061B00003230446FFF7E7FF18B9136813B96FF01C
:1061C000670038BD013B136023681A78002AF6D1B6
:1061D00001332360F5E72DE9F74390461F4601AAF6
:1061E000302305468946FFF7CEFF0446F8B92E68EE
:1061F000A9EB0609B9F1000F35DD01993378424664
:106200000E4442F8043B314606232846FFF7BBFF05
:10621000044660B92A68D8F80410C8F80820531852
:10622000B3422B6007D10C213846FEF761F92046B6
:1062300003B0BDE8F083515C3A46013342F8041BD9
:1062400028462B603146FFF756FF04460028EED162
:106250002B687A68BB601344B3422B600CBF0446C2
:106260006FF06504E3E76FF05F04E0E7F8B5B1F1C4
:10627000005F00AF0546144610D2D31D23F007037C
:106280006E46ADEB030D684600F0AAF9694622465A
:106290002846FEF7E7FBB546BD46F8BDFEF7E2FB34
:1062A000FAE760B1436803F00303012B03D0032B2B
:1062B00005D103681BB100238360184670476FF057
:1062C000150070474368816003F00303032B4FF010
:1062D00000020CBF03681346426018467047002056
:1062E00070470FB407B504A951F8040B0191FBF7EF
:1062F00037F803B05DF804EB04B07047038B13F07C
:10630000070305D10368002B0CBF00200320704752
:10631000022B05D1438B002B14BF002004207047B3
:10632000012B05D10368002B0CBF0020052070470E
:106330000020704773B50D4606461946281D019288
:106340000093FFF7BFFF044640B1DDE90032294664
:106350003046A44602B0BDE87040604702B070BD50
:1063600010B44FF02004EFF3118284F31288BFF3CE
:106370006F8F41615DF8044B0121FAF7FFBF10B543
:106380000C4640B139B1081DFFF78BFF28B9A3684F
:1063900033F0030301D06FF0150010BD38B50C4683
:1063A000054658B151B10B6843B14B6833B11C225B
:1063B000002100F020F92C61002038BD6FF015009D
:1063C000FBE770B504460E46FFF7D9FF051E31DB2B
:1063D0004FF02003EFF3118183F31288BFF36F8F27
:1063E000638B208B4FF6FF75AB4200F007022ED077
:1063F000022A0ED1013363831546012381F31188EC
:10640000BFF36F8FB3B1002331462046FFF792FFF1
:1064100010E0830701D0062A0ED1002333606368A1
:1064200093B9C4E90066154662B90A4620460221BE
:10643000FAF7A4FF284670BD052A0CBF6FF085054A
:106440006FF004050023D9E71E606660EBE76FF08C
:106450000A05F7E770470FB407B504A951F8040B14
:106460000191FAF77DFF03B05DF804EB04B07047CB
:10647000704773B50C1E054601921E4611DB8168FC
:10648000E3188B420DD8C068FDF766FE69682144A9
:106490008368019A1C683346A44602B0BDE8704088
:1064A00060476FF0150002B070BD73B50C1E054655
:1064B00001921E4611DB8168E3188B420DD8C0683B
:1064C000FDF74AFE696821448368019A5C68334697
:1064D000A44602B0BDE8704060476FF0150002B0FE
:1064E00070BD70B50C1E054616460EDBA3188268FB
:1064F00093420AD8C068FDF72FFE6968214483687B
:1065000032469B68BDE8704018476FF0150070BDBB
:1065100008B5C068FDF720FE8368DB68984700680F
:1065200008BD08B5C068FDF717FE8368DB689847AB
:10653000007908BD70B502684C68A24216D38B681A
:1065400023449A4206D2D1E90435AB4204D36FF01A
:106550000B038B6100200AE0CD68121B05EBC3061C
:1065600045F833204268726001330B61012070BD31
:1065700008B50020FBF714FA704701460068FBF7E6
:1065800099BA00210120FBF795BA08B5FBF7F6FA96
:10659000BDE80840FBF778BB034600201A5C02B94F
:1065A00070470130FAE70138013910F8013F11F85E
:1065B000012F934201D1002BF7D1981A704710B5E3
:1065C00062B103460139841813F8010B11F8012F49
:1065D000A34201D09042F7D0801A10BD1046FCE7CC
:1065E00010B5431E0A44914200D110BD11F8014B71
:1065F00003F8014FF7E7C9B202440346934200D1C2
:10660000704703F8011BF9E70369C9B20C2201FBCB
:106610000233186C00F0070070474FF02003EFF3CF
:10662000118283F31288BFF36F8F036803F0C003F6
:1066300043F00203036082F31188BFF36F8F70474A
:10664000034670B50069C9B24FF02004EFF311861C
:1066500084F31288BFF36F8F0C2505FB0104246CB3
:1066600014F0C00401D0A24211D105FB01000122A7
:106670000264002086F31188BFF36F8F30B95B6826
:106680000C2202FB01314B689847002070BD4FF08F
:10669000FF30EFE78022FFF7D3BFF8B5069F04690C
:1066A000C9B24FF02005EFF3118C85F31288BFF3C8
:1066B0006F8F0C2606FB0146356C05F0070EBEF108
:1066C000010F10D1376400258CF31188BFF36F8F51
:1066D0003DB90C2671430C44C4E90E2343685B5852
:1066E00098472846F8BD05F0C005AF4214BF4FF0EB
:1066F000FF356FF07705E7E713B580240094FFF7C7
:10670000CCFF02B010BD6FF085007047006910B477
:10671000CBB21C2403FB040000215DF8044B10479E
:10672000002000F007BB002000F041BB43685B681D
:10673000D3F810350B600020704743685B68D3F8CE
:10674000040542400A404240C3F804250020704737
:1067500043685B680020C3F80815704743685B68AE
:106760000020C3F80C15704743685A68D2F8043506
:106770005940C2F80415002070470369586830B5C5
:1067800058B10024814212D108689D6854B98D42E5
:10679000586000D19860002008606AB9002030BDC0
:1067A0002846EFE78D42206008BF9C60F3E705684C
:1067B0000446002DF4D13AB198685A680A605960CD
:1067C0000028EBD19960EAE76FF01500E7E738B5EC
:1067D00005460C4600F043FB002D07DBA84205D917
:1067E000401B84428CBF0020012038BD0020FCE704
:1067F0002DE9F047836886B01B698846914601A958
:1068000002AA98470024A2462546029BAB4202D822
:1068100006B0BDE8F087019F07EBC50700267B683F
:1068200004933A68B2420AEB060302D801359A464D
:10683000EBE7494603A803940593C0470028E7D037
:10684000049B01361C44ECE702690B4692E8030006
:1068500083E803000020704702690B46D2E901017A
:1068600083E803000020704743681B68D3F8800466
:10687000C3F880047047436802691B68D3F81001AD
:1068800048B1527C0A700020C3F81001D3F81021DF
:1068900001221A6070474FF0FF3070470268D2F84B
:1068A000583143B94168890707D4D2F8200100382C
:1068B00018BF012070470120704718467047426892
:1068C0001368D3F80413C90518D5D3F82011A9B15A
:1068D0004FF02000EFF3118180F31288BFF36F8F28
:1068E000D3F8200130B10020C3F82001D3F82001F3
:1068F0000120D86081F31188BFF36F8F5268D206F0
:1069000015D54FF02001EFF3118281F31288BFF308
:106910006F8FD3F8581111B10021C3F800154FF44F
:106920008001C3F8081382F31188BFF36F8F70479B
:106930002DE9F3410022064601212820FBF706F944
:106940002820FBF7E5F8776835693C68D7F80C80B4
:106950000021C4F8001501AA2E60404600F03AF864
:10696000002834DB019BD8F800201979186800F062
:1069700068F800282BDB291D3046FCF71BFA30BBDA
:106980000823C4F800353B7A5BB9C4F81001D4F889
:10699000103105F11103C4F834350123C4F838353A
:1069A00023607B689A075CBF4FF48072C4F80423AD
:1069B000DB0644BF4FF48003C4F8043310350023D2
:1069C000C4F84455C4F848350123A360E36002B01D
:1069D000BDE8F08130B543681360037A03F10053DA
:1069E000013BDB00456814681D44AC4202D96FF0DE
:1069F000010030BD65798D4202D008341460F1E7A2
:106A00000020F6E737B500F48053002B044600F071
:106A10003F0301A80EBF1546012500210193FCF795
:106A2000CDFCC4F38112019B04F4706444EA820437
:106A3000214303F5E07341EA450140F8231003B018
:106A400030BDF7B51546044600EB81070126BC4270
:106A500002D1002003B0F0BD23681A0C062A50D8DA
:106A6000DFE802F004171D4A22394A0003F03F0311
:106A7000C5F80C35236801A803F03F030193FCF728
:106A80009DFC019B06FA03F3C0F80835012211466C
:106A90001CE003F03F03C5F814350022F7E703F0CC
:106AA0003F03C5F80835E5E703F03F03C5F80835AF
:106AB000236801A803F03F030193FCF77FFC019BCF
:106AC00006FA03F3C0F80C35002201212068FFF715
:106AD00099FF0434BBE703F03F03C5F80C35236886
:106AE00001A803F03F030193FCF768FC019B06FA41
:106AF00003F3C0F80C35C9E703F03F03C5F81035C0
:106B0000CBE76FF08500A5E773B5054601A80C46F5
:106B10001646FCF761FC70BB4FF080531969B5FB5A
:106B2000F1F201FB125242BB1969B4FBF1F201FB15
:106B3000124212BB1A695B695343A3421DD3E4B1ED
:106B4000019B1B0103F1804101F5F031C1F80058B0
:106B5000C1F80448C1F80868D1F8002895420FD15F
:106B6000D1F8042894420BD1D1F80838DBB2B342F3
:106B700018BF6FF00D0002B070BD6FF01500FAE79E
:106B80006FF00D00F7E70222FFF7BEBFFDF75EBC16
:106B900008B5FAF76BFFFFF7EFFCBDE80840FDF71B
:106BA00055BC38B50C4615462544FFF7BAFC2146BE
:106BB000A94201D1012038BD11F8013B9842F7D01C
:106BC0000020F8E78068183820F007001038704778
:106BD000042809D0052803D1481E18BF012070479A
:106BE000431A5842584170470120704711B10AB109
:106BF000FFF7D7BF0020704738B50C460123114678
:106C000022460546FFF735FC002810DB012221460D
:106C10002846FFF7EBFF18B103232370002038BD8F
:106C20002378012B0CBF012302232370F7E70120F7
:106C3000F5E72DE9F7431D4606460F469046FFF758
:106C400067FC6C1E044443421C40082C1AD8304692
:106C5000FFF767FC2A46814641466846FFF7C0FCBD
:106C6000621B49460DEB0500FFF7C5FC23466A464B
:106C700039463046FFF719FC003818BF012003B031
:106C8000BDE8F0834FF0FF30F9E707B501238DF839
:106C9000042001AAFFF7CDFF03B05DF804FB816873
:106CA0001839012221F00701FFF7EFBF8268183A77
:106CB00022F00702FFF7A0BF13B50C46C0B201A92E
:106CC000FAF782FE50B921460198FCF7CDFB044645
:106CD0000198FFF7CDFB204602B010BD0124FAE772
:106CE00013B541EA021204468DF80720FFF76AFF48
:106CF000012301460DF107022046FFF79AFF02B07B
:106D000010BD4FF08053D3F83001A0F10803584272
:106D100058417047004700F0C5B808B50020FAF7A1
:106D200007FF08B9FAF7F4FE4FF080430022C3F8DA
:106D3000182508BD08B510B101282DD008BD4FF0A9
:106D40008042D2F81814D2F8183413F480330BD1DF
:106D5000D2F81414C90710D5D2F81C349B0708D4F4
:106D60000223C2F80433E9E701F00303012B04D046
:106D70001BB10020FCF79CFD00234FF08042C2F8BD
:106D800018350023C2F80431D2F804310223C2F8C6
:106D9000043301239360D1E74FF080430022C3F80E
:106DA0000021D3F80021C3F804031860C6E7FCF7FC
:106DB0007FBDF7B5019001A8DDE9084617461D46DD
:106DC000FCF70EFE019B002F00EB830014BF022393
:106DD0000023002918BF43F00103002D14BF4FF01A
:106DE0000C0C4FF0000C002C43EA0C0314BF4FF4C2
:106DF000E06C4FF0000C002E43EA0C03D0F80027A3
:106E000014BF4FF4403C4FF0000C43EA0C0322EA5D
:106E1000030301B109780FB13F787F0019430DB129
:106E20002D78AD0039430CB1227814020D430EB118
:106E3000367836042C433443C0F8004703B0F0BD25
:106E40001FB50DF10F03019300238DF80F10009370
:106E50001A461946FFF7ADFF05B05DF804FB4FF089
:106E600080531A695869504370474FF0805318692E
:106E700070474FF0805358697047704738B1C36806
:106E80001888C0F30800A0F5807358425841704735
:106E9000FFF7B1BBFFF7A4BBEFF30580003818BFC5
:106EA0000120704708B1FBF733BA704770472DE9EE
:106EB000F041069F044615461E46FDF789FC38B989
:106EC0003B46324629462046BDE8F041FDF7A6BCC8
:106ED000BDE8F0810A460021FDF728BFFFF780BB1F
:106EE000FFF789BB0A460021FFF785BB01EB820251
:106EF00004388A4201D10020704752F8043D1BBA81
:106F000040F8043FF5E70000FCF79CBB2892FF7FA8
:106F100001000000BD2200000000000099230000D5
:106F2000646F0000A5260000946F0000A5260000F5
:106F30007C6F00008D6B000000000000A92C000099
:106F4000AC6F000031690000C46F0000D531000053
:106F500000000000916B000000000000912800007C
:106F6000DC6F00001E7F0000C4720000AC720000E5
:106F700014010020540E0020D2710000457F000053
:106F80000C730000E87200001C010020AC0E002011
:106F9000CC7100003E7F00001C730000E87200000E
:106FA00018010020B80E0020C6710000BF7F00004D
:106FB00064730000687300002401002010000020AA
:106FC000C0710000C67F0000AC7300009873000021
:106FD0002801002018000020BA710000817500000F
:106FE000000000002C7300002001002000000000C1
:106FF000B471000079390000156D00000000000038
:1070000083650000000000008365000000000000B0
:1070100083650000000000008365000000000000A0
:1070200083650000F93E0000156D000000000000BF
:107030008365000000000000836500000000000080
:107040008365000000000000836500000000000070
:107050008365000000000000836500000000000060
:107060008365000000000000836500000000000050
:107070008365000000000000836500000000000040
:107080005532000000000000836500000000000091
:107090008365000000000000836500000000000020
:1070A0008365000000000000836500000000000010
:1070B0008365000000000000836500000000000000
:1070C00083650000000000008365000000000000F0
:1070D00083650000000000008365000000000000E0
:1070E00083650000000000008365000000000000D0
:1070F00083650000000000008365000000000000C0
:1071000083650000000000008365000000000000AF
:10711000836500000000000083650000000000009F
:10712000836500000000000083650000000000008F
:1071300083650000C46F0000BF680000000000000D
:10714000836500000000000083650000000000006F
:10715000836500000000000083650000000000005F
:10716000836500000000000083650000000000004F
:1071700083650000307F000003000000F37F000003
:1071800003000000B57F00000300000078760000D7
:1071900003000000B47E00000300000083810000B3
:1071A000030000001A7F000003000000CD7F0000F4
:1071B0000300000000800080FF7F00800080FF7FD0
:1071C00000800080FF7F00800080FF7F00800080C3
:1071D000FF7F00800080FF7FFFFFFFFFFFFFFFFFBB
:1071E000020000000000000085490000BD490000C9
:1071F0000338FDD87047000001000000A7790000A7
:10720000047200005B0000000000000000000000AD
:1072100000C00000817500000100000000C00000F7
:1072200000020000817500000200000000C00000A4
:1072300000A00700817500000300000000C20000EC
:10724000009E0700817500000400000000C20000DD
:10725000009E070081750000050000000060080026
:1072600000A007008175000006000000000000007B
:1072700071650000000000200000000000000B0607
:10728000201000202000000000000B15020000006C
:1072900094720000000000000B7F00002600020234
:1072A00000000020137F000022000B110767000080
:1072B00095660000F9660000000000000966000005
:1072C0000000000049240000AD240000247F0000DD
:1072D00021670000276700002A7F00005523000077
:1072E0002523000000000000212700002D6700007A
:1072F0003B670000516700005D67000069670000A0
:10730000D12500007B67000000000000FFFFFFFFA9
:10731000000000500000000000000000FFFF00001F
:10732000000300500000000001000000A928000038
:1073300071290000052A0000892800007928000032
:1073400004000000FF000000002000405C7300000B
:107350000100000016000000D1000100547300007D
:107360000200000048730000912A0000C52A0000B6
:10737000B52A0000412B000049680000008002404F
:10738000907300000100000004000000C50001002F
:10739000887300000200000077680000FD2C0000E8
:1073A00069680000B52D00005968000000800240A7
:1073B00000000000000000007C730000146F00005B
:1073C0004C6F0000546F0000646F0000646F000099
:1073D00039810000478100005B8100006A81000064
:1073E00076810000FF8FFFFFFF8FFFFFFE8FFFFF03
:1073F000FE8FFFFFFD8FFFFFFC8FFFFFFC8FFFFF66
:10740000436F756C64206E6F74206C6F636B2070BB
:107410006F7765722073617665206D75746578008D
:107420006D757465785F667265652063616C6C6507
:10743000642077697468204E554C4C2070617261ED
:107440006D6574657200000043616E277420696E7B
:10745000697469616C697A65206D757465782C2032
:10746000776173204E554C4C0D0A0000FFFFFFFF63
:10747000FFFFFFFFFFFFFFFF000000000000000014
:107480000000000001000000FFFFFFFFFCFFFFFF06
:10749000FFFFFFFFFFFFFFFF0000000000000000F4
:1074A0000000000001000000FFFFFFFF512563FC0A
:1074B000C2CAB9F3849E17A7ADFAE6BCFFFFFFFF6F
:1074C000FFFFFFFF00000000FFFFFFFF00000000C4
:1074D00096C298D84539A1F4A033EB2D817D03776E
:1074E000F240A463E5E6BCF847422CE1F2D1176B09
:1074F000F551BF376840B6CBCE5E316B5733CE2BDC
:10750000169E0F7C4AEBE78E9B7F1AFEE242E34F0A
:10751000FFFFFFFF7F000000800000000000000070
:1075200000000000FFFFFFFF7F0000008000000060
:10753000000000000000000067E6096A85AE67BB36
:1075400072F36E3C3AF54FA57F520E518C68059B45
:10755000ABD9831F19CDE05B77C295F360D2EF7F83
:107560003552500F2CB6798025633A2053746172DE
:1075700074696E6720626F6F746C6F616465720A04
:10758000004E52465F464C4153485F4452565F4E50
:10759000414D450025633A20466C6173682064655F
:1075A00076696365202573206E6F7420666F756E33
:1075B000640A0025633A20556E61626C6520746F21
:1075C0002066696E6420626F6F7461626C65206909
:1075D0006D6167650A0025633A20426F6F746C6FB6
:1075E0006164657220636861696E6C6F61642061BB
:1075F000646472657373206F66667365743A2030D5
:107600007825780A0025633A204A756D70696E679F
:1076100020746F2074686520666972737420696DC8
:1076200061676520736C6F740A0025633A2050729D
:107630006F74656374206D6375626F6F7420666C20
:10764000617368206661696C65642C2063616E6398
:10765000656C20737461727475702E0A0025633A2C
:10766000204E657665722073686F756C642067655F
:107670007420686572650A006D6375626F6F7400CF
:1076800025633A20696E76616C696420666C61736B
:10769000682049442025643B2065787065637465E3
:1076A000642025640A002A8648CE3D0201002A860D
:1076B00048CE3D030107007365636F6E64617279A4
:1076C000007072696D6172790025633A20496D61BD
:1076D000676520696E2074686520257320736C6F60
:1076E00074206973206E6F742076616C6964210A5E
:1076F0000025633A202564207374617475732077C4
:1077000072697465206661696C7320706572666F5A
:10771000726D696E672074686520737761700A0006
:1077200025633A204661696C65642072656164690D
:107730006E6720736563746F72733B20424F4F54C2
:107740005F4D41585F494D475F534543544F525336
:107750003D2564202D20746F6F20736D616C6C3F2C
:107760000A0025633A204661696C65642072656190
:1077700064696E6720696D6167652068656164652D
:1077800072733B20496D6167653D25750A0025636D
:107790003A204661696C65642072656164696E6750
:1077A00020626F6F74207374617475733B20496D30
:1077B0006167653D25750A0025633A2070616E6931
:1077C00063210A0025633A20446574656374656427
:1077D00020696E636F6E73697374656E7420737461
:1077E00061747573210A0025633A2043616E6E6FE0
:1077F0007420757067726164653A206E6F742061E1
:1078000020636F6D70617469626C6520616D6F7566
:107810006E74206F6620736563746F72730A00253F
:10782000633A2043616E6E6F742075706772616495
:10783000653A206D6F726520736563746F72732093
:107840007468616E20616C6C6F7765640A002563F3
:107850003A2043616E6E6F74207570677261646563
:107860003A206E6F742073616D6520736563746F69
:1078700072206C61796F75740A00676F6F640075B0
:107880006E73657400626164005072696D61727933
:1078900020696D6167650025633A2025733A206D84
:1078A000616769633D25732C20737761705F74791C
:1078B00070653D307825782C20636F70795F646F38
:1078C0006E653D307825782C20696D6167655F6F46
:1078D0006B3D307825780A005365636F6E64617282
:1078E0007920696D6167650025633A20426F6F7486
:1078F00020736F757263653A207072696D61727979
:1079000020736C6F740A0025633A20426F6F7420F5
:10791000736F757263653A206E6F6E650A0025633A
:107920003A205374617274696E67207377617020B6
:107930007573696E67206D6F766520616C676F7215
:107940006974686D2E0A0025633A204E6F742065B5
:107950006E6F756768206672656520737061636518
:1079600020746F2072756E20737761702075706758
:10797000726164650A0025633A20726571756972E7
:1079800065642025642062797465732062757420B3
:107990006F6E6C7920256420617265206176616963
:1079A0006C61626C650A003059301306072A8648FC
:1079B000CE3D020106082A8648CE3D030107034258
:1079C00000042ACB403CE8FEED5BA44995A1A91D2B
:1079D000AEE8DBBE1937CD14FB2F245737E59539B8
:1079E00088D994B9D65AEBD7CDD5308AD6FE48B2CD
:1079F0004A6A810EE5F07D8B6834CC3A6AFC538E7E
:107A0000FAC12D002B00305800307800286E696CC8
:107A100029004661696C656420746F207265626F2D
:107A20006F743A207370696E6E696E6720656E645C
:107A30006C6573736C792E2E2E0A0025633A2072C2
:107A4000302F61313A20203078253038782020726C
:107A5000312F61323A20203078253038782020725A
:107A6000322F61333A20203078253038780A0025CB
:107A7000633A2072332F61343A2020307825303831
:107A800078207231322F69703A20203078253038D2
:107A900078207231342F6C723A20203078253038BB
:107AA000780A0025633A2020787073723A202030DB
:107AB00078253038780A0025633A204661756C7461
:107AC000696E6720696E737472756374696F6E2076
:107AD0006164647265737320287231352F70632975
:107AE0003A203078253038780A0025633A202A2A4F
:107AF0002A2A2A204D5055204641554C54202A2AE6
:107B00002A2A2A0A0025633A202020537461636BD5
:107B1000696E67206572726F722028636F6E74657C
:107B200078742061726561206D6967687420626590
:107B3000206E6F742076616C6964290A0025633AAF
:107B4000202020556E737461636B696E67206572C7
:107B5000726F720A0025633A20202044617461200C
:107B60004163636573732056696F6C6174696F6EEE
:107B70000A0025633A2020204D4D464152204164A1
:107B800064726573733A20307825780A0025633A69
:107B9000202020496E737472756374696F6E204182
:107BA00063636573732056696F6C6174696F6E0AE5
:107BB0000025633A202020466C6F6174696E672D42
:107BC000706F696E74206C617A792073746174656A
:107BD00020707265736572766174696F6E2065726C
:107BE000726F720A0025633A202A2A2A2A2A20550F
:107BF00053414745204641554C54202A2A2A2A2AD7
:107C00000A0025633A2020204469766973696F6E03
:107C1000206279207A65726F0A0025633A2020205D
:107C2000556E616C69676E6564206D656D6F727904
:107C3000206163636573730A0025633A2020204E38
:107C40006F20636F70726F636573736F7220696EFC
:107C5000737472756374696F6E730A0025633A20DA
:107C60002020496C6C6567616C206C6F6164206FCB
:107C700066204558435F52455455524E20696E74F4
:107C80006F2050430A0025633A202020496C6C6520
:107C900067616C20757365206F6620746865204588
:107CA0005053520A0025633A202020417474656DB8
:107CB000707420746F206578656375746520756EC7
:107CC000646566696E656420696E73747275637449
:107CD000696F6E0A0025633A202A2A2A2A2A20423E
:107CE0005553204641554C54202A2A2A2A2A0A0054
:107CF00025633A202020537461636B696E672065A9
:107D000072726F720A0025633A20202050726563F8
:107D10006973652064617461206275732065727295
:107D20006F720A0025633A202020424641522041CA
:107D30006464726573733A20307825780A0025638D
:107D40003A202020496D7072656369736520646113
:107D5000746120627573206572726F720A00256308
:107D60003A202020496E737472756374696F6E20B7
:107D7000627573206572726F720A00526573657264
:107D800076656420457863657074696F6E2028009D
:107D900053707572696F757320696E746572727550
:107DA00070742028495251200025633A20535053C3
:107DB000454C20696E20746872656164206D6F6443
:107DC0006520646F6573206E6F7420696E646963EB
:107DD000617465205053500A0025633A202A2A2AEC
:107DE0002A2A2048415244204641554C54202A2AF0
:107DF0002A2A2A0A0025633A202020427573206629
:107E000061756C74206F6E20766563746F72207478
:107E100061626C6520726561640A0025633A202006
:107E2000204465627567206576656E740A00256377
:107E30003A2020204661756C7420657363616C6123
:107E400074696F6E20287365652062656C6F772991
:107E50000A0025633A20415243485F455843455044
:107E600054207769746820726561736F6E2025787D
:107E70000A0A0025633A202A2A2A2A2A204465620F
:107E80007567206D6F6E69746F72206578636570B9
:107E900074696F6E202A2A2A2A2A0A0025633A204A
:107EA0002A2A2A2A2A20257320256429202A2A2AD8
:107EB0002A2A0A006D70750025633A205061727499
:107EC0006974696F6E2025753A2073616E697479E3
:107ED00020636865636B206661696C65642E0A00C7
:107EE00025633A204661696C656420746F20616C7B
:107EF0006C6F63617465206E6577204D50552072FC
:107F00006567696F6E2025750A0A00464C41534823
:107F10005F30005352414D5F3000736F6300434C3C
:107F20004F434B006866636C6B006C66636C6B0060
:107F3000636C6F636B5F636F6E74726F6C0047503E
:107F4000494F5F31004750494F5F300025633A2069
:107F5000696E76616C696420616464726573733AFA
:107F60002030782530386C783A257A750A002563F8
:107F70003A206E6F7420776F72642D616C69676E42
:107F800065643A2030782530386C783A257A750A5D
:107F90000025633A20756E616C69676E65642061C7
:107FA0006464726573733A2030782530386C783A9F
:107FB000257A750A00666C6173685F6E726600559B
:107FC0004152545F3000554152545F310075617227
:107FD000745F6E7266785F75617274650025633ACE
:107FE00020526573657474696E6720737973746564
:107FF0006D0A00666174616C5F6572726F72007207
:1080000065766572740074657374007065726D00D6
:108010004255473B2063616E27742068617070652C
:108020006E0025633A205365636F6E646172792038
:10803000696D616765206F6620696D616765207095
:10804000616972202825642E2920697320756E725B
:108050006561636861626C652E205472656174208D
:10806000697420617320656D7074790A0025633A24
:10807000205377617020747970653A2025730A0067
:1080800025633A205377617020747970653A206EC9
:108090006F6E650A00040104030402040104010474
:1080A00003010303040104000000000001010000BB
:1080B000000000556E6B6E6F776E206572726F7286
:1080C0000025633A203E3E3E205A455048595220F2
:1080D000464154414C204552524F522025643A208B
:1080E0002573206F6E204350552025640A002563B8
:1080F0003A204661756C7420647572696E672069F8
:108100006E746572727570742068616E646C696EED
:10811000670A0A00756E6B6E6F776E0025633A20F2
:1081200043757272656E74207468726561643A207A
:10813000257020282573290A00435055206578634F
:10814000657074696F6E00556E68616E646C65640D
:1081500020696E7465727275707400537461636B1C
:10816000206F766572666C6F77004B65726E656C1A
:10817000206F6F7073004B65726E656C2070616E5E
:108180006963006F73000000FFFFFFFFFFFFFFFF49
:10819000DF6200000872000000E10000000103003F
:1081A0000000000000E100000001030000000000EA
:1081B000000000000090D00300000000000000005C
:1081C00000000000000000000000000000000000AF
:1081D000000000000000000000000000000000009F
:1081E000000000000000000000000000000000008F
:1081F000000000000000000000000000000000007F
:10820000000000000000000000000000000000006E
:10821000000000000000000000000000000000005E
:108220000000000000000000FF000000000000004F
:1082300000000000AC000020AC00002000000000A6
:1082400085440000EC000020F8000020F000002031
:10825000E8000020C4000020F40E002011000000FF
:1082600095470000014700002947000069470000CA
:108270000C010020D00000200401002000000000BC
:10828000FC000020F80E002011000000FC0E002071
:1082900011000000000F002011000000000000008D
:1082A00000000000000000000000000000000000CE
:0482B00000000000CA
:10C000003DB8F3960000000000020000EC7802004A
:10C010000000000000000000000000000000000020
:10C02000FFFFFFFFFFFFFFFFFFFFFFFFFFFFFFFF20
:10C03000FFFFFFFFFFFFFFFFFFFFFFFFFFFFFFFF10
:10C04000FFFFFFFFFFFFFFFFFFFFFFFFFFFFFFFF00
:10C05000FFFFFFFFFFFFFFFFFFFFFFFFFFFFFFFFF0
:10C06000FFFFFFFFFFFFFFFFFFFFFFFFFFFFFFFFE0
:10C07000FFFFFFFFFFFFFFFFFFFFFFFFFFFFFFFFD0
:10C08000FFFFFFFFFFFFFFFFFFFFFFFFFFFFFFFFC0
:10C09000FFFFFFFFFFFFFFFFFFFFFFFFFFFFFFFFB0
:10C0A000FFFFFFFFFFFFFFFFFFFFFFFFFFFFFFFFA0
:10C0B000FFFFFFFFFFFFFFFFFFFFFFFFFFFFFFFF90
:10C0C000FFFFFFFFFFFFFFFFFFFFFFFFFFFFFFFF80
:10C0D000FFFFFFFFFFFFFFFFFFFFFFFFFFFFFFFF70
:10C0E000FFFFFFFFFFFFFFFFFFFFFFFFFFFFFFFF60
:10C0F000FFFFFFFFFFFFFFFFFFFFFFFFFFFFFFFF50
:10C10000FFFFFFFFFFFFFFFFFFFFFFFFFFFFFFFF3F
:10C11000FFFFFFFFFFFFFFFFFFFFFFFFFFFFFFFF2F
:10C12000FFFFFFFFFFFFFFFFFFFFFFFFFFFFFFFF1F
:10C13000FFFFFFFFFFFFFFFFFFFFFFFFFFFFFFFF0F
:10C14000FFFFFFFFFFFFFFFFFFFFFFFFFFFFFFFFFF
:10C15000FFFFFFFFFFFFFFFFFFFFFFFFFFFFFFFFEF
:10C16000FFFFFFFFFFFFFFFFFFFFFFFFFFFFFFFFDF
:10C17000FFFFFFFFFFFFFFFFFFFFFFFFFFFFFFFFCF
:10C18000FFFFFFFFFFFFFFFFFFFFFFFFFFFFFFFFBF
:10C19000FFFFFFFFFFFFFFFFFFFFFFFFFFFFFFFFAF
:10C1A000FFFFFFFFFFFFFFFFFFFFFFFFFFFFFFFF9F
:10C1B000FFFFFFFFFFFFFFFFFFFFFFFFFFFFFFFF8F
:10C1C000FFFFFFFFFFFFFFFFFFFFFFFFFFFFFFFF7F
:10C1D000FFFFFFFFFFFFFFFFFFFFFFFFFFFFFFFF6F
:10C1E000FFFFFFFFFFFFFFFFFFFFFFFFFFFFFFFF5F
:10C1F000FFFFFFFFFFFFFFFFFFFFFFFFFFFFFFFF4F
:10C20000C07B00203D48010055950200F547010024
:10C21000F5470100F5470100F54701000000000067
:10C22000000000000000000000000000E1380100F4
:10C23000F54701000000000089380100F5470100C2
:10C24000C1390100A3CC0200C1390100C13901008C
:10C25000C1390100C1390100C1390100C1390100F2
:10C26000C1390100C1390100C1390100C1390100E2
:10C27000C1390100C1390100C1390100C1390100D2
:10C28000C1390100C1390100C1390100C1390100C2
:10C29000C1390100C1390100C1390100C1390100B2
:10C2A000C1390100C1390100C1390100C1390100A2
:10C2B000C1390100C1390100C1390100C139010092
:10C2C000C1390100C1390100C1390100C139010082
:10C2D000C1390100C1390100C1390100C139010072
:10C2E000C1390100C1390100C1390100C139010062
:10C2F000C1390100C1390100C1390100C139010052
:10C3000081F0004102E000BF83F0004330B54FEA06
:10C3100041044FEA430594EA050F08BF90EA020F73
:10C320001FBF54EA000C55EA020C7FEA645C7FEA06
:10C33000655C00F0E2804FEA5454D4EB5555B8BF29
:10C340006D420CDD2C4480EA020281EA030382EA9A
:10C35000000083EA010180EA020281EA0303362D2C
:10C3600088BF30BD11F0004F4FEA01314FF4801CFF
:10C370004CEA113102D0404261EB410113F0004F11
:10C380004FEA03334CEA133302D0524263EB4303C8
:10C3900094EA050F00F0A780A4F10104D5F1200E66
:10C3A0000DDB02FA0EFC22FA05F2801841F10001C1
:10C3B00003FA0EF2801843FA05F359410EE0A5F195
:10C3C00020050EF1200E012A03FA0EFC28BF4CF0C6
:10C3D000020C43FA05F3C01851EBE37101F000457C
:10C3E00007D54FF0000EDCF1000C7EEB00006EEB89
:10C3F0000101B1F5801F1BD3B1F5001F0CD3490813
:10C400005FEA30004FEA3C0C04F101044FEA445269
:10C4100012F5800F80F09A80BCF1004F08BF5FEAF0
:10C42000500C50F1000041EB045141EA050130BDD0
:10C430005FEA4C0C404141EB0101013C28BFB1F5E2
:10C44000801FE9D291F0000F04BF01460020B1FA2D
:10C4500081F308BF2033A3F10B03B3F120020CDA00
:10C460000C3208DD02F1140CC2F10C0201FA0CF0DE
:10C4700021FA02F10CE002F11402D8BFC2F1200C43
:10C4800001FA02F120FA0CFCDCBF41EA0C019040F9
:10C49000E41AA2BF01EB0451294330BD6FEA040442
:10C4A0001F3C1CDA0C340EDC04F11404C4F120022D
:10C4B00020FA04F001FA02F340EA030021FA04F33F
:10C4C00045EA030130BDC4F10C04C4F1200220FA96
:10C4D00002F001FA04F340EA0300294630BD21FAD4
:10C4E00004F0294630BD94F0000F83F4801306BF9A
:10C4F00081F480110134013D4EE77FEA645C18BF8E
:10C500007FEA655C29D094EA050F08BF90EA020F24
:10C5100005D054EA000C04BF1946104630BD91EA1C
:10C52000030F1EBF0021002030BD5FEA545C05D11F
:10C530004000494128BF41F0004130BD14F580045E
:10C540003CBF01F5801130BD01F0004545F0FE41D2
:10C5500041F470014FF0000030BD7FEA645C1ABF07
:10C56000194610467FEA655C1CBF0B46024650EA3E
:10C57000013406BF52EA033591EA030F41F400216A
:10C5800030BD00BF90F0000F04BF0021704730B5F0
:10C590004FF4806404F132044FF000054FF00001C5
:10C5A00050E700BF90F0000F04BF0021704730B586
:10C5B0004FF4806404F1320410F0004548BF40425B
:10C5C0004FF000013EE700BF42004FEAE2014FEAB0
:10C5D00031014FEA02701FBF12F07F4393F07F4F8B
:10C5E00081F06051704732F07F4208BF704793F08E
:10C5F0007F4F04BF41F40021704730B54FF46074A1
:10C6000001F0004521F000411CE700BF50EA0102A3
:10C6100008BF704730B54FF000050AE050EA01024C
:10C6200008BF704730B511F0004502D5404261EBBC
:10C6300041014FF4806404F132045FEA915C3FF4FD
:10C64000D8AE4FF003025FEADC0C18BF03325FEA9A
:10C65000DC0C18BF033202EBDC02C2F1200300FA4B
:10C6600003FC20FA02F001FA03FE40EA0E0021FA70
:10C6700002F11444BDE600BF70B54FF0FF0C4CF45E
:10C68000E06C1CEA11541DBF1CEA135594EA0C0F10
:10C6900095EA0C0F00F0DEF82C4481EA030621EA4B
:10C6A0004C5123EA4C5350EA013518BF52EA033586
:10C6B00041F4801143F4801338D0A0FB02CE4FF038
:10C6C0000005E1FB02E506F00042E0FB03E54FF068
:10C6D0000006E1FB03569CF0000F18BF4EF0010E60
:10C6E000A4F1FF04B6F5007F64F5407404D25FEA5C
:10C6F0004E0E6D4146EB060642EAC62141EA55510F
:10C700004FEAC52040EA5E504FEACE2EB4F1FD0C50
:10C7100088BFBCF5E06F1ED8BEF1004F08BF5FEACE
:10C72000500E50F1000041EB045170BD06F0004680
:10C7300046EA010140EA020081EA0301B4EB5C042D
:10C74000C2BFD4EB0C0541EA045170BD41F4801125
:10C750004FF0000E013C00F3AB8014F1360FDEBF4A
:10C76000002001F0004170BDC4F10004203C35DA26
:10C770000C341BDC04F11404C4F1200500FA05F3A9
:10C7800020FA04F001FA05F240EA020001F000424A
:10C7900021F0004110EBD37021FA04F642EB0601C0
:10C7A0005EEA430E08BF20EAD37070BDC4F10C04EA
:10C7B000C4F1200500FA04F320FA05F001FA04F2AE
:10C7C00040EA020001F0004110EBD37041F100019A
:10C7D0005EEA430E08BF20EAD37070BDC4F12005A5
:10C7E00000FA05F24EEA020E20FA04F301FA05F20D
:10C7F00043EA020321FA04F001F0004121FA04F2B5
:10C8000020EA020000EBD3705EEA430E08BF20EA84
:10C81000D37070BD94F0000F0FD101F000464000BE
:10C8200041EB010111F4801F08BF013CF7D041EA40
:10C83000060195F0000F18BF704703F00046520044
:10C8400043EB030313F4801F08BF013DF7D043EA15
:10C850000603704794EA0C0F0CEA135518BF95EACB
:10C860000C0F0CD050EA410618BF52EA4306D1D152
:10C8700081EA030101F000414FF0000070BD50EA71
:10C88000410606BF1046194652EA430619D094EAFB
:10C890000C0F02D150EA013613D195EA0C0F05D1E5
:10C8A00052EA03361CBF104619460AD181EA030139
:10C8B00001F0004141F0FE4141F470014FF00000F1
:10C8C00070BD41F0FE4141F4780170BD70B54FF08C
:10C8D000FF0C4CF4E06C1CEA11541DBF1CEA13550C
:10C8E00094EA0C0F95EA0C0F00F0A7F8A4EB0504EE
:10C8F00081EA030E52EA03354FEA013100F08880E5
:10C900004FEA03334FF0805545EA131343EA1263AD
:10C910004FEA022245EA111545EA10654FEA002662
:10C920000EF000419D4208BF964244F1FD0404F51B
:10C93000407402D25B084FEA3202B61A65EB030577
:10C940005B084FEA32024FF480104FF4002CB6EB34
:10C95000020E75EB030E22BFB61A754640EA0C00B4
:10C960005B084FEA3202B6EB020E75EB030E22BFF4
:10C97000B61A754640EA5C005B084FEA3202B6EB35
:10C98000020E75EB030E22BFB61A754640EA9C00F4
:10C990005B084FEA3202B6EB020E75EB030E22BFC4
:10C9A000B61A754640EADC0055EA060E18D04FEA82
:10C9B000051545EA16754FEA06164FEAC30343EA22
:10C9C00052734FEAC2025FEA1C1CC0D111F4801FEF
:10C9D0000BD141EA00014FF000004FF0004CB6E7E8
:10C9E00011F4801F04BF01430020B4F1FD0C88BF87
:10C9F000BCF5E06F3FF6AFAEB5EB030C04BFB6EB92
:10CA0000020C5FEA500C50F1000041EB045170BD84
:10CA10000EF0004E4EEA113114EB5C04C2BFD4EBB1
:10CA20000C0541EA045170BD41F480114FF0000E35
:10CA3000013C90E645EA060E8DE60CEA135594EAB1
:10CA40000C0F08BF95EA0C0F3FF43BAF94EA0C0FB4
:10CA50000AD150EA01347FF434AF95EA0C0F7FF429
:10CA600025AF104619462CE795EA0C0F06D152EA7D
:10CA700003353FF4FDAE1046194622E750EA410661
:10CA800018BF52EA43067FF4C5AE50EA41047FF472
:10CA90000DAF52EA43057FF4EBAE12E74FF0FF3CD7
:10CAA00006E000BF4FF0010C02E000BF4FF0010CA8
:10CAB0004DF804CD4FEA410C7FEA6C5C4FEA430C21
:10CAC00018BF7FEA6C5C1BD001B050EA410C0CBF70
:10CAD00052EA430C91EA030F02BF90EA020F0020D2
:10CAE000704710F1000F91EA030F58BF994208BF39
:10CAF00090422CBFD8176FEAE37040F001007047F6
:10CB00004FEA410C7FEA6C5C02D150EA013C07D14C
:10CB10004FEA430C7FEA6C5CD6D152EA033CD3D097
:10CB20005DF8040B704700BF8446104662468C4691
:10CB30001946634600E000BF01B5FFF7B7FF0028C4
:10CB400048BF10F1000F01BD4DF808EDFFF7F4FFED
:10CB50000CBF012000205DF808FB00BF4DF808ED78
:10CB6000FFF7EAFF34BF012000205DF808FB00BF9B
:10CB70004DF808EDFFF7E0FF94BF012000205DF8BD
:10CB800008FB00BF4DF808EDFFF7CEFF94BF012072
:10CB900000205DF808FB00BF4DF808EDFFF7C4FF6B
:10CBA00034BF012000205DF808FB00BF80F000408A
:10CBB00002E000BF81F0004142001FBF5FEA410375
:10CBC00092EA030F7FEA226C7FEA236C6AD04FEA75
:10CBD0001262D2EB1363C1BFD218414048404140BA
:10CBE000B8BF5B42192B88BF704710F0004F40F46C
:10CBF000000020F07F4018BF404211F0004F41F488
:10CC0000000121F07F4118BF494292EA030F3FD053
:10CC1000A2F1010241FA03FC10EB0C00C3F1200366
:10CC200001FA03F100F0004302D5494260EB4000F5
:10CC3000B0F5000F13D3B0F1807F06D340084FEA60
:10CC4000310102F10102FE2A51D2B1F1004F40EB55
:10CC5000C25008BF20F0010040EA030070474900BD
:10CC600040EB0000013A28BFB0F5000FEDD2B0FA5A
:10CC700080FCACF1080CB2EB0C0200FA0CF0AABF7D
:10CC800000EBC25052421843BCBFD040184370471B
:10CC900092F0000F81F4000106BF80F40000013221
:10CCA000013BB5E74FEA41037FEA226C18BF7FEAF8
:10CCB000236C21D092EA030F04D092F0000F08BF3A
:10CCC0000846704790EA010F1CBF0020704712F021
:10CCD0007F4F04D1400028BF40F00040704712F160
:10CCE00000723CBF00F50000704700F0004343F0C5
:10CCF000FE4040F4000070477FEA226216BF0846FB
:10CD00007FEA23630146420206BF5FEA412390EABD
:10CD1000010F40F4800070474FF0000304E000BFB3
:10CD200010F0004348BF40425FEA000C08BF704764
:10CD300043F0964301464FF000001CE050EA010228
:10CD400008BF70474FF000030AE000BF50EA01023D
:10CD500008BF704711F0004302D5404261EB41012A
:10CD60005FEA010C02BF84460146002043F0B6434F
:10CD700008BFA3F18053A3F50003BCFA8CF2083A74
:10CD8000A3EBC25310DB01FA02FC634400FA02FC7D
:10CD9000C2F12002BCF1004F20FA02F243EB020084
:10CDA00008BF20F00100704702F1200201FA02FCE6
:10CDB000C2F1200250EA4C0021FA02F243EB0200D9
:10CDC00008BF20EADC7070474FF0FF0C1CEAD0521D
:10CDD0001EBF1CEAD15392EA0C0F93EA0C0F6FD0DE
:10CDE0001A4480EA010C400218BF5FEA41211ED0BC
:10CDF0004FF0006343EA501043EA5111A0FB0131A8
:10CE00000CF00040B1F5000F3EBF490041EAD3717C
:10CE10005B0040EA010062F17F02FD2A1DD8B3F1F8
:10CE2000004F40EBC25008BF20F00100704790F067
:10CE3000000F0CF0004C08BF49024CEA502040EAB9
:10CE400051207F3AC2BFD2F1FF0340EAC25070477F
:10CE500040F400004FF00003013A5DDC12F1190FBD
:10CE6000DCBF00F000407047C2F10002410021FA2F
:10CE700002F1C2F1200200FA02FC5FEA310040F147
:10CE8000000053EA4C0308BF20EADC70704792F0C0
:10CE9000000F00F0004C02BF400010F4000F013AF8
:10CEA000F9D040EA0C0093F0000F01F0004C02BFF3
:10CEB000490011F4000F013BF9D041EA0C018FE762
:10CEC0000CEAD15392EA0C0F18BF93EA0C0F0AD068
:10CED00030F0004C18BF31F0004CD8D180EA01008E
:10CEE00000F00040704790F0000F17BF90F0004F27
:10CEF000084691F0000F91F0004F14D092EA0C0F09
:10CF000001D142020FD193EA0C0F03D14B0218BF9B
:10CF1000084608D180EA010000F0004040F0FE40E1
:10CF200040F40000704740F0FE4040F4400070477D
:10CF30004FF0FF0C1CEAD0521EBF1CEAD15392EAFC
:10CF40000C0F93EA0C0F69D0A2EB030280EA010CEC
:10CF500049024FEA402037D04FF0805343EA111185
:10CF600043EA10130CF000408B4238BF5B0042F1E3
:10CF70007D024FF4000C8B4224BF5B1A40EA0C0088
:10CF8000B3EB510F24BFA3EB510340EA5C00B3EBBA
:10CF9000910F24BFA3EB910340EA9C00B3EBD10FA8
:10CFA00024BFA3EBD10340EADC001B0118BF5FEAFA
:10CFB0001C1CE0D1FD2A3FF650AF8B4240EBC25023
:10CFC00008BF20F0010070470CF0004C4CEA5020E4
:10CFD0007F32C2BFD2F1FF0340EAC250704740F433
:10CFE00000004FF00003013A37E792F0000F00F025
:10CFF000004C02BF400010F4000F013AF9D040EAA3
:10D000000C0093F0000F01F0004C02BF490011F436
:10D01000000F013BF9D041EA0C0195E70CEAD1532E
:10D0200092EA0C0F08D142027FF47DAF93EA0C0F15
:10D030007FF470AF084676E793EA0C0F04D14B02F9
:10D040003FF44CAF08466EE730F0004C18BF31F0AB
:10D05000004CCAD130F000427FF45CAF31F00043A5
:10D060007FF43CAF5FE700BF4FF0FF3C06E000BF3E
:10D070004FF0010C02E000BF4FF0010C4DF804CD61
:10D080004FEA40024FEA41037FEA226C18BF7FEA71
:10D09000236C11D001B052EA530C18BF90EA010F73
:10D0A00058BFB2EB030088BFC81738BF6FEAE17002
:10D0B00018BF40F0010070477FEA226C02D15FEA9E
:10D0C000402C05D17FEA236CE4D15FEA412CE1D00A
:10D0D0005DF8040B704700BF844608466146FFE7D1
:10D0E0000FB5FFF7C9FF002848BF10F1000F0FBDB3
:10D0F0004DF808EDFFF7F4FF0CBF012000205DF8AC
:10D1000008FB00BF4DF808EDFFF7EAFF34BF012030
:10D1100000205DF808FB00BF4DF808EDFFF7E0FFC9
:10D1200094BF012000205DF808FB00BF4DF808ED1A
:10D13000FFF7D2FF94BF012000205DF808FB00BF7D
:10D140004DF808EDFFF7C8FF34BF012000205DF85F
:10D1500008FB00BF4FEA4002B2F1FE4F0FD34FF081
:10D160009E03B3EB12620DD94FEA002343F0004354
:10D1700010F0004F23FA02F018BF404270474FF002
:10D180000000704712F1610F01D1420205D110F089
:10D19000004008BF6FF0004070474FF0000070473C
:10D1A00042000ED2B2F1FE4F0BD34FF09E03B3EB11
:10D1B000126209D44FEA002343F0004323FA02F03D
:10D1C00070474FF00000704712F1610F01D1420229
:10D1D00002D14FF0FF3070474FF00000704700BFA2
:10D1E00053B94AB9002908BF00281CBF4FF0FF31CE
:10D1F0004FF0FF3000F02AB8ADF1080C6DE904CE15
:10D2000000F05FF8DDF804E0DDE9022304B07047C8
:10D21000D0B50C4B002206460F46FFF72DFA00F062
:10D2200017F80446FFF7AEF9074B0022FFF724FA80
:10D2300002460B4630463946FFF766F800F008F81C
:10D240002146D0BD0000F03D0000F041704700BF16
:10D250004A0011D212F5001211D20DD56FF4787375
:10D26000B3EB62520ED44FEAC12343F0004343EACA
:10D27000505323FA02F070474FF00000704750EA15
:10D28000013002D14FF0FF3070474FF0000070477F
:10D2900038B505460C460022002328462146FFF7F4
:10D2A0005DFC28B928462146BDE83840FFF7B0BFED
:10D2B000284604F10041FFF7ABFF404261EB41011A
:10D2C00038BD2DE9F04F07468C460846099E1546A5
:10D2D0003C461946002B40F0C6808242B2FA82F7E3
:10D2E00046D94FB1C7F1200E24FA0EFE00FA07F31B
:10D2F000BD404EEA030CBC404FEA15481FFA85FEBC
:10D30000BCFBF8F9220C08FB19C309FB0EFA42EA30
:10D3100003439A4528D9EB1809F1FF3004D29A4506
:10D3200002D9A9F102002B44A3EB0A03A4B2B3FB78
:10D33000F8F208FB123302FB0EFE44EA0344A64552
:10D3400014D92C1902F1FF3303D2A64501D9931E3B
:10D350002C44A4EB0E0443EA00401EB1FC40002321
:10D3600034607360BDE8F08F4846DDE71346F0E7B0
:10D3700002B9FFDE87BB831A01214FEA154EAAB21C
:10D38000B3FBFEFC200C0EFB1C330CFB02F840EA46
:10D390000343984563D9EB180CF1FF3004D298454C
:10D3A00002D9ACF102002B44A3EB0803A4B2B3FBF7
:10D3B000FEFC0EFB1C330CFB02F244EA0344A242C7
:10D3C0004FD92C190CF1FF3304D2A24202D9ACF18F
:10D3D00002032C44A41ABEE7C7F1200C20FA0CF873
:10D3E00000FA07F324FA0CFCBD404CEA03024FEAB2
:10D3F000154EABB2B8FBFEFC110C0EFB1C800CFBF7
:10D4000003F941EA0040814504FA07F423D92818BA
:10D410000CF1FF3104D2814502D9ACF1020128445C
:10D42000A0EB090092B2B0FBFEFC0EFB1C000CFB53
:10D4300003F842EA004398450FD9EB180CF1FF328C
:10D4400004D2984502D9ACF102022B44A3EB0803A5
:10D4500042EA014191E76146E2E76246F6E760464B
:10D46000A2E76346B6E7834205D90EB1C6E900706C
:10D470000021084676E7B3FA83F181B9834201D3EC
:10D48000BA420AD8BC1A60EB030301209C46002E66
:10D4900068D0C6E9004C002164E70846F7E7C1F10F
:10D4A000200C8B4022FA0CF41C4302FA01F500FA1E
:10D4B00001F327FA0CF220FA0CFB4FEA144913434C
:10D4C000BBFBF9F81FFA84FE09FB18BB1A0C08FB1A
:10D4D0000EFA42EA0B42924507FA01F73ED9A2182A
:10D4E00008F1FF3004D2924502D9A8F1020022448B
:10D4F000A2EB0A029BB2B2FBF9F809FB182208FB67
:10D500000EFE43EA024296452AD9A21808F1FF33DB
:10D5100004D2964502D9A8F10203224443EA00400E
:10D52000A0FB0593A2EB0E029A42CE46984602D388
:10D5300006D14F4504D2B9EB050E63EB0408013860
:10D5400086B1B7EB0E0362EB080707FA0CFCCB4081
:10D550004CEA0303CF40C6E900379CE74046C7E7E3
:10D560004346DBE73146FDE608B507A3D3E90023D0
:10D57000FFF782F8FFF78CFE054B064A1AF01DFAFA
:10D5800008BD00BFAFF3008000000000D01263416F
:10D5900000D2496B002EB69400295CD030B591B012
:10D5A00005460C4691F834308DF80030088BFFF7B3
:10D5B000B3FB2D49FFF7BCFC0190608BFFF7ACFB80
:10D5C0002949FFF7B5FC0290B4F91C00FFF7A8FB4E
:10D5D0002549FFF7ADFC03902068FEF7E3FF20A389
:10D5E000D3E90023FFF772F9CDE904016068FEF783
:10D5F000D9FF1BA3D3E90023FFF768F9CDE90601A2
:10D60000A3680893E368099394F835308DF82830BF
:10D6100023690B9394F836308DF8303094F8373016
:10D620008DF8313094F838308DF8323094F8393044
:10D630008DF8333094F83A308DF8343063690E93B6
:10D64000694605F15B0002F057FF30B9012385F808
:10D65000353311B030BD012070470120F9E700BF1C
:10D6600000000000D01263410000C842000000002A
:10D67000002940D030B58DB005460C4691F83230C7
:10D680008DF8003091F833308DF801300868FEF7DE
:10D6900089FF1BA3D3E90023FFF718F9CDE90201A5
:10D6A0006068FEF77FFF16A3D3E90023FFF70EF9AA
:10D6B000CDE90401238BADF81830638BADF81A3037
:10D6C000A3680793E368089394F834308DF8243006
:10D6D00094F835308DF8253023690A9363690B93EC
:10D6E000694605F21D2003F0DFF830B9012385F803
:10D6F00047330DB030BD012070470120F9E700BF6E
:10D7000000000000D012634110B504460023A0F8C9
:10D710007430A0F876200A48A1FB000C06A3D3E9D8
:10D72000002340F6181E0EFB01C1FFF759FD20F043
:10D730007F40A06710BD00BF8D49FD1A07000000A3
:10D7400000A0724E000000002DE9F04782B00F46A5
:10D750001D460B9C4FF6FF739D4222D0814690469A
:10D7600004F11C0A23780133DBB22370002B42D072
:10D77000334EC6F80090C6F8048035819DF82830F5
:10D78000B372C6F80CA02F4B9E60002211460120F8
:10D7900009F0D6FC00283CD1236C13B120460CF0D4
:10D7A000EDFF294B009300231A4640F24711204613
:10D7B0000BF0AEFCB4F874302B440133A4F8743091
:10D7C000A66FAEB1A16E2148A1FB000C1AA3D3E94C
:10D7D00000234FF0910E0EFB01C1FFF701FD20F079
:10D7E0007F4005FB00053D44AE4220D9751BA5676F
:10D7F00002B0BDE8F08740F6A203154A1549164865
:10D800001BF003FA404080F311884FF0030002DF61
:10D81000AEE740F6AF030E4A10490F481BF0F5F98A
:10D82000404080F311884FF0030002DFB4E7A067A7
:10D83000DEE700BFAFF300808D49FD1A070000004E
:10D84000743B002060040020D9900100002AE78486
:10D8500004210300B82103006819030034200300E9
:10D8600070B582B0C469B4F8763053B1B4F874209E
:10D87000934206D80023A4F87630E66B4323337234
:10D8800018E0A56F002D37D0A66E3148A6FB000129
:10D890002DA3D3E900234FF0910C0CFB0611FFF7E9
:10D8A0009FFC20F07F40854226D80023A367E66BCB
:10D8B0003C233372274D651B274AA2FB0535C5F370
:10D8C0004715022D1AD812233371F5804FF6FF73D6
:10D8D0007381B4F874307372236CEBB118680CF078
:10D8E000A1FA421D00941D4BD2B20121002009F083
:10D8F0004BFF08B1022818D102B070BD40F2AC73E2
:10D90000174A184918481BF080F9404080F31188E5
:10D910004FF0030002DFD6E7AA1C0094134BD2B2EB
:10D920000121002009F030FFE3E740F2C5730C4A03
:10D930000F490D481BF069F9404080F311884FF002
:10D94000030002DFD8E700BF8D49FD1A0700000081
:10D95000002AE784C4390020E1830F3E759001005E
:10D9600004210300642203006819030031900100C0
:10D97000BC210300000000002DE9F04F97B00546E0
:10D980000B9300294FD01646022850D8DFF8448167
:10D9900000EB40144FEA840908EB840494F87C30CF
:10D9A00013F0010F43D1002C41D0FF2384F8223023
:10D9B00094F8200080090DF065FC94F87C3003F0A9
:10D9C0000603042B6ED0062B6CD094F8253002335E
:10D9D00004EB8303D3F820A094F83130043304EB34
:10D9E00083035F6A3A46514620461EF000FA83469A
:10D9F00000284DD11DF032FD00286DD00AF0F4FC56
:10DA00000C90002800F08E810AF0C0FD00285AD04A
:10DA1000002202710C9A0260E0630B9A31462046A4
:10DA2000FFF772FE5EE00BF011FC834630E01DF064
:10DA300015FD58B3022D00F26681264B05EB451407
:10DA400003EB840494F87C3013F0010F00F05E8146
:10DA5000002C00F05E8194F82530023304EB830340
:10DA600094F83120043204EB8202526A196A20468B
:10DA70001EF0BDF9834658B9E56B002D00F04C81CE
:10DA80002B794BB12B79002B40F049814FF0000BE3
:10DA9000584617B0BDE8F08F0B9A31462046FFF785
:10DAA00033FEEFE794F87C00002204F17D01C0F31F
:10DAB000C0000DF059FD84F82200FF2885D0002019
:10DAC0000DF0FAFB81E70C980AF096FC4FF0070B7B
:10DAD000DEE700BFC43900200021E1630A4620468A
:10DAE000FFF712FE94F8216006F007030B93C6F3CC
:10DAF00080160023A4F8743094F82030C3F3020396
:10DB00008DF8533001210DF153001CF0F8FC024652
:10DB1000002800F00A8100960B9B394650461EF003
:10DB200095F8B4F868300C93002608F80960A661EF
:10DB3000666166603123A360E66081497EA3D3E914
:10DB40000023A0FB0101FFF74BFB20F07F40206189
:10DB50001CF028FF0B90D4F810908DF84760666C8D
:10DB600046B1366896F8563003F00303012B00F0F7
:10DB7000A7800026276C002F00F0BD803F680B9B1C
:10DB800009EB030808F10208384600F095F98246CF
:10DB9000002E00F0AD803B69034408EB0302023223
:10DBA0003146204600F060FB002840F0A9809DF837
:10DBB000473084F8253001230F93A26E910F930014
:10DBC000981841F10001C90041EA5071C000801A63
:10DBD00061F10001090141EA10710001801841F171
:10DBE000000142F6DC33C01840F2E2424FF000037D
:10DBF00041F10001FFF7F4FA3887524641463846B2
:10DC000000F086F900287BD101230E93022315939F
:10DC100009F24712DFF82C816B000D9305EB4503E9
:10DC200048F823204FF0000A4748DDF830E0AEFB0B
:10DC3000000141A3D3E900234FF0910C0CFB0E111E
:10DC4000FFF7CEFAAA1C0D9B1D4408EB850509952C
:10DC500015AD08953D4B079306943D4B0593CDF8C4
:10DC600010904FF6FF730393CDF808A020F07F408B
:10DC70000190CDF800A00B9BD2B20321504609F0D1
:10DC8000E1FC29460AF070FD002851D10E9A6AB1D4
:10DC900097F84A3062F3000387F84A300F9A2AB1A6
:10DCA00096F8563062F3410386F8563094F87C308B
:10DCB00043F0010384F87C3001201EF0D6FFE7E634
:10DCC0000DF1470301930022009213AB202120465F
:10DCD0000CF030F908B18346DAE604220DF14D016B
:10DCE00012A81BF003FD129930461EF0B4FB41E769
:10DCF000CDF83CB061E7CDF838B0CDF83CB085E761
:10DD00004FF00C0BC4E64FF00C0BC1E64FF00C0BC0
:10DD1000BEE64FF00C0BBBE64FF00C0BB8E64FF035
:10DD20000C0BB5E64FF0070BB2E64FF00C0BAFE66D
:10DD30004FF00C0BACE600BF8D49FD1A0700000048
:10DD400000CA9A3B503B0020002AE784D983010097
:10DD500049D70000000000002DE9F0418AB00446D8
:10DD60000E46174690F8213003F00708C3F38015DC
:10DD700090F82030C3F302038DF8233001210DF118
:10DD800023001CF0BCFB0246009543463946304652
:10DD90001DF05CFF1E491CA3D3E90023A0FB010179
:10DDA000FFF71EFA20F07F452169A94221D9491BBE
:10DDB000002302220992174AA21A1748A0FB020266
:10DDC0005209023209AE06961448059000200490CC
:10DDD00003900291019300900346D2B203211CF0FC
:10DDE000B9FD31460AF0C0FC50B925610AB0BDE862
:10DDF000F081A94202D26B1A0021DAE70020F5E790
:10DE00000C20F3E7AFF300808D49FD1A07000000F6
:10DE100000CA9A3BC4390020E1830F3ED983010038
:10DE20002DE9F0418AB005461EF006F91E491CA3F3
:10DE3000D3E90023A0FB0101FFF7D2F920F07F44D2
:10DE40002F69A74223D93F1B0026022309934C22A6
:10DE5000164928461CF017FBC2B205320DF1240802
:10DE6000CDF81880124B0593002004900390029780
:10DE7000019600900346D2B203211CF06BFD41468F
:10DE80000AF072FC50B92C610AB0BDE8F081A742DB
:10DE900002D2E61B0027D8E70020F5E70C20F3E7C5
:10DEA0008D49FD1A0700000000CA9A3BB83B0020CC
:10DEB000D98301000000000038B50446026A90F8DA
:10DEC0002D30043300EB8303517D043102EB8102DA
:10DED0009268196A1EF0B0F8002565603123A360CE
:10DEE000E560094906A3D3E90023A0FB0101FFF780
:10DEF00077F920F07F402061284638BDAFF30080DD
:10DF00008D49FD1A0700000000CA9A3B000000007E
:10DF10002DE9F0438DB0044688469146068F40F2C5
:10DF2000E24101FB06F600250570856145614C2242
:10DF300017491CF0A8FAC7B202230B93154912A384
:10DF4000D3E90023A6FB0101FFF74AF9226905374F
:10DF50000BAE0896104B07930694104B05934A445A
:10DF600004920395029520F07F400190009543466E
:10DF7000FAB2032128461CF0D2FC31460AF0F4FB29
:10DF80000DB0BDE8F08300BF8D49FD1A0700000009
:10DF9000B83B002000CA9A3BD9830100BD9C010018
:10DFA00038B51546041DC37813F0010F01D000F1F8
:10DFB0000A0413F0020F00D0063413F0080F00D04B
:10DFC00002341B48A1FB000C17A3D3E900234FF038
:10DFD000070E0EFB01C1FFF703F9401B154BA3FB16
:10DFE00000231A095B0C12D0134AA2FB0030C0F3C5
:10DFF00047136370C0F34430A37823F01F03184322
:10E00000A070237843F080032370204638BD6270EF
:10E01000C2F30422A37823F01F031343A3702378D1
:10E020006FF3C7132370F0E700CA9A3B00000000AB
:10E030008D49FD1A89888888B5814E1B0000000033
:10E040002DE9F0418AB08046476C58227C493868F7
:10E050001CF019FAC6B20636F6B2FF238DF81D3051
:10E0600000230993089304252BE00221002009F0E6
:10E070000FFC069B022BF8D039E040F28763714A0F
:10E08000714972481AF0C1FD404080F311884FF089
:10E09000030002DF2EE040F289636A4A6C496B4854
:10E0A0001AF0B3FD404080F311884FF0030002DF07
:10E0B00025469DF81D30FF2B25D09DF81D30B3421D
:10E0C0002FD0089C0221069106AB0593614B049367
:10E0D0000020039002900DF11E03019309AB009301
:10E0E00008AB0DF11D0209F08DFB0228C1D0069B83
:10E0F000002BC2D1089BA342DBD06C1EE4B2002DE2
:10E10000C9D02546D5E740F28B634E4A52494F4865
:10E110001AF07BFD404080F311884FF0030002DFCE
:10E12000CBE7099D6B1CBB62D8F84020137CDBB2A7
:10E13000517C8B4203D00133DBB2022B6CD002EB5B
:10E1400083035A69141DD37813F0010F01D002F133
:10E150000A0413F0020F00D0063413F0080F00D0A9
:10E16000023413F0100F00D003343C48A5FB00012B
:10E1700031A3D3E90023072606FB0511FFF730F88A
:10E180000346B0F5161F05D3A0F51613627842F0CA
:10E1900040026270324AA2FB03121109520C3DD0B8
:10E1A000304AA2FB0323C3F347122270C3F3443364
:10E1B000627822F01F0213436370DBB243F0200346
:10E1C0006370BB8A3A8A1344BDF81E2012FA83F3A7
:10E1D0009AB2238297F8243097F825108B4205D005
:10E1E000F88C121A12F4004F00D10B4603EB4301D6
:10E1F0004900183105223944201D1BF077FA237A93
:10E2000003F01F0323721EF0B1FD237A43EA40138B
:10E2100023720AB0BDE8F081002390E72170C1F3BA
:10E220000421637823F01F0319436170CBB26FF3AD
:10E2300045136370C5E700BF00CA9A3B00000000A9
:10E24000283C0020A823030038230300681903009A
:10E25000402303000BC30200702303008D49FD1A05
:10E2600089888888B5814E1B2DE9F0478CB00C4613
:10E27000174600260E708E614E6191F849300A33C0
:10E2800001EB83035B6A597820461EF0C4F8666090
:10E290003123A360E6602A4D27A3D3E90023A0FB26
:10E2A0000501FEF79DFF20F07F402061B4F8548007
:10E2B00040F2E24000FB08F85822224920461CF0B8
:10E2C000E2F85FFA80FA02230B93A8FB05581AA321
:10E2D000D3E9002328464146FEF782FF20F07F491C
:10E2E0001948A9FB0001072303FB0911281A4FF461
:10E2F0007A724FF0000368EB0101FEF771FF2369AA
:10E300000AF106020BAD08951049079106941049D1
:10E310000591049303960290CDF8049000963B4635
:10E32000D2B2032130461CF0FAFA29460AF01CFA50
:10E330000CB0BDE8F08700BF8D49FD1A0700000052
:10E3400000CA9A3B283C00208D49FD1AD983010060
:10E35000ADA90100000000002DE9F0418AB005469A
:10E3600049781EF058F820491DA3D3E90023A0FBEB
:10E370000101FEF735FF20F07F442E69A64222D925
:10E38000A6EB0408002602230993582217492846C1
:10E390001CF079F8821D09AF0697154B05930020F4
:10E3A00004900390CDF80880019600900346D2B205
:10E3B00003211CF0CFFA39460AF0D6F958B92C617E
:10E3C0000AB0BDE8F081A64203D2A61B4FF00008B8
:10E3D000D9E70020F4E70C20F2E700BFAFF300809C
:10E3E0008D49FD1A0700000000CA9A3B283C002016
:10E3F000D9830100000000002DE9F04F8FB00B9091
:10E400000DF136010DF137001DF0B5FB9DF837A079
:10E410009DF836B01CF0C6FA0A90DFF8BC90D9F827
:10E4200000500027DFF8B480A5FB086528A3D3E9D6
:10E43000002330462946FEF7D3FE20F07F442848CB
:10E44000A4FB0001072303FB0411301A4FF47A7276
:10E450004FF0000365EB0101FEF7C2FE0546D9F857
:10E4600004001BA3D3E90023A0FB0801FEF7B8FEBC
:10E47000089707970B9A06921A4B059320F07F4056
:10E48000049003970295019400970A9B5A46032132
:10E4900050461CF044FA08B1022816D1124A002353
:10E4A000124814F0ADFF20B90B4BD8680FB0BDE88F
:10E4B000F08F002300939DF8362003219DF837004C
:10E4C00009F062F96FF07300F0E76FF08B00EDE791
:10E4D0008D49FD1A07000000984E002000CA9A3BA3
:10E4E0008D49FD1A29FD0100447B0B00A84E002038
:10E4F00068B505461CF056FA0D4EB1681CF056FA88
:10E50000B0FBF5F5054471680A4807A3D3E9002379
:10E51000A1FB0001FEF764FE20F07F40854201D898
:10E52000002068BD0120FCE78D49FD1A07000000AE
:10E53000984E002000CA9A3B2DE9F04FC9B08246A0
:10E54000D0F808B0C3680193036902934369039349
:10E5500083690493C3690593036A0693436A079327
:10E56000002205E051F8223008A840F8223001329C
:10E570000F2AF7DD102222E0931E08A951F823107C
:10E580004FEAF14383EA714383EA9123D11F08A83C
:10E5900050F821100B44A2F10F0150F821004FEA6E
:10E5A000B04181EAF01181EAD0010B44A2F11001DF
:10E5B00008A850F821100B4440F8223001323F2ABD
:10E5C000DADDDDF81CE0069E059F049ADDF80C807C
:10E5D000029C019DDC4600202FE04FEAF22383EAF3
:10E5E000B21383EA7263734402EA070126EA020E59
:10E5F00081EA0E010B44234951F820100B4408A96D
:10E6000051F820100B444FEA7C3181EABC0181EAC9
:10E61000BC5185EA040E0EEA0C0E05EA04098EEAE6
:10E62000090E71440130B6463E46174608EB030218
:10E63000A0462C46654603EB010C3F28CDDD0CEBD4
:10E640000B03CAF80830019B1D44CAF80C50029B0A
:10E650001C44CAF81040039B4344CAF81430049B7E
:10E660001A44CAF81820059B1F44CAF81C70069B60
:10E670001E44CAF82060079B7344CAF8243049B08E
:10E68000BDE8F08F800E03000023036043600B4B56
:10E6900083600B4BC3600B4B03610B4B43610B4B14
:10E6A00083610B4BC3610B4B036203F17453A3F5FE
:10E6B0002303A3F692434362704700BF67E6096AEB
:10E6C00085AE67BB72F36E3C3AF54FA57F520E5193
:10E6D0008C68059BABD9831F00EB4000014B03EB1B
:10E6E000C00070473C1B0020024B40F2231202FB8B
:10E6F00000307047F4180020002800F0A9802DE9B0
:10E70000F043A1B00D461646074602F1020902F594
:10E710008B7802F21D1406A8FFF7B6FF202207F13E
:10E72000100106A818F01DFE0A22494606A818F096
:10E7300018FEF27806F10C0106A818F012FE02226B
:10E7400006F58A7106A818F00CFE0722414606A8B5
:10E7500018F007FE04A906A818F04CFE0622214670
:10E7600004A81AF09EFF18B1002021B0BDE8F08384
:10E7700096F8169100220023CDE9022306F217181D
:10E780000622414602A81AF0B1FF002D62D00024F3
:10E7900001E00134A4B22A88A24213D9F17904EB32
:10E7A000C4032B44DB789942F3D1317A04EBC403E0
:10E7B0002B441B799942ECD104EBC40028448378A4
:10E7C0004B45E6D1A2421AD10F2A45D8029B2549D2
:10E7D0005B18039941F10001F868D7F808C0634558
:10E7E00071EB00033AD3F17904EBC4032B44D970E5
:10E7F000317A197183F8029001322A8013E00022E5
:10E800000023CDE9002304EBC4012944062205318D
:10E8100068461AF06BFF029B009A9A42039B019A8A
:10E8200072EB030312D204EBC4042C4406224146CB
:10E83000601D1AF05BFF029A039BB868F96890426A
:10E8400099410DD2BA60FB6001208EE700208CE771
:10E8500001207047002088E7002086E7002084E739
:10E86000012082E7808D5B0000B54FF48C7C4FF077
:10E87000000EE64520D20EEB0C0301335A0823F0BC
:10E88000010101EB53030E4951F8233083420ED8A6
:10E8900083420FD302EB4203094951F823308342EC
:10E8A0000CD102EB420201EB82005DF804FB02F1A5
:10E8B000FF3CDEE79646DCE77246EBE70020F4E734
:10E8C0005401030038B50B78032B14D00C46022BEF
:10E8D00024D0052B21D1224B1B784FF40C722149F7
:10E8E00002FB03118368DC686423A0471E4A936817
:10E8F0000133936011E01A4A1378B3FA83F35B098A
:10E9000013704FF40C7281680C69164902FB0311F5
:10E91000A047154A53680133536038BD8D6800E045
:10E920000135A368E2681344B3F50C7F28BF4FF4A8
:10E930000C73AB42F1D961680C4B0D4A495D002064
:10E9400018F0D8FF0028EBD000220023084909481E
:10E9500014F06CFB044A136801331360E0E700BF56
:10E96000525A0020B81E0020542400203C240020CD
:10E97000182300206007002008B502488368DB697F
:10E98000984708BD78F902002DE9F0478CB006469B
:10E99000894617461D46FFF79FFE0446037B13F08A
:10E9A000020A08D103690BB31B7813F0010F20D1C1
:10E9B0004FF0000801E04FF00008BAF1000F1FD03F
:10E9C000B9F1FF0F18D8FE238DF824308DF82550AB
:10E9D000A3798DF82630624B1A788DF827205B7862
:10E9E0008DF828308DF82990052333E04FF000088A
:10E9F000E3E74FF00108E0E7A3780133A3709AE062
:10EA0000B8F1000F01D04FF0010A9DF850103846C0
:10EA100018F089FD0546FD238DF824308DF825007A
:10EA20008DF826A000238DF82730A3798DF82830A3
:10EA30004B4B1A788DF829205B788DF82A308DF8A9
:10EA40002B904FEA19238DF82C304FEA19498DF895
:10EA50002D900923A2790132A2711FFA83F9484649
:10EA60004FF6FF7C0DF1250216E012F801EB5FFA7C
:10EA70008CF08EEA000E8EEA0E1E5FFA8EFE4FEAD2
:10EA80001C2C4CEA0E2C0FFA8CFC8CEACE0C8CEA77
:10EA90001E1C1FFA8CFC0846411E89B20028E4D1D6
:10EAA0001FFA85FA3A46504615E012F8010B5FFA54
:10EAB0008CFE80EA0E0080EA0010C0B24FEA1C2CE7
:10EAC0008CEA002C0FFA8CFC8CEAC00C8CEA101C2F
:10EAD0001FFA8CFC0846411E89B20028E5D15FFA76
:10EAE0008CF19DF854204A4082EA0212D1B24FEADA
:10EAF0001C2282EA012212B282EAC10282EA1112C7
:10EB00008DF82020C2F307228DF82120B8F1000FE4
:10EB100014D1002409F1010209A9304618F00EFFB2
:10EB200052463946304618F009FF022208A93046FD
:10EB300018F004FF74B90CB0BDE8F087206908AA8A
:10EB4000029201950097013309AA04A918F0A4FCC8
:10EB50000446DFE7A2B204A9304618F0EFFEEAE768
:10EB600044010020F0B589B002AF684C204619F08E
:10EB70006CF994F85142002C00F0A482C4F109040D
:10EB8000624B93F8503214FB03F4A4B2C4F1E404D2
:10EB9000A4B2FA233B72FF237B720D23BB725C4A43
:10EBA0001378591C1170FB72251DFA2D00F28D820D
:10EBB000584E042207F1080130461AF097FD22460C
:10EBC0005549301D1AF092FD6C4688B002A96B467B
:10EBD00013F1180253D00C231AB1042B01DD4F4856
:10EBE000486112B1082B00DD8D610B2B4ADD0C2032
:10EBF00052B10023032666F307036FF30F236FF36D
:10EC000017436FF31F630B6100216FF300016FF374
:10EC100041016FF382016FF3C501032363F3881190
:10EC200000F47B7363F352216FF3DE416FF3DF7106
:10EC300000233B481AF03BFBA5463A4916230B70CC
:10EC4000344B4B604D70384B186800230093012201
:10EC50001BF08DFB0446C0B92C4B93F83333002BCB
:10EC60006AD1324B1B78002B00F07481304B1B783B
:10EC7000002B00F0D98120461C37BD46F0BD6FF057
:10EC80000043A9E76FF01B00B2E76D4688B002A908
:10EC90006B4613F1180232D00C231AB1042B01DD9C
:10ECA0002448486112B1082B00DD8C610B2B29DD53
:10ECB0000C2052B10023032666F307036FF30F23E2
:10ECC0006FF317436FF31F630B6100216FF30001B4
:10ECD0006FF341016FF382016FF3C501032363F307
:10ECE000881100F47B7363F352216FF3DE416FF3FD
:10ECF000DF7100230A481AF0DAFAAD46BBE76FF07D
:10ED00000043CAE76FF01B00D3E700BF6C1B002075
:10ED1000585A0020F8170020BB1D002048FD0200B3
:10ED200040FB0200F017002098140020555A0020E4
:10ED3000535A00205CFD0200AE481AF094FC82B2E7
:10ED40001346042A28BF0423DBB2002A89D0D01A34
:10ED5000A94DA84B0344A94AA949284605F042FFFA
:10ED6000A84928461AF092FC002800F09F80022350
:10ED70003B716D4688B002AE6B4613F118027CD031
:10ED80000D201AB1042801DD9F4B736102233B71F2
:10ED90001AB1082801DD984BB36122B106F11C03BA
:10EDA000002100296CD00C2873DD0D205AB10023FE
:10EDB000032161F307036FF30F236FF3174301215F
:10EDC00061F31F63336100216FF300016FF34101B1
:10EDD0006FF382016FF3C501032363F38811C0F35E
:10EDE000090363F352216FF3DE416FF3DF710023F8
:10EDF00086481AF05CFAAD467F4807F0DFF9054611
:10EE000000284FD06C4688B002A96B4613F1180257
:10EE100042D00C231AB1042B01DD7D48486112B1A8
:10EE2000082B00DD8D610B2B39DD0C2052B1002346
:10EE3000032666F307036FF30F236FF317436FF394
:10EE40001F630B6100216FF300016FF341016FF34A
:10EE500082016FF3C501032363F3881100F47B7310
:10EE600063F352216FF3DE416FF3DF7100236748D4
:10EE70001AF01DFAA5462C46FDE66FF0004080E72B
:10EE800007F1180C8C441CF814CC03F801CB0131A9
:10EE900087E76FF01B0089E76FF00043BAE76FF078
:10EEA0001B00C3E7544957481AF0B9FB594B1B786C
:10EEB000002B7FF4D6AEBB81BB7307F10C01564B20
:10EEC000586807F07DFF054618B9524B01221A70A9
:10EED000C7E66C4688B002A96B4613F1180233D01E
:10EEE0000C231AB1042B01DD4C48486112B1082BE8
:10EEF00000DD8D610B2B2ADD0C2052B1002303268F
:10EF000066F307036FF30F236FF317436FF31F636A
:10EF10000B6100216FF300016FF341016FF3820178
:10EF20006FF3C501032363F3881100F47B7363F36C
:10EF300052216FF3DE416FF3DF71002333481AF083
:10EF4000B6F9A5462C4696E66FF00043C9E76FF088
:10EF50001B00D2E73B82BB7407F110012E4B1868EF
:10EF600007F02EFF054618B92D4B01221A707DE6D9
:10EF70006C4688B002A96B4613F1180233D00C23FB
:10EF80001AB1042B01DD2748486112B1082B00DDBE
:10EF90008D610B2B2ADD0C2052B10023032666F372
:10EFA00007036FF30F236FF317436FF31F630B61B7
:10EFB00000216FF300016FF341016FF382016FF3E2
:10EFC000C501032363F3881100F47B7363F35221BB
:10EFD0006FF3DE416FF3DF7100230C481AF067F91D
:10EFE000A5462C4647E66FF00043C9E76FF01B00CB
:10EFF000D2E700BF971B0020E017002088FD020029
:10F0000090FD0200A817002098FD020040FB0200BE
:10F01000B4FD0200565A002098140020D8FD0200CA
:10F02000555A002004FE0200BB82BB7507F1140193
:10F03000274B986807F0C4FE044618B9254B0122F7
:10F040001A7018E66D4688B002A96B4613F11802D3
:10F0500032D00C231AB1042B01DD1F48486112B1D4
:10F06000082B00DD8C610B2B29DD0C2052B1002315
:10F07000032666F307036FF30F236FF317436FF352
:10F080001F630B6100216FF300016FF341016FF308
:10F0900082016FF3C501032363F3881100F47B73CE
:10F0A00063F352216FF3DE416FF3DF7100230B48EE
:10F0B0001AF0FDF8AD46DEE56FF00043CAE76FF0E9
:10F0C0001B00D3E74FF0FF34D5E54FF0FF34D2E516
:10F0D00098140020535A00202CFE020040FB02002E
:10F0E000B0B500AF724B1B7863B9724B1B78002B25
:10F0F0004FD1714B1B78002B40F0928000242046AA
:10F10000BD46B0BD6D4B58681BF0F3F804460028AF
:10F11000EBD06D4688B06B4613F1100233D00C2152
:10F120001AB1042901DD6648586112B1082900DDD1
:10F130009C610B292ADD0C205AB100214FF0030CF1
:10F140006CF307016FF30F216FF317416FF31F612A
:10F15000196100216FF300016FF341016FF3820128
:10F160006FF3C501032363F3881100F47B7363F32A
:10F1700052216FF3DE416FF3DF71002351481AF023
:10F1800096F8AD46BBE76FF00041C9E76FF01B0092
:10F19000D2E74A4B18681BF0ACF804460028A8D008
:10F1A0006D4688B06B4613F1100233D00C211AB1B2
:10F1B000042901DD4448586112B1082900DD9C6131
:10F1C0000B292ADD0C205AB100214FF0030C6CF3FF
:10F1D00007016FF30F216FF317416FF31F6119617F
:10F1E00000216FF300016FF341016FF382016FF3B0
:10F1F000C501032363F3881100F47B7363F3522189
:10F200006FF3DE416FF3DF7100232E481AF04FF8E1
:10F21000AD4674E76FF00041C9E76FF01B00D2E71D
:10F22000264B98681BF065F8044600283FF467AF4A
:10F230006D4688B06B4613F1100233D00C211AB121
:10F24000042901DD2148586112B1082900DD9C61C3
:10F250000B292ADD0C205AB100214FF0030C6CF36E
:10F2600007016FF30F216FF317416FF31F611961EE
:10F2700000216FF300016FF341016FF382016FF31F
:10F28000C501032363F3881100F47B7363F35221F8
:10F290006FF3DE416FF3DF7100230A481AF007F8BD
:10F2A000AD462CE76FF00041C9E76FF01B00D2E7D5
:10F2B000565A0020555A0020535A00209814002016
:10F2C00058FE020040FB020084FE0200ACFE020079
:10F2D000F0B5C3B000AF07F58271052003F078FCEC
:10F2E0000025D7F804018468A54262D2641BB4F5F6
:10F2F000807F28BF4FF4807423463A1D29461AF0B8
:10F3000055F8002206E06FF0004512E06FF01B0593
:10F310001FE001321346944249D9391D895CFF2907
:10F32000F7D02B446C4688B0684610F11002EAD042
:10F3300010251AB1042D01DD204E466112B1082DB1
:10F3400000DD836112B10C2D00DDC1610F2DDDDD0B
:10F35000102552B10023042161F307036FF30F233B
:10F360006FF317436FF31F63036100216FF3000115
:10F370006FF341016FF382016FF3C501032363F360
:10F38000881105F47D7363F352216FF3DE416FF34F
:10F39000DF7100230A4819F08AFFA546D7F8040157
:10F3A0001AF003F8002007F58677BD46F0BD254426
:10F3B00097E719F0FAFF0120F5E700BFD8FE020039
:10F3C00040FB0200F0B5D7B002AF0446437A827A20
:10F3D00043EA0223C27A43EA024343F2732293428E
:10F3E0006BD843F26422934217D3A3F54953243BCD
:10F3F0000F2B00F28A83DFE813F044015F017A01EA
:10F40000A301BE01D9018803880388038803880308
:10F410008803880388038803F401832B4BD1C578C4
:10F42000FF22002107F108001AF08FF92A4604F1A3
:10F430000C0107F108001AF059F9BA4A93685268AA
:10F440009C1AFC2C28BFFC2438899108B64DA5FBDA
:10F450000151B0EBD10F00F05482B24C63683B60B5
:10F4600000203871787198230193062300933A465F
:10F470004CF25531FFF788FA20F0E2F84A0142EAEF
:10F48000D06243011B1A62EB0102920042EA9372BE
:10F490009B001B1842EB0102D20042EA5372C3F3F5
:10F4A000103343EA424323616368A1688B4280F0D2
:10F4B0006982FF202AE3FF2028E34CF25432934272
:10F4C00040F0DD80C5780A2D28BF0A250A220021D8
:10F4D00007F108001AF039F92A4604F10C0107F186
:10F4E00008001AF003F98F4B1B78002B40F09E8028
:10F4F000B968012018F031FAFD68854200F08C816E
:10F500006C4688B002A96B4613F1180200F0BD8169
:10F5100010231AB1042B01DD844E4E6112B1082B69
:10F5200000DD886112B10C2B00DDCD610F2B40F3A3
:10F53000AF81102052B10023042565F307036FF358
:10F540000F236FF317436FF31F630B6100216FF3FA
:10F5500000016FF341016FF382016FF3C5010323D3
:10F5600063F3881100F47D7363F352216FF3DE417E
:10F570006FF3DF7100236E4819F099FEA546694CC0
:10F5800000236360FB68E36001232370BB68A36012
:10F59000FFF7A6FD4FF40040002114F091FCA56890
:10F5A000E0686C4688B002A96B4613F1180200F0BF
:10F5B000728110231AB1042B01DD5E4E4E6112B12F
:10F5C000082B00DD8D6112B10C2B00DDC8610F2B03
:10F5D00040F36481102052B10023042565F3070332
:10F5E0006FF30F236FF317436FF31F630B6100215A
:10F5F0006FF300016FF341016FF382016FF3C501F7
:10F60000032363F3881100F47D7363F352216FF3D6
:10F61000DE416FF3DF710023454819F048FEA5462F
:10F62000454819F0BDFE002840F03B813D4C636821
:10F630003B60002038717871982301930623009372
:10F640003A464CF25531FFF79FF91FF0F9FF4A0196
:10F6500042EAD06243011B1A62EB0102920042EAC5
:10F6600093729B001B1842EB0102D20042EA5372D4
:10F67000C3F3103343EA42432361FF2046E2FF20F5
:10F6800044E2C5782C2D28BF2C252C22002107F11F
:10F6900008001AF05AF82A4604F10C0107F1080094
:10F6A0001AF024F807F10801244818F08DFC00280E
:10F6B00000F03082FF2029E2C5783B2D28BF3B2592
:10F6C0003B22002107F108001AF03FF82A4604F116
:10F6D0000C0107F108001AF009F807F108011748B2
:10F6E000FDF75AFF002800F01782FF200EE2C578D0
:10F6F000352D28BF35253522002107F108001AF0E5
:10F7000024F82A4604F10C0107F1080019F0EEFF75
:10F7100007F10801094818F097FC002800F0FE8165
:10F72000FF20F3E1C81600202108822010FF02000C
:10F7300040FB020048FF0200A41400206C1B0020C4
:10F74000C5782E2D28BF2E252E22002107F1080076
:10F7500019F0FBFF2A4604F10C0107F1080019F02B
:10F76000C5FF07F10801B24818F0AAFC002800F014
:10F77000D781FF20CAE1C578362D28BF362536222D
:10F78000002107F1080019F0E0FF2A4604F10C01FE
:10F7900007F1080019F0AAFF07F10801A448FDF7D6
:10F7A00067FF002800F0BE81FF20AFE1C5782B2D58
:10F7B00028BF2B252B22002107F1080019F0C5FFD7
:10F7C0002A4604F10C0107F1080019F08FFF07F138
:10F7D0000801974818F097FC002800F0A581FF2049
:10F7E00094E1C578F92D28BFF925F922002107F108
:10F7F000080019F0AAFF2A4604F10C0107F10800DD
:10F8000019F074FF07F10801894818F09FFC0028DF
:10F8100000F08C81FF2079E1864BC7F8343100235A
:10F82000022262F307036FF30F236FF317436FF3A3
:10F830001F63C7F8303100216FF300016FF34101FE
:10F840006FF382016FF3C501032363F3881108236B
:10F8500063F352216FF3DE416FF3DF71002307F58D
:10F860009872754819F023FD4FF0FF333B6000207C
:10F870003871787198230193062300933A464CF22D
:10F880005531FFF781F8FF2040E16FF0004340E67B
:10F890006FF01B004EE66FF000438BE66FF01B002D
:10F8A00099E6664BC7F81C310023022262F3070376
:10F8B0006FF30F236FF317436FF31F63C7F818310C
:10F8C00000216FF300016FF341016FF382016FF3C9
:10F8D000C501012363F38811082363F352216FF3F9
:10F8E000DE416FF3DF71002307F58C72524819F087
:10F8F000DEFC4FF40040002114F0E2FA02F0CCFCF0
:10F9000094E62244934214BF00230123224607F1C8
:10F910000A014B4819F011FD20B94A4A53682344A3
:10F9200053609AE5484BC7F84C310023022262F33A
:10F9300007036FF30F236FF317436FF31F63C7F8CA
:10F94000483100216FF300016FF341016FF3820131
:10F950006FF3C501012363F38811082363F3522178
:10F960006FF3DE416FF3DF71002307F5A4723248B5
:10F9700019F09DFC4FF40040002114F0A1FA02F0B0
:10F980008BFCCAE7002017F0E8FFE16881425FD0F6
:10F990002C4B9E686C468AB002AD6B4613F1180280
:10F9A00000F0AD8014232AB1042B03DDDFF89CC0E6
:10F9B000C5F814C012B1082B00DDAE6112B10C2BDA
:10F9C00000DDE86112B1102B00DD2962132B40F33A
:10F9D0009980142052B10023052161F307036FF3CE
:10F9E0000F236FF317436FF31F632B6100216FF336
:10F9F00000016FF341016FF382016FF3C501012331
:10FA000063F3881100F47D7363F352216FF3DE41D9
:10FA10006FF3DF710023084819F049FCA5464FF445
:10FA20000040002114F04CFA02F036FCFF206DE09B
:10FA30006C1B0020F4FE020040FB020074FF020079
:10FA4000A4140020C81600208CFF0200C8FF02008A
:10FA50006C4688B002AD6B4613F1180249D00C23F6
:10FA60001AB1042B01DD3249696112B1082B00DDA6
:10FA7000A8610B2B40DD0C2352B10021032060F361
:10FA800007016FF30F216FF317416FF31F612961B6
:10FA900000216FF300016FF341016FF382016FF3F7
:10FAA000C501032060F3881103F47B7363F35221D3
:10FAB0006FF3DE416FF3DF7100231E4819F0F7FB8F
:10FAC000A5464FF0FF333B600020387178719823D2
:10FAD0000193062300933A464CF25531FEF754FF4A
:10FAE0004FF40040002114F0EBF901201DF05AFB07
:10FAF00095E76FF00043B3E76FF01B03BCE76FF0CF
:10FB0000004350E76FF01B0064E7FF2007F5AA777A
:10FB1000BD46F0BD0020F9E70120F7E70220F5E738
:10FB20000320F3E70420F1E70520EFE70F20EDE7DE
:10FB3000A4FF020040FB020090B585B002AFFA239B
:10FB40003B71FF237B710D23BB71764A1378591CDF
:10FB50001170FB71744B1B78042B00F29180DFE86D
:10FB600003F0032B445D7600704B93F8353383B973
:10FB700000206D490A7801326D4B83FB02435B1014
:10FB800003EB8303D31A0B7000287BD10C37BD46DF
:10FB900090BD684C0422B918204619F0A7FD19221F
:10FBA0006549201D19F0A2FD644B16221A705C6095
:10FBB0001D225A700120DCE75C4B93F833330BB9FC
:10FBC0000020D6E75B4C0422B918204619F08EFDC0
:10FBD00019225B49201D19F089FD584B16221A7015
:10FBE0005C601D225A700120C3E7504B93F84633E6
:10FBF0000BB90020BDE74F4C0422B918204619F07C
:10FC000075FD19224F49201D19F070FD4B4B16222E
:10FC10001A705C601D225A700120AAE7434B93F8CA
:10FC200047330BB90020A4E7424C0422B918204600
:10FC300019F05CFD19224449201D19F057FD3F4B76
:10FC400016221A705C601D225A70012091E7374B12
:10FC500093F848330BB900208BE7364C0422B918CF
:10FC6000204619F043FD19223849201D19F03EFDA8
:10FC7000324B16221A705C601D225A70012078E700
:10FC8000002076E7324B98680023009301222B492D
:10FC90001AF06DFB014600283FF478AF6C4688B03F
:10FCA0000DF1080C6B4613F1180235D00C2322B16C
:10FCB000042B02DD2748CCF814001AB1082B01DD13
:10FCC000CCF818100B2B2ADD0C205AB1002303218D
:10FCD00061F307036FF30F236FF317436FF31F6392
:10FCE000CCF8103000216FF300016FF341016FF386
:10FCF00082016FF3C501032363F3881100F47B7362
:10FD000063F352216FF3DE416FF3DF71002312487A
:10FD100019F0CDFAA54639E76FF00043C7E76FF059
:10FD20001B00D2E7575A0020545A00206C1B0020B9
:10FD300067666666C0170020C71B0020B817002042
:10FD4000951B0020701D0020891D0020A21D002091
:10FD5000981400205CFD020040FB02002DE9F041F8
:10FD6000F0B002AFFFF7B4FA002800F0138100F002
:10FD700093FE054600283AD06C4688B002A96B462F
:10FD800013F1180200F077810C231AB1042B01DD66
:10FD9000BD48486112B1082B00DD8D610B2B40F38B
:10FDA0006D810C2052B10023032565F307036FF327
:10FDB0000F236FF317436FF31F630B6100216FF382
:10FDC00000016FF341016FF382016FF3C50101235D
:10FDD00063F3881100F47B7363F352216FF3DE4108
:10FDE0006FF3DF710023A94819F061FAA5461C20C2
:10FDF00000F05AFE054600283AD06C4688B002A9A9
:10FE00006B4613F1180200F03C810C231AB1042B4D
:10FE100001DD9F48486112B1082B00DD8D610B2B7D
:10FE200040F346810C2052B10023032565F30703FC
:10FE30006FF30F236FF317436FF31F630B61002101
:10FE40006FF300016FF341016FF382016FF3C5019E
:10FE5000012363F3881100F47B7363F352216FF382
:10FE6000DE416FF3DF710023884819F020FAA546C0
:10FE7000012000F021FE054600283AD06C4688B0EB
:10FE800002A96B4613F1180200F015810C231AB178
:10FE9000042B01DD7F48486112B1082B00DD8D6124
:10FEA0000B2B40F30B810C2052B10023032565F38B
:10FEB00007036FF30F236FF317436FF31F630B6198
:10FEC00000216FF300016FF341016FF382016FF3C3
:10FED000C501012363F3881100F47B7363F352219E
:10FEE0006FF3DE416FF3DF710023684819F0DFF92B
:10FEF000A54669481EF07FFE002800F0E2806748B2
:10FF000017F023FF64488368DC6864234FF40C72A5
:10FF10006349A0470546002800F006816C4688B07A
:10FF200002A96B4613F1180200F0F8800C231AB1F5
:10FF3000042B01DD5B48486112B1082B00DD8D61A7
:10FF40000B2B40F3EE800C2052B10023032565F308
:10FF500007036FF30F236FF317436FF31F630B61F7
:10FF600000216FF300016FF341016FF382016FF322
:10FF7000C501032363F3881100F47B7363F35221FB
:10FF80006FF3DE416FF3DF710023404819F08FF902
:10FF9000A546BEE0444BC7F86C310023022262F351
:10FFA00007036FF30F236FF317436FF31F63C7F854
:10FFB000683100216FF300016FF341016FF382019B
:10FFC0006FF3C501032363F38811082363F3522100
:10FFD0006FF3DE416FF3DF71002307F5B4722B4836
:10FFE00019F065F905201DF0E5F8054600283FF4F5
:10FFF000BEAE6C4688B002A96B4613F1180234D02D
:020000040001F9
:100000000C231AB1042B01DD2848486112B1082BDA
:1000100000DD8D610B2B2BDD0C2052B1002303255D
:1000200065F307036FF30F236FF317436FF31F633A
:100030000B6100216FF300016FF341016FF3820147
:100040006FF3C501012363F3881100F47B7363F33D
:1000500052216FF3DE416FF3DF7100230B4819F07B
:1000600026F9A54602F018F981E66FF00043C8E7CB
:100070006FF01B00D1E76FF0004386E66FF01B00C6
:1000800090E66FF00043C1E63C00030040FB020035
:100090005C0003007C00030078F902006C1B002068
:1000A000B81E0020B80003000C0003001C00030071
:1000B0006FF01B00B7E66FF00043E8E66FF01B003F
:1000C000F2E6B14BC7F8B4310023022262F3070312
:1000D0006FF30F236FF317436FF31F63C7F8B0314C
:1000E00000216FF300016FF341016FF382016FF3A1
:1000F000C501032363F38811082363F352216FF3CF
:10010000DE416FF3DF71002307F5D8729F4819F0C5
:10011000CEF807F5DC77BD46BDE8F0816FF000430F
:1001200005E76FF01B000FE7994B9B681B681BB13D
:100130000022984996489847002006F05FF8054647
:1001400000283FD06C4688B002A96B4613F1180214
:1001500032D00C231AB1042B01DD8F48486112B153
:10016000082B00DD8D610B2B29DD0C2052B1002303
:10017000032565F307036FF30F236FF317436FF343
:100180001F630B6100216FF300016FF341016FF3F7
:1001900082016FF3C501032363F3881100F47B73BD
:1001A00063F352216FF3DE416FF3DF710023774871
:1001B00019F07DF8A546ACE76FF00043CAE76FF091
:1001C0001B00D3E7754BC7F884310023022262F38A
:1001D00007036FF30F236FF317436FF31F63C7F822
:1001E000803100216FF300016FF341016FF3820151
:1001F0006FF3C501032363F38811082363F35221CE
:100200006FF3DE416FF3DF71002307F5C0725F48C3
:1002100019F04DF8624A0021624806F0A1FD00285D
:100220007FF477AF604A0021604806F099FD00280E
:100230007FF46FAF5E4A00215E4806F091FD002812
:100240007FF467AF5C4BC7F89C310023022262F356
:1002500007036FF30F236FF317436FF31F63C7F8A1
:10026000983100216FF300016FF341016FF38201B8
:100270006FF3C501032363F38811082363F352214D
:100280006FF3DE416FF3DF71002307F5CC723F4857
:1002900019F00DF84FF0000846460422002307F13C
:1002A0003401464812F01EFF05461FF0C9F94A0105
:1002B00042EAD06243011B1A62EB0102940044EA55
:1002C00093749B001B1844EB0104E40044EA53744C
:1002D000C3F3103343EA44447DB1A31BB3F57A7FE3
:1002E00018D8A4EB0803962BD7D9354B1B78002BD5
:1002F000D3D1FFF721FCA046CFE707F13400FFF789
:1003000061F8FF28E9D02E4B1B78002BE5D1FEF7D2
:1003100029FCE2E70020386022233B7103237B7134
:10032000B871F8713B7232230193092300933A4666
:100330000146FEF729FB224B1B7893B101233B704A
:1003400032222049F81819F0D1F98B230193332375
:1003500000933A4643F276210020FEF715FB26462D
:10036000BFE700253D7032221749781C19F0BEF90D
:100370008B230193332300933A4643F27621284698
:10038000FEF702FB2646ACE7A000030040FB02009C
:1003900078F90200C5E80000DC000300FC0003005F
:1003A00098140020080100209C1400201C0100204B
:1003B000A014002030010020140103006007002079
:1003C000C81600203C01030084FD020038B5044635
:1003D0000D461149FCF7A0FE50B100232B704FF0E1
:1003E00081412046FCF7F0FCFCF7DAFEC0B238BDD4
:1003F00001232B7008492046FCF7DCFB4FF07D51B0
:10040000FCF796FDFCF7A6FEFF230022C11717F0AC
:10041000D4FAC0B2EBE700BF00007F4208B508493C
:10042000FCF7CAFB0146FCF7C7FBFCF793FE4FF64F
:10043000FF730022C11717F0C0FA80B208BD00BFD9
:1004400000007A4408B5054BA3FB00300021FF23D0
:100450000A46C00817F0B1FAC0B208BDCDCCCCCC6A
:1004600010B504460B49FCF743FE10B14FF6FF7080
:1004700010BD09492046FCF7A7FCFCF7A5F814F0CD
:10048000ABFA48F6A0430022C11717F096FA80B2E3
:10049000EEE700BF00FF7F470000204180B110B5AC
:1004A00004464022002119F050F9064B6360064BC8
:1004B000A360064BE360064B23626362E36210BDF8
:1004C000704700BF0080B44300007F4300007C42BF
:1004D00000007AC460B110B504463022002119F042
:1004E00034F901232383034BE3612362A36210BD2C
:1004F000704700BF00007AC4002800F07981F0B591
:1005000083B00C460546002900F074810F220021BB
:10051000207817F06FFA002800F06E810122002188
:1005200094F8280017F066FA002800F068810F227E
:10053000002194F8300017F05DFA002800F0618186
:100540000F22002194F8310017F054FA002800F02F
:100550005A810F22002194F8320017F04BFA00283C
:1005600000F053810F22002194F8330017F042FA73
:10057000002800F04C810F22002194F8340017F07D
:1005800039FA002800F04581666800213046FCF702
:10059000B9FD002840F03F81B4493046FCF7D0FD5A
:1005A000002840F03A81B2493046FCF7C9FD30B12D
:1005B000AE493046FCF7A6FD002840F03081A66821
:1005C00000213046FCF79EFD002840F02A81A94911
:1005D0003046FCF7B5FD002840F02581A64930469D
:1005E000FCF7AEFD30B1A3493046FCF78BFD002887
:1005F00040F01B81E668A1493046FCF783FD0028E6
:1006000040F015819E493046FCF79AFD002840F0E5
:1006100010819C493046FCF793FD30B19849304633
:10062000FCF770FD002840F00681D4E90467002241
:10063000954B30463946FCF791FA002840F0FD8092
:100640000022924B30463946FCF7A6FA002840F0CB
:10065000F680D4E9066700228D4B30463946FCF718
:100660007DFA002840F0ED8000228A4B3046394662
:10067000FCF792FA002840F0E680266A8649304668
:10068000FCF740FD002840F0E08084493046FCF74C
:1006900057FD002840F0DB80666A7F493046FCF752
:1006A00031FD002840F0D5807C493046FCF748FDFC
:1006B000002840F0D080E66A77493046FCF722FDFA
:1006C000002840F0CA8075493046FCF739FD002803
:1006D00040F0C580A66B00213046FCF713FD0028D2
:1006E00040F0BF806E493046FCF72AFD30B16D49BD
:1006F0003046FCF7FDFC002800F0B5802B78012285
:1007000062F307132B70DBB2022262F303032B7038
:1007100022786B7862F307136B70DBB26FF3C3035D
:100720006B700DF10701606817F06EF9A8706B78B7
:100730009DF8072062F341036B700DF10701A0687B
:10074000FFF744FEE8706B789DF8072062F3000322
:100750006B70E06817F040F92871D4E90401FCF7E8
:1007600003FFC5F80500D4E90601FCF7FDFEC5F856
:100770000900206AFFF752FEA5F80D00606AFFF736
:100780004DFEA5F80F0094F828206B7862F38203E1
:100790006B70E06AFFF742FEA5F8110094F8302074
:1007A000EB7C62F30303EB7494F83120DBB262F369
:1007B0000713EB7494F832202B7D62F307132B752B
:1007C00094F83320DBB262F303032B7594F83420E2
:1007D000EB7D62F30303EB75DBB26FF30713EB758D
:1007E000A06BFFF73DFEA5F815000020287604E079
:1007F00001207047012000E0012003B0F0BD01207E
:10080000FBE70120F9E70120F7E70120F5E70120E8
:10081000F3E70120F1E70120EFE70120EDE70120F8
:10082000EBE70120E9E70120E7E70120E5E7012008
:10083000E3E70120E1E70120DFE70120DDE7012018
:10084000DBE70120D9E70120D7E70120D5E7012028
:10085000D3E70120D1E70120CFE70120CDE7012038
:10086000CBE70120C9E70120C7E700BF0080B44300
:100870000000B44300007F4300407E43000078C284
:1008800000007C4200007842008056C00080564044
:10089000008066C00080664000007AC4002FF846E1
:1008A0000000614500FF7F47002800F0C680F8B5D2
:1008B0000C460546002900F0C28003220021207862
:1008C00017F098F8002800F0BC800722002160781B
:1008D00017F090F8002800F0B6800F22002194F85D
:1008E000240017F087F8002800F0AF800F220021C5
:1008F00094F8250017F07EF8002800F0A880D4E9CD
:10090000026700225E4B30463946FCF727F9002883
:1009100040F09F8000225B4B30463946FCF73CF9A3
:10092000002840F09880D4E904670022564B3046F6
:100930003946FCF713F9002840F08F800022534B12
:1009400030463946FCF728F9002840F08880628B51
:1009500040F6F6139A4200F28480E6694C4930462C
:10096000FCF7D0FB00287ED14A493046FCF7E8FB73
:1009700000287AD1266A46493046FCF7C3FB002896
:1009800075D144493046FCF7DBFB002871D1A66ADB
:100990003F493046FCF7B6FB00286CD13D49304654
:1009A000FCF7CEFB002868D12B78042262F30713F2
:1009B0002B70DBB2022262F303032B706B786FF3B0
:1009C00047136B702278DBB262F301036B706278BD
:1009D000DBB262F384036B70D4E90201FCF7C4FD5F
:1009E000C5F80200D4E90401FCF7BEFDC5F8060015
:1009F000238B6B81608BFFF725FD2873E069FFF780
:100A00000DFDA5F80D00206AFFF708FDA5F80F0001
:100A100094F824206B7C62F307136B7494F8252000
:100A2000DBB262F303036B74A06AFFF7F7FC688222
:100A3000E36A6B610020287604E001207047012002
:100A400000E00120F8BD0120FCE70120FAE70120C9
:100A5000F8E70120F6E70120F4E70120F2E70120A2
:100A6000F0E70120EEE70120ECE70120EAE70120B2
:100A7000E8E70120E6E70120E4E70120E2E700BF24
:100A8000008056C000805640008066C000806640EE
:100A900000007AC4002FF84608B5024B1B681B689B
:100AA000984708BD6024002008B5024B1B689B696D
:100AB000984708BD6024002008B5024B1B681B6ADC
:100AC000984708BD6024002018B1034A1060002038
:100AD00070476FF0150070476024002008B9024885
:100AE00070470248704700BF640100206C0100207D
:100AF000054B984204D0054B984203D00020704724
:100B0000002070470120704718F9020000F9020028
:100B10002DE9F04105460F4616469846FFF7DEFFE1
:100B2000002D39D1002E39D0364B93F84D20437922
:100B3000B34237D00479A4006034E4B204F18044B5
:100B400004F5C044002E4ED02E4B1B6D03F5A0764D
:100B50000021C3F84011D3F84011C3F84085D3F801
:100B6000001241F4807141F00101C3F800122648DF
:100B700002F1A20140F8316000EBC1014C6001219B
:100B800001FA02F2C0F80425AFB9196005F18045F9
:100B900005F58055296033E00425C3E7194B93F828
:100BA0004E20C4E70479A4003034E4B204F1804458
:100BB00004F5C044C6E7134A92F84C00124A00F10B
:100BC000A20142F8317002EBC1014B6005F1804592
:100BD00005F5805500F5117342F823500123834039
:100BE000C2F804350CE0084902F1A20341F8337061
:100BF00001EBC3035C60012303FA02F2C1F8042590
:100C0000BDE8F0814801002000F0014038B51446ED
:100C1000134B0222BFF35B8F53E8005F012D04D119
:100C200043E8002CBCF1000FF6D1BFF35B8F14D169
:100C30000C4B18600C4D2960234601220146002010
:100C4000FFF766FF296809B9002038BD2346002256
:100C50001046FFF75DFF0020F7E76FF00F00F4E7A5
:100C60006C2400206424002068240020244B93F886
:100C70004D2001219140234BC3F80815A2320021D9
:100C800043F8321003EBC203596059601E4B1B68D6
:100C9000ABB11B4B93F84C3001219940194AC2F873
:100CA000081503F1A200002142F8301002EBC00049
:100CB000416003F5117342F8231042F82310134BDF
:100CC0001B687BB10E4B93F84E20012191400D4BD8
:100CD000C3F80815A232002143F8321003EBC20317
:100CE000596059600A4B0122BFF35B8F53E8001F24
:100CF00043E800200028F9D1BFF35B8F704700BFA5
:100D00004801002000F001406424002068240020F5
:100D10006C24002008B5084BD3F8503603F00103CB
:100D200020B1184617F06FFA0B3808BD184617F0B7
:100D300040FA0B38F9E700BF0010004008B50E4834
:100D400011F0A6FA0D4B98420DD10D4811F0A0FA02
:100D50000A4B98420AD10B4811F09AFA074B984275
:100D600007D1002008BD6FF00500FBE76FF005001C
:100D7000F8E76FF00500F5E7950100200000AD0BE6
:100D8000960100209401002038B53F4811F050F939
:100D90003E4B984271D13E4CE06AFFF7A9FE94F8B1
:100DA000303003F01F0343EA4013E361012384F86A
:100DB000213004F1280011F03BF9344B98425FD107
:100DC000606BFFF795FE94F8383003F01F0343EA99
:100DD00040136362012384F8293094F82000E2690B
:100DE00094F8211059402B4B00F5A27053F8205075
:100DF00025F4991525F4F85543F8205053F8205060
:100E0000120202F47C52090501F480110A432A43BC
:100E100043F8202094F8202002F5A27253F8221003
:100E200041F0030143F8221094F82800626A94F814
:100E3000291081F0010100F5A27053F8205025F42B
:100E4000991525F4F85543F8205053F82050120214
:100E500002F47C52090501F480110A432A4343F845
:100E6000202094F8282002F5A27253F8221041F0B5
:100E7000030143F82210002038BD6FF00500FBE7A6
:100E80006FF00500F8E700BF680100200000AD0B1F
:100E9000480100200060004038B5324BD86B1DF08F
:100EA000AAFE002857D02F4BD86B93F84010B3F808
:100EB000423043F4B0138568046913F4402F04D022
:100EC00013F0010F01D083F4402323F4801213F0B8
:100ED000010F0AD0012303FA01FC236843EA0C0343
:100EE00023602B68984740B138BD012303FA01FC09
:100EF000236823EA0C032360F3E71A4B586C1DF0B8
:100F00007AFE58B3174B586C93F84810B3F84A3030
:100F100043F4B0138568046913F4402F04D013F030
:100F2000010F01D083F4402323F4801213F0010F4A
:100F300009D0012303FA01FC236843EA0C03236070
:100F40002B689847D0E7012303FA01FC236823EAC2
:100F50000C032360F4E76FF01200C5E76FF0120096
:100F6000C2E700BF4801002038B5214B18691DF0C9
:100F700042FE002836D01E4B1869197DDB8A43F4E7
:100F8000B0138568046913F4402F04D013F0010FE7
:100F900001D083F4402323F4801213F0010F0CD00E
:100FA000012303FA01FC236843EA0C0323602B6846
:100FB0009847044648B1204638BD012303FA01FC96
:100FC000236823EA0C032360F1E70A4811F04AFC86
:100FD000074B186048B11DF00EFE0028EBD16FF0F2
:100FE0001204E8E76FF01204E5E76FF00504E2E7AA
:100FF00048010020800F030008B5154B1B6DD3F886
:10100000042522F00302C3F80425D3F8082522F0B2
:101010000302C3F80825D3F8102522F00F0242F08E
:101020000402C3F81025FFF737FF034608B118463E
:1010300008BDFFF7A9FE03460028F8D1FFF77EFEA2
:1010400003460028F3D1FFF78FFF0346EFE700BF09
:101050004801002008B5FFF7CFFF00B108BD0248E6
:10106000FFF732FDFAE700BF880F030008B51E4BFB
:101070000222BFF35B8F53E8001F012903D143E82D
:1010800000200028F7D1BFF35B8F2AD1174BD86B14
:1010900093F8401003691A6801238B401A4217D154
:1010A0000023BBB1012303FA01F18368DB68984791
:1010B000021E18BF01220C4BBFF35B8F53E8001FC9
:1010C00043E8002CBCF1000FF8D1BFF35B8F08BDE3
:1010D0000123E6E7012303FA01F183681B699847BE
:1010E000E6E76FF00F00F2E76C24002048010020D3
:1010F0002DE9F04105460F461646244B0222BFF368
:101100005B8F53E8001F012903D143E8002000282A
:10111000F7D1BFF35B8F35D11D4B1869197D03697A
:101120001B6801248C4023420CD1012363B10123AD
:1011300003FA01F18368DB689847044664B12046EE
:10114000BDE8F0810023F1E7012303FA01F1836890
:101150001B6998470446F1E70E4B1D60DFF83880A5
:10116000C8F800703346012229461046FFF7D0FC2C
:10117000D8F800100029E2D0334600220120FFF702
:10118000C7FCDCE76FF00F04D9E700BF6C24002038
:1011900048010020642400206824002008B5204A6B
:1011A00092F828C092F8293083F001031D480CF50D
:1011B000A27C50F82C1021F480111B0503F480133D
:1011C0000B4340F82C3092F820C092F8213083F085
:1011D00001030CF5A27C50F82C1021F480111B05A2
:1011E00003F480130B4340F82C301069117D036920
:1011F0001A6801238B401A4208D1002343B101230E
:1012000003FA01F18368DB68984708BD0123F5E71D
:10121000012303FA01F183681B699847F5E700BFD2
:10122000480100200060004010B586B004463A4BEB
:101230000222BFF35B8F53E8001F012903D143E86B
:1012400000200028F7D1BFF35B8F62D11F2C0FD98C
:101250006FF01500304B0122BFF35B8F53E8001F86
:1012600043E80024002CF9D1BFF35B8F06B010BD1A
:101270002A4B1869197D03691A6801238B401A42A9
:1012800036D10023002B35D0012303FA01F1836806
:10129000DB6898470028DDD1C0238DF81430A40006
:1012A00004F07C048DF8154005AB039302230493EE
:1012B00003AB01930123029318490A69097D14695C
:1012C00024688B401C4200D10120D0B1012303FAD5
:1012D00001F19368DB68104698470028BAD10F499E
:1012E00051F8040B83681C68002301AAA047B1E7EA
:1012F0000123C7E7012303FA01F183681B699847BB
:10130000C8E7012303FA01F193681B691046984767
:10131000E3E76FF00F00A9E76C24002048010020EC
:1013200010B5304B0222BFF35B8F53E8001F00293A
:1013300003D143E800200028F7D1BFF35B8F4ED1E3
:10134000294BD86B93F8401003691A6801238B402E
:101350001A421BD10123DBB1012303FA01F1836897
:10136000DB6898470446DCB1002C34D0B4FA84F32F
:101370005B091C4ABFF35B8F52E8001F42E8003054
:101380000028F9D1BFF35B8F204610BD0023E2E7B0
:10139000012303FA01F183681B6998470446E2E7D9
:1013A000114B1869197D03691A6801238B401A4291
:1013B00000D001243CB1012303FA01F18368DB680A
:1013C00098470446D0E7012303FA01F183681B69BB
:1013D00098470446C8E712201EF036F9C6E76FF0BA
:1013E0000F04D1E76C2400204801002010B52D4BDC
:1013F0000222BFF35B8F53E8004F43E8002100292E
:10140000F9D1BFF35B8F944248D078B1012829D03D
:101410006FF01500234BBFF35B8F53E8002F43E8B9
:1014200000410029F9D1BFF35B8F10BD1E4B586CF2
:1014300093F8481003691A6801238B401A4208D1B7
:10144000002343B1012303FA01F18368DB68984765
:10145000E0E70123F5E7012303FA01F183681B6943
:101460009847D7E7104B586C93F8481003691A68EF
:1014700001238B401A4208D1012343B1012303FA0F
:1014800001F18368DB689847C4E70023F5E701238F
:1014900003FA01F183681B699847BBE76FF00F00FF
:1014A000C3E700BF6C240020480100202DE9F04F65
:1014B0008BB0054692460593149EDDF854B0039117
:1014C00061B195F80280CDF80880B8F1000F08D01E
:1014D00016F0010F0ED14FF0000904E016F0D8FE0F
:1014E000EFE74FF00009EF783FB116F0020F2BD174
:1014F000002303E04FF00109F5E7002313B9B9F128
:10150000000F23D02C78A300019305EB8404BAF1DB
:10151000000F25D0019A2946504618F0E7F8019BA4
:1015200053440493B9F1000F40F09680029B1BB125
:1015300016F0040F40F09E804FF000088AF80280F9
:10154000DDF810900023B1E00123D7E7BAF1000FD6
:1015500004D0039A2946504618F0C8F8039878E05A
:10156000B9F1000F20D1029B002B3DD016F0040AE8
:101570002FD01C444FF0000A2BE00744013408F13F
:101580000108C8451ED2227800235BF822201946A4
:10159000184616F092FE002DEFD0B245EDD225F898
:1015A0001A000AF1010AE8E74FF00008C246DDF828
:1015B00008900197039F1496CDF854B0AB46169E41
:1015C000159DDEE70397019F149E15955D46DDF896
:1015D00054B006F0050301934FF00008DDF80C90BD
:1015E000CDF854B0AB4624E0DDF808A0F1E70023C5
:1015F0001D4613B116F0010F03D195B916F0020F75
:101600000FD000231946184616F057FE159B3BB124
:10161000169B9A4504D2159B23F81A000AF1010A79
:1016200081441DB1019B0BB909F1FF39013408F167
:101630000108B8450CD223785BF82320584B9A4216
:10164000D5D3584B9A4201D30023D1E70123CFE7EA
:1016500048460BB0BDE8F08FDDF808904A462146B9
:1016600006A818F043F800238AF802304C44DDF84D
:10167000109067E798461A462146DDF810904846D4
:1016800018F034F8C14444444FF000085AE70021F0
:1016900031B316F0010F18D008F101010AA88044F7
:1016A00008F8102C5FFA81F801340133BB4226D2CE
:1016B000227855F822103A488142E8D339488142CD
:1016C00001D30021E4E70121E2E716F0040FEBD09B
:1016D00009F8012B9AF8022001328AF80220E3E788
:1016E00016F0020F08D008F101010AA8804408F89A
:1016F000102C5FFA81F8D7E709F8012BD4E79AF8A4
:10170000013043448AF80130049BA9EB0303DBB2A8
:101710009AF802209B1A8AF80330029B019A13441C
:101720001F44039BDF1B3A462146484617F0DEFF65
:10173000B944B8F1000F09D0A9EB0A0A059BA3EB45
:101740000A0AD04525D200245E4611E0A9EB0A0022
:101750007FE7002309F8011B0AF1FF3A514648468A
:1017600016F0ABFD002817DBAAEB000A8144013418
:10177000A0450ADD0AAB234413F8101C55F82120BC
:10178000002EE6D036F81430E4E7059BA3EB0A0000
:101790005FE76FF01B005CE76FF01B0059E700BFCD
:1017A00048F8020090320300C0434FF0000C94450B
:1017B00019D230B511F80C3083EA000E0EF00F0E7E
:1017C0000A4C54F82E5085EA101080EA131303F0E7
:1017D0000F0354F8233083EA10100CF1010C9445E8
:1017E000E8D3C04330BDC043704700BFAC0F030017
:1017F00008B50B6801330B60014B1B68984708BDA7
:10180000A0010020014B1860704700BFA00100201C
:1018100000B583B002460B460021019101A903489F
:1018200000F052FA03B05DF804FB00BFF1170100AD
:1018300010B584B00446019002910021039101A9E2
:10184000054800F041FA039B029A934201DA002214
:10185000E254039804B010BDB58302002DE9F043B3
:1018600083B0044608461546238B13F0080F05D1B4
:1018700003F0070600230093019369E0012909D0D2
:1018800043F02003238385F31188BFF36F8F03B0E8
:10189000BDE8F08343F010032383F4E7204616F0FD
:1018A000E4FD57E0D4F814904A466946204616F005
:1018B000F5FD00275AE023691F680621204616F02F
:1018C000ADFD4FF0000951E023695F680421204617
:1018D00016F0A4FD4FF0000948E023699F68052138
:1018E000204616F09BFD4FF000093FE0002246E045
:1018F000002244E043F00803238385F31188BFF3FB
:101900006F8F002944D1009B2BB14B46424669465C
:10191000204616F03AFE17B125492046B8474FF049
:101920002003EFF3118583F31288BFF36F8F238BAE
:1019300023F008032383238B13F0100F2ED023F002
:10194000100323830120268B06F0070600289AD077
:101950000228A3D0002896D00128A3D00328AAD01B
:101960000428B1D00528B8D00027B946238B03F04E
:101970000708B045BAD0A268002AB9D001221146A2
:10198000002AB7D1009A002AB4D1002FB2D1D2E7F1
:101990004A464146204616F049FDB4E713F0200FB1
:1019A00004D023F0200323830220CCE70020CAE7E1
:1019B000B985020070B582B004460023036043601D
:1019C00083604B78252B02D04E1C01251FE0881C1C
:1019D000E37045E1237843F004032370B5B1013689
:1019E00014E0237843F008032370F7E7237843F0EB
:1019F00010032370F2E7237843F020032370EDE710
:101A0000237843F040032370E8E7002545B333789B
:101A1000203B102BF9D801A252F823F0ED19010058
:101A20000B1A01000B1A0100F71901000B1A010033
:101A30000B1A01000B1A01000B1A01000B1A01000E
:101A40000B1A01000B1A0100E31901000B1A010027
:101A5000D51901000B1A01000B1A0100011A01002F
:101A6000237803F04403442B5FD00196237843F09E
:101A70008003237033782A2B5CD001A817F02FF84D
:101A8000019B9E420FD0237843F080032370606057
:101A9000DBB2C3F34003002854DB00221343227857
:101AA00063F341022270019B01931B782E2B14BF1C
:101AB00000230123627863F341026270002B43D05C
:101AC000019B5A1C01925B782A2B3FD001A817F08A
:101AD00006F8A0602378C3F3400300283EDB002211
:101AE0001343227863F341022270019803784C3B40
:101AF0002E2B00F29D80DFE803F0909B9B9B9B9B2D
:101B00009B9B9B9B9B9B9B9B9B9B9B9B9B9B9B9B25
:101B10009B9B9B9B9B9B339B579B459B9B9B9B9B17
:101B20009B9B899B9B9B9B9B820023786FF38613D7
:101B300023709AE7637843F00103637033460133FF
:101B40000193B1E70122A9E70198CFE7637843F059
:101B500004036370104601300190C7E70122BFE71C
:101B6000421C4378682B06D06378022161F3C603D8
:101B7000637010461EE06378012262F3C60363704F
:101B8000023017E0421C43786C2B06D063780321A7
:101B900061F3C603637010460CE06378042262F3BD
:101BA000C6036370023005E06378052262F3C60362
:101BB0006370013010F8013BE370A3F14102372A52
:101BC0007DD8DFE802F05E7C7C7C5E5E5E7C7C7CA7
:101BD0007C7C7C7C7C7C7C7C7C7C7C7C7C4F7C7C72
:101BE0007C7C7C7C7C7C5E7C4F3A5E5E5E7C3A7C5E
:101BF0007C7C7C654F717C7C717C4F7C7C4F6378F6
:101C0000062262F3C60363700130D3E763780722CC
:101C100062F3C60363700130CCE76378082262F395
:101C2000C60363700130237843F002032370C1E7D9
:101C300063786FF3C6036370BCE7A278012161F398
:101C40000202A270627802F07802402A10D0632B60
:101C500013D02378C3F34002154365F34103237087
:101C600002B070BDA278022161F30202A270E9E71E
:101C7000217841F001012170E9E7151E18BF012507
:101C8000E7E7A378042262F30203A3700125E0E7EB
:101C9000A378032262F30203A370637803F078034E
:101CA000402BD6D10125D4E7A378032262F30203A7
:101CB000A370637813F0780FCBD00125C9E72378A0
:101CC00043F001032370C4E72DE9F04F91B00646BD
:101CD0000D4691460393002499F80000002800F077
:101CE000D582252808D009F101092946B0470028E6
:101CF000C0F2CD820134EFE70023049305930693ED
:101D0000079308930993494606A8FFF753FE0290EC
:101D10009DF8193013F0010F00F09780039B1A1DF6
:101D200003921F68002FC0F288809DF8193013F0CD
:101D3000040F00F09C80039B1A1D0392D3F800A0AF
:101D4000BAF1000FC0F28A800023079308939DF830
:101D50001A3003F007039DF81910C1F3C301012BDA
:101D600000F08E80022B00F0D380042B00F0248141
:101D7000032B00F03B819DF8188018F0030B40F016
:101D80003B819DF81B30253B532B00F2E681DFE8B9
:101D900013F04001E401E401E401E401E401E401A1
:101DA000E401E401E401E401E401E401E401E4010B
:101DB000E401E401E401E401E401E401E401E401FB
:101DC000E401E401E401E401E401E401E401E401EB
:101DD000E401E401E401E401E401E401E401E401DB
:101DE000E401E401E401E401E401E401E401E401CB
:101DF000E401E401E401E4018101E401E401E4011E
:101E0000E401E401E401E401E401E401E4015E0130
:101E10006701E401E401E401E4016701E401E40194
:101E2000E401E401BE018101A201E401E4014D01EC
:101E3000E4018101E401E40181019DF8183043F0DF
:101E400004038DF818307F426FE79DF91830002B9E
:101E500002DB4FF0FF3768E7079F66E79DF8193010
:101E60006FF341038DF819304FF0FF3A6CE713F030
:101E7000020F02D0DDF820A066E74FF0FF3A63E7DB
:101E8000CB1E042B04D8DFE803F00B1D29353500E9
:101E9000039B1A1D03921B68DA170493059206E050
:101EA000039B1A1D03921B68DA17049305920129FC
:101EB00028D002297FF45FAFBDF91030DA17049300
:101EC000059258E7039B073323F0070303F1080249
:101ED0000392D3E90023CDE90423E8E7039B07330A
:101EE00023F0070303F108020392D3E90023CDE9AD
:101EF0000423DCE7039B1A1D03921B68DA17049383
:101F00000592D4E79DF8103004930023059332E73F
:101F1000CB1E042B04D8DFE803F00B1F3541410032
:101F2000039B1A1D03921B680493002305931EE074
:101F30009DF81B30632B07D0039B1A1D03921B686F
:101F400004930023059312E0039B1A1D03921B6860
:101F50000493002305930AE0039B073323F0070350
:101F600003F108020392D3E90023CDE904230129F8
:101F70001CD002297FF4FFAEBDF81030049300237B
:101F80000593F8E6039B073323F0070303F10802E8
:101F90000392D3E90023CDE90423E8E7039B1A1D4C
:101FA00003921B68049300230593E0E79DF810302B
:101FB000049300230593DEE608290BD0039B073327
:101FC00023F0070303F108020392D3E90023CDE9CC
:101FD0000423D0E6039B073323F0070303F1080231
:101FE0000392D3E90023CDE90423C4E6039B1A1D21
:101FF00003921B680493BEE6029F3B464A4629466D
:10200000304616F0E8FD0028C0F241810444B9468C
:1020100062E629462520B0470028C0F23881013405
:10202000D8460DF13E0A4FF000099BE0DDF8109014
:10203000BAF1000F07DB5146484617F01DFB09EBCC
:10204000000AD8468EE0484617F00DFBF7E7049BE0
:102050008DF82830D8460DF1290A0DF1280981E0C4
:1020600018F0080F05D118F0100804D04FF0200820
:1020700001E04FF02B08049A059B002B02DB049231
:10208000059308E0524263EB4303049205934FF03B
:102090002D0800E0D8460DF13E0300930AAB06AAD6
:1020A000DDE9040116F02DFD8146BAF1000FC0F202
:1020B00088800DF13E03A3EB09039DF818206FF310
:1020C00086128DF818209A457ED9AAEB0303079350
:1020D0000DF13E0A46E0049828B9D846DFF8B4A1CD
:1020E000AAF105093EE00DF13E0300930AAB06AAF2
:1020F000002116F006FD81469DF81A3043F01003CA
:102100008DF81A3078238DF81B30D846CDE7049A25
:102110009DF81930C3F3C303072B06D8DFE803F09B
:10212000040B0D0F1115191B1460D8460DF13E0A52
:102130004FF0000916E01470F7E71480F5E714601B
:10214000F3E7E31714605360EFE7E317146053609D
:10215000EBE71460E9E71460E7E7D8460DF13E0AC3
:102160004FF00009B9F1000F00F08D80AAEB0903D0
:10217000B8F1000F00D001339DF81A2012F0100FB3
:1021800025D0023307990B4412F0400F01D0089A72
:102190001344002F31DDFF1A9DF8183013F0040F9F
:1021A0002BD113F0400F17D0B8F1000F17D02946EC
:1021B0004046B04700286ADB0134D8464FF0300B68
:1021C0000FE00DF13E0ACDE70DF13E0ACAE712F02D
:1021D000080FD7D00133D5E74FF0200B01E04FF0C7
:1021E000300B3B465F1E002B07DD29465846B047A3
:1021F00000284CDB01343B46F4E7B8F1000F05D072
:1022000029464046B047002841DB01349DF81A308A
:10221000C3F30012C3F3C003134305D02946302093
:10222000B047002833DB01349DF81A3013F0100F4B
:1022300006D029469DF81B00B047002827DB013453
:10224000079B03F1FF38002B07DD29463020B047FC
:1022500000281CDB01344346F3E753464A4629462F
:10226000304616F0B8FC002811DB0444002F07DDCF
:1022700029462020B047002809DB0134013FF5E75B
:10228000DDF8089028E5DDF8089025E5204611B036
:10229000BDE8F08FF10F030008B54FF02002EFF317
:1022A000118382F31288BFF36F8F02F0C9FC0348D9
:1022B00016F098F801F012F9FCE700BFF40F0300E4
:1022C00008B5064B186018B1054B1B68092B00DCDC
:1022D00008BD044811F06CF8FAE700BFBC240020E8
:1022E000702400209007002008B5024811F060F823
:1022F00008BD00BF9007002030B589B000220F490B
:102300000F481DF0D3F90F4D00220023CDE906231D
:10231000002404940E2303930294019400940A4B26
:102320004FF44072094928461CF062FD08492846CE
:1023300010F090FD204609B030BD00BFE922010039
:10234000600C0020980C0020F9260100805A002023
:1023500020100300014B53F8200070472C1003009D
:10236000184BBFF35B8F53E8002F511C43E800105C
:102370000028F8D1BFF35B8F1ABB70B5002409E0C9
:10238000114B03EB06135B6804221968284600F022
:10239000D9F901340D4B0C4A9B1AB4EB231F0FDA09
:1023A0002646094D05EB04152B7B002BF1D02301AC
:1023B000054AD3589B69002BE2D028469847DFE7AF
:1023C00070BD70477824002098FC0200A8FC020031
:1023D00038B108B5044A1060084600F09FFB0020A1
:1023E00008BD6FF015007047A401002008B5054B2B
:1023F0001B781BB1034B01221A7008BD024810F074
:10240000D7FFF7E7595A0020900700200D4BBFF384
:102410005B8F53E8002F013243E800210029F8D1F7
:10242000BFF35B8F00B97047074BBFF35B8F53E877
:10243000002F013A43E800210029F8D1BFF35B8F58
:10244000F1E700BF7424002070240020064B002018
:102450000246BFF35B8F53E8000F43E800210029D9
:10246000F9D1BFF35B8F70477424002038B5FFF7B4
:10247000EDFF0546002400E001340B4B0B4A9B1A8C
:10248000B4EB231F0FDA094800EB041043685B79B3
:10249000002BF1D02301054AD3581B69002BEBD048
:1024A00029469847E8E738BDA8FC020098FC0200DE
:1024B000034B18680028D4BF00200120704700BFDC
:1024C0007424002008B50249024816F05EFC08BDDD
:1024D000381003007C24002008B50023054A13703F
:1024E000054A13604FF400410448FFF771FFFFF7FE
:1024F000E9FF08BD5A5A00207424002069910200A7
:1025000008B5014600220023014816F065FC08BD0D
:102510007C24002008B5024816F056FD08BD00BF17
:102520007C24002008B50146014816F0BEFD08BD18
:102530007C240020F8B50646E9B9002400E0013407
:102540000F4B104A9B1AB4EB231F14DA0D4D05EB09
:1025500004156B685B79002BF1D03146284616F0E4
:1025600001FE0028EBD02701064BDB591B683146E2
:1025700028469847E3E73046FFF7D4FFF8BD00BF91
:10258000A8FC020098FC020008B5024816F0CAFD3B
:1025900008BD00BF7C24002010B50446114B1B78F9
:1025A00003B9D0B116F0E9FD034680B15CB90E4A1B
:1025B000BFF35B8F52E8001F013942E8001000288A
:1025C000F8D1BFF35B8F21461846FFF7B3FF14B96C
:1025D000FFF76EFF10B916F0D4FD10BDFFF746FFF0
:1025E000F9E700BF595A00207024002010B582B0CE
:1025F0001D4BBFF35B8F53E8002F511C43E80010C5
:102600000028F8D1BFF35B8F184B1B783BB9184BF0
:102610001B6803B19AB10A2A1CD002B010BD4FF05A
:102620002003EFF3118483F31288BFF36F8F002030
:10263000FFF7B2FF84F31188BFF36F8FEDE700223D
:102640000023CDE900234FF400420023094811F094
:1026500061FEE2E7002BE0D006481DF033F80648A3
:1026600010F0A6FED9E700BF702400205A5A0020BF
:10267000BC240020600C00209007002010B5044608
:10268000054B1B689847A0602146044816F03BFCA8
:10269000FFF7ACFF10BD00BFA40100207C24002088
:1026A000124B1B7803B1704710B5FFF759FE002499
:1026B00000E001340E4B0F4A9B1AB4EB231F0CDAD7
:1026C0000C4800EB041043685B79002BF1D0230128
:1026D000084AD3585B699847EBE70020FFF75CFF97
:1026E0000028FAD1014B01221A7010BD5A5A00205D
:1026F000A8FC020098FC020008B5FFF731FE11F0BB
:102700000BFCFFF7DDFD0020FFF746FF0028FAD1A4
:102710004FF0FF324FF0FF33014810F071FEF2E747
:1027200090070020054B064A9B1AB1EBD30F02D24B
:1027300052F8310070470020704700BF98FC02003B
:1027400040FB020008B5074BC31A1B110133426856
:10275000137143681960436801225A71FFF746FEFE
:1027600008BD00BF98FC02000EB400B582B001465F
:1027700003AB53F8042B01930348FFF7A5FA02B00B
:102780005DF804EB03B070472992020030B585B0C4
:1027900011F0440F05D01A4B1C6834B9002005B065
:1027A00030BD1849FFF7E0FFF9E7174B1968B2FB96
:1027B000F1F1B1FBF4FC154AA2FB0C32D20A4FF442
:1027C000616E0EFB12CE124BA3FB0E535B0904FB92
:1027D0001C114FF47A7C0CFB01F1B1FBF4F505FB05
:1027E00014110CFB01F1B1FBF4F102910195C3EB63
:1027F0000311AEEB810100910649FFF7B5FFCEE76B
:10280000C02400204C100300C4240020C5B3A291B2
:10281000898888885810030061B108B52AB1064A32
:1028200052F8232012B9054A00E0044A0449FFF790
:102830009BFF08BD704700BFD01003007410030059
:102840007C10030011F0100F0BD108B511F0200F10
:1028500003D00449FFF788FF08BD0349FFF784FF51
:10286000FAE77047D4FE02006C3103002DE9F04115
:1028700005460F46164698460699FFF7E3FF0024E3
:10288000444505DA23492846FFF76EFF0134F7E790
:10289000002409E01F492846FFF766FF0BE01E49A8
:1028A0002846FFF761FF01340F2C0CDC002C02DD01
:1028B00014F0070FEED0B442F1D23A5D1749284622
:1028C000FFF752FFEFE716492846FFF74DFF0024B8
:1028D00009E010492846FFF747FF0BE01149284659
:1028E000FFF742FF01340F2C12DC002C02DD14F044
:1028F000070FEED0B44206D23A5DA2F120035E2B60
:10290000ECD92E22EAE703492846FFF72DFFE9E735
:10291000BDE8F081A41003008810030080100300BC
:102920008C100300901003002DE9F04180461646FC
:102930001D46BDF9187059B90024002F1CDB86B163
:102940000123079A934013F0100F18D10D4E09E0A0
:102950000D4B079A53F822200C49FFF705FF044658
:10296000EBE7084E39462846FFF7DCFE02463146C3
:102970004046FFF7F9FE04442046BDE8F081044ECE
:10298000F0E700BF941003000C110300A010030037
:102990009C1003002DE9F04F85B005460C46164605
:1029A00003939DF8388001F0020B01F0010AC1F396
:1029B000C00916F0EAFBE8B1024613492846FFF7C2
:1029C000D3FE0746BBF1000F16D1424651462846BA
:1029D00016F0EAFBCDF80480BDF9403000939DF875
:1029E0003C30324649462846FFF79EFF384405B042
:1029F000BDE8F08F0027E5E7039A21462846FFF758
:102A0000C5FE0744E1E700BFA81003002DE9F0432D
:102A100085B006460C4617468B680A88C2F38218B2
:102A200012F4E07F35D04A680978C1F3C2016AB375
:102A30002048121A42F3CF0202920191CDF8008091
:102A4000002239463046FFF7A5FF8146254655F856
:102A5000103BC3F3492343B1B8F1000F1CD1164812
:102A60002B463246154915F03CFC6288C2F3CB0276
:102A70002168C1F34921294482B9B8F1000F13D16B
:102A8000304616F0C4FB05B0BDE8F0834FF0FF32CE
:102A9000D2E74FF00009D9E70948E1E700974B4634
:102AA000304616F099FBE8E742463946304616F0C4
:102AB00087FBE5E740FB020061920200C91C0100B0
:102AC0002992020070B582B00446056842F20F7385
:102AD0008B4228BF0B460E4A0521684615F090FC34
:102AE000064663685B680B220A49284616F04FFBCE
:102AF00063685B6832466946284616F048FB63689F
:102B00005B681B220449284616F041FB02B070BDE9
:102B1000AC10030000110300E4100300074B012276
:102B20001A6004E04008054A13685B001360044B18
:102B30009842F7D8034B1860704700BFC4240020A8
:102B400040420F00C024002070B506460D46002408
:102B500006E0054B1868315D8368DB6998470134EE
:102B6000AC42F6D3284670BDE0240020014B19602A
:102B700000207047D0240020014B024A1A607047A1
:102B8000E024002060F9020008B5034B01221A700E
:102B9000024816F03CFB08BD5B5A002060110300A0
:102BA00008B50248FFF78EFF08BD00BF60110300A3
:102BB00010B50C46044B1868FFF7CCFB03460F22F8
:102BC00021460248984710BDD02400206011030020
:102BD0000F4B1B68B3B130B4002300E001330D4A42
:102BE0001268934208DA1A01094C246804EB0315B1
:102BF000A25C9042F2D100E0002535B10D600020CA
:102C000030BC70476FF00C0070476FF00100F7E7C1
:102C1000AC010020B4120300F8B500AF46690369A7
:102C20001E448368002B00F006810446C068836858
:102C3000DB6898470268A568B5FBF2F302FB135501
:102C40005DB1551BE0688368DB689847A3682A4636
:102C500001792068184416F078FDA3682B44E068D9
:102C6000226881684D683146A847054618B9E3696E
:102C7000002B48D15AE06C4688B06B4613F1100225
:102C800036D010211AB1042901DD6D48586112B106
:102C9000082900DD9D6112B10C2900DDDE610F29DC
:102CA00029DD102052B10021042666F307016FF3DD
:102CB0000F216FF317416FF31F61196100216FF34B
:102CC00000016FF341016FF382016FF3C50101232E
:102CD00063F3881100F47D7363F352216FF3DE41D7
:102CE0006FF3DF710023574816F0E1FAA546A3E021
:102CF0006FF00041C6E76FF01B00D3E72068435D2B
:102D0000DB4343550135A368AB42F7D8E06822683E
:102D100081680D683146A847054670B9E3693246B7
:102D2000A168206898470546002845D1A268236914
:102D3000134423610023A3607EE06C4688B06B4699
:102D400013F1100232D00C211AB1042901DD3E48E2
:102D5000586112B1082900DD9D610B2929DD0C2085
:102D600052B10021032666F307016FF30F216FF3C1
:102D700017416FF31F61196100216FF300016FF3B9
:102D800041016FF382016FF3C501012363F38811E1
:102D900000F47B7363F352216FF3DE416FF3DF7155
:102DA0000023284816F083FAA54645E06FF000415D
:102DB000CAE76FF01B00D3E76C4688B06B4613F18F
:102DC000100232D00C211AB1042901DD1F485861CC
:102DD00012B1082900DD9D610B2929DD0C2052B1BB
:102DE0000021032666F307016FF30F216FF31741EC
:102DF0006FF31F61196100216FF300016FF341014F
:102E00006FF382016FF3C501012363F3881100F4AE
:102E10007B7363F352216FF3DE416FF3DF710023A5
:102E2000084816F044FAA54606E06FF00041CAE7EC
:102E30006FF01B00D3E700252846BD46F8BD00BF54
:102E40007011030048FB020094110300AC11030051
:102E500010B586B00C460B684268934205D84B68A3
:102E600013444B60012006B010BD144B05930023A2
:102E7000022262F307036FF30F236FF317436FF31D
:102E80001F63049300216FF300016FF341016FF39F
:102E900082016FF3C501012363F38811082363F3F3
:102EA00052216FF3DE416FF3DF71002304AA04485F
:102EB00016F0FDF900206060D5E700BFC0110300E7
:102EC00048FB02002DE9F0438FB0169FDDF85C80CF
:102ED000002800F095800C4691461E4605460029C4
:102EE00000F09180002A00F091800093002301936C
:102EF0008B68DB68084698470268B6FBF2F302FB72
:102F00001363002B2CD16A46434920461AF0B5FDC5
:102F1000019B002B7DD007EB0802934248D3A368A6
:102F2000DB68204698470268B7FBF2F302FB137395
:102F3000002B3DD1EC60C5F800906E6000232B6142
:102F4000AB606F61B8F1000F02D1019BA3EB0708E2
:102F5000C5F81880189BEB6100200FB0BDE8F08326
:102F60002E4B0D930023022262F307036FF30F230E
:102F70006FF317436FF31F630C9300216FF300018E
:102F80006FF341016FF382016FF3C501012363F316
:102F90008811082363F352216FF3DE416FF3DF7171
:102FA00000230CAA1E4816F082F96FF00D00D4E73A
:102FB0001C4B07930023022262F307036FF30F23D6
:102FC0006FF317436FF31F63069300216FF3000144
:102FD0006FF341016FF382016FF3C501012363F3C6
:102FE0008811082363F352216FF3DE416FF3DF7121
:102FF000002306AA0A4816F05AF96FF00D00ACE754
:103000006FF00D00A9E76FF00D00A6E76FF00D005F
:10301000A3E76FF00D00A0E7512E0100E0110300BF
:1030200048FB02001812030070B52A4B1D7D05F005
:103030001F0301229A406909274B03EB8103D04308
:10304000BFF35B8F53E8001F01EA000443E800462A
:10305000002EF7D1BFF35B8F0A4200D170BD1F482D
:1030600005EB45029300C1181D4A72B14978C05C56
:1030700016F0A5FB4FF02003EFF3118683F31288BF
:10308000BFF36F8F174B1C6810E0002383F3118888
:10309000BFF36F8FEEE70F4B1B7D03EB43039900EC
:1030A0000E4B585C90470CB1246824B11CB1A26847
:1030B000002AF0D1F7E786F31188BFF36F8F074836
:1030C00005EB4505AA008118002383504B608B60F7
:1030D000C4E700BF484F002000250020F024002056
:1030E000BF970200E824002070B50446574B1D7DB1
:1030F0006A09BFF35B8F564B53F82230BFF35B8FE7
:1031000005F01F02134113F0010F15D005EB450325
:10311000504A12F82330F3B1B4F1FF3F31D110F02F
:103120009BFB4FF02003EFF3118683F31288BFF36C
:103130006F8F494B1C6845E00146284600F0A4F813
:103140000028E3D005EB4503424A02EB830307C89E
:1031500083E80700DAE705F01F02012393406D09B9
:103160003B4A02EB8505DB43BFF35B8F55E8002F3D
:103170001A4045E800210029F8D1BFF35B8F0020F9
:1031800062E005EB4503334A02EB83039868410C88
:10319000C003324BC018324A4FF0000341F1000126
:1031A000FAF71EF80121201A1CF01BFAB7E7274B8B
:1031B0001B7D03EB4303274911F8230090470CB113
:1031C000246824B11CB16268002AF0D1F7E786F3C5
:1031D0001188BFF36F8F05F01F03012199406B0920
:1031E000204A02EB8303BFF35B8F53E8002F0A43AF
:1031F00043E800200028F8D1BFF35B8F1A4B4BB196
:10320000144B05EB450203EB8201497813F82200C9
:1032100016F0C9FAFFF708FF05F01F03012404FAAE
:1032200003F36D090A4A02EB8505DB43BFF35B8FAD
:1032300055E8002F1A4045E800210029F8D1BFF3D6
:103240005B8F10F02BFD204670BD00BF484F002063
:10325000FC240020F0240020E82400203F420F003E
:1032600040420F0000250020A7970200BFF35B8FAC
:10327000044B53F82000BFF35B8F003818BF0120C8
:10328000704700BF042500202DE9F04182B00E46B2
:1032900001A900F043F8441E24B207E0B6F1FF3F55
:1032A00032D04044B0422FD9013C24B2002C2ADB5A
:1032B000019B04EB440203EB820513F82200FFF7A5
:1032C000D5FF0028F0D16868410CC003104FC01929
:1032D000104A4FF0000341F10001F9F781FF8046E9
:1032E000AB68590CDB03D8190A4A4FF0000341F1CF
:1032F0000001F9F775FF084B1B68B3F1FF3FCDD014
:103300008342CBD8D0E70025284602B0BDE8F08143
:103310003F420F0040420F00A801002008B9024BB5
:103320000B600020704700BF4012030008B5024840
:1033300011F0C4FB08BD00BFB8120300D0B108B53E
:103340004268042A05D0D2B100680FF0B3FF002014
:1033500008BD03680022BFF35B8F53E8001F0129FB
:1033600003D143E800200028F7D1BFF35B8F04D1DD
:103370001046EDE76FF4E04070470248E8E7024886
:10338000E6E700BFE98FFFFFEA8FFFFF20B308B534
:103390004268042A02D092B911480FE00368012262
:1033A000BFF35B8F53E8001F002903D143E80020DF
:1033B0000028F7D1BFF35B8F0CD1002008BD006857
:1033C0004FF0FF324FF0FF330FF0EAFE0028F5D048
:1033D0000448F3E70348F1E76FF4E040704700BFAB
:1033E000EA8FFFFFE98FFFFF10B5044688B16368DD
:1033F000042B0DD0082B0BD053B113F0020F0DD0BE
:10340000214609481BF09FFC0023236000236360D2
:1034100010BD064B5B6806489847E8E71422002178
:10342000206816F092F9F1E72025002078060020A8
:10343000C012030010B5044678B16368042B0BD0AA
:10344000082B09D00BB9236863B120681BF00EFD6F
:10345000636843F00103636010BD0F4B5B680F4866
:103460009847EAE74FF0FF324FF0FF3321460C4810
:103470000FF098FC08B923681BB9074B5B68094833
:10348000984714220021206816F05FF9636843F022
:1034900002036360D9E700BF78060020C012030072
:1034A00020250020E812030008B540231422044917
:1034B00004481BF03AFC0449044811F0B3FB08BD72
:1034C0003C250020202500202813030018130300AA
:1034D000014910220A60704710ED00E072B64040CA
:1034E00080F31188BFF36F8FBFF34F8F30BF62B689
:1034F000BFF36F8F704700BF72B6494081F31188E8
:1035000020BF80F3118862B6704700BFF8B500AFE6
:103510000446D0F800C0466880686D468AB06B46A5
:1035200013F1100200F0FC8014212AB1042903DDFC
:10353000DFF81CE2C3F814E01AB1082901DDC3F872
:1035400018C012B10C2900DDDE6112B1102900DDB6
:103550001862132940F3E78014205AB100214FF07C
:10356000050C6CF307016FF30F216FF317416FF335
:103570001F61196100216FF300016FF341016FF3C7
:1035800082016FF3C501012363F3881100F47D7399
:1035900063F352216FF3DE416FF3DF7100236D4857
:1035A00015F085FEAD46D4F80CC0266960696D46FD
:1035B0008AB06B4613F1100200F0B88014212AB1D2
:1035C000042903DDDFF890E1C3F814E01AB10829FB
:1035D00001DDC3F818C012B10C2900DDDE6112B1A3
:1035E000102900DD1862132940F3A38014205AB17A
:1035F00000214FF0050C6CF307016FF30F216FF3FF
:1036000017416FF31F61196100216FF300016FF320
:1036100041016FF382016FF3C501012363F3881148
:1036200000F47D7363F352216FF3DE416FF3DF71BA
:103630000023484815F03BFEAD46E0696D4688B072
:103640006B4613F1100277D00C211AB1042901DD69
:10365000424E5E6112B1082900DD98610B296EDDD2
:103660000C205AB100214FF0030C6CF307016FF3EB
:103670000F216FF317416FF31F61196100216FF381
:1036800000016FF341016FF382016FF3C501012364
:1036900063F3881100F47B7363F352216FF3DE410F
:1036A0006FF3DF7100232B4815F001FEAD46A069D2
:1036B00088B06B4613F1100244D00C211AB10429D2
:1036C00001DD274C5C6112B1082900DD98610B29EE
:1036D0003BDD0C2052B10021032464F307016FF39A
:1036E0000F216FF317416FF31F61196100216FF311
:1036F00000016FF341016FF382016FF3C5010123F4
:1037000063F3881100F47B7363F352216FF3DE419E
:103710006FF3DF7100230F4815F0C9FDBD46F8BDFA
:103720006FF0004101E76FF01B0016E76FF00041FA
:1037300045E76FF01B005AE76FF0004185E76FF037
:103740001B008EE76FF00041B8E76FF01B00C1E788
:103750003C13030070FC02006C1303009C13030075
:10376000AC13030040B2002807DB00F01F02400941
:1037700001239340014A42F82030704700E100E005
:1037800040B200280CDB00F01F02400901239340E7
:103790002030044A42F82030BFF34F8FBFF36F8FC1
:1037A000704700BF00E100E04209054B53F82220BA
:1037B00000F01F00012303FA00F01040704700BF23
:1037C00000E100E0013140B2002808DB4901C9B244
:1037D00000F1604000F5614080F80013704700F090
:1037E0000F004901C9B2014B1954704714ED00E0B4
:1037F00008B572B6054B9B690BB962B608BD034BA1
:1038000000229A611BF016FBF7E700BF484F00202B
:1038100030BFFFF7FDBF00BF08B50B4B0B4A22F0CE
:103820007F029A60BFF34F8FBFF36F8FD3F888206A
:1038300022F47002C3F888200FF0ECF910F0AEFB10
:1038400000F0E2FF0FF044FA00ED00E000C20000DB
:103850000A4A9368C3F8B80009490968C3F8BC105C
:1038600008494B6843F080534B60002383F3118871
:10387000BFF36F8F9368D3F8BC007047484F0020A8
:10388000E02F030000ED00E013498A684FF030009C
:103890001044EFF3098C80E8F01F202080F3128899
:1038A000BFF36F8F0D4F4FF00066CA698A603E60AC
:1038B000D2F8B8000023C2F8B83080F3118804B5FC
:1038C000104601F04BF8BDE8044002F1300090E8EA
:1038D000F01F8CF309887047484F002004ED00E08A
:1038E0001EF0040F0CBFEFF30880EFF3098081692D
:1038F00011F8021C0229FFD001B515F01FFE01BD11
:1039000010B4A2F120040E4942F8081C21F0010174
:1039100042F8081C42F8203C019B42F81C3C029BE8
:1039200042F8183C039B42F8143C4FF0807342F875
:10393000043C04650023C0F8B83010BC704700BFD9
:10394000C7860200124B9A6802B310F1160F11D00D
:10395000D2F8A830A3F1200C844505D8834205D9BC
:103960008B4205D800210BE0002109E0002107E08F
:10397000012105E0D2F8A8308B4294BF002101213B
:1039800009B900207047D2F8A8007047002070479E
:10399000484F002008B50D461446084B986000F0CB
:1039A000DDFF204685F30988002163B681F3118885
:1039B000BFF36F8F0022002314F085FE484F0020D4
:1039C00001B572B60B4A906900281EBF00219161B3
:1039D0001BF030FA62B6EFF30580A0F110004FEA59
:1039E000C0000549014409C99847BDE801400349A1
:1039F00008470000484F0020C0F90200013A0100CA
:103A0000044B9968D869884203D003494FF080522B
:103A10000A607047484F002004ED00E02DE9F041B6
:103A2000AAB000AF05460E461446CA4B7B61002380
:103A3000022262F307036FF30F236FF317436FF351
:103A40001F633B6100216FF300016FF341016FF3CE
:103A500082016FF3C501012363F38811082363F327
:103A600052216FF3DE416FF3DF71002307F1100283
:103A7000B94815F01CFCB94B9B6A13F4805F2AD13E
:103A8000B64B9B6A13F4006F4CD1B44B9B6A13F492
:103A9000007F6ED1B14B9B6A13F4806F40F0E080E1
:103AA000AE4B9B6A13F4807F40F00181AB4B9B6A65
:103AB00013F4005F40F02481A84A936A43F47F43E3
:103AC00093620121284615F04BFD20700020A83795
:103AD000BD46BDE8F081A24BFB620023022262F3E7
:103AE00007036FF30F236FF317436FF31F63BB627B
:103AF00000216FF300016FF341016FF382016FF357
:103B0000C501012363F38811082363F352216FF386
:103B1000DE416FF3DF71002307F128028E4815F0B4
:103B2000C6FBADE78F4B7B640023022262F30703E1
:103B30006FF30F236FF317436FF31F633B64002191
:103B40006FF300016FF341016FF382016FF3C50161
:103B5000012363F38811082363F352216FF3DE41DD
:103B60006FF3DF71002307F140027B4815F09FFBE4
:103B70008BE77D4BFB650023022262F307036FF3A3
:103B80000F236FF317436FF31F63BB6500216FF3C0
:103B900000016FF341016FF382016FF3C50101234F
:103BA00063F38811082363F352216FF3DE416FF34F
:103BB000DF71002307F15802674815F078FB674B67
:103BC000986B9B6A13F4004F3FF464AFE84688B0EB
:103BD0006B4613F110023DD00C212AB1042903DDFC
:103BE000DFF888C1C3F814C012B1082900DD98615C
:103BF0000B2932DD0C205AB100214FF0030C6CF37D
:103C000007016FF30F216FF317416FF31F61196104
:103C100000216FF300016FF341016FF382016FF335
:103C2000C501012363F3881100F47B7363F3522110
:103C30006FF3DE416FF3DF710023474815F037FB68
:103C4000C546002E3FF426AF444A936A23F400434E
:103C500093621FE76FF00041BFE76FF01B00CAE7F8
:103C6000434B7B670023022262F307036FF30F23AA
:103C70006FF317436FF31F633B6700216FF300017E
:103C80006FF341016FF382016FF3C501012363F309
:103C90008811082363F352216FF3DE416FF3DF7164
:103CA000002307F170022C4815F001FBF8E6314BB8
:103CB000C7F8A4300023022262F307036FF30F2337
:103CC0006FF317436FF31F63C7F8A03000216FF342
:103CD00000016FF341016FF382016FF3C50101230E
:103CE00063F38811082363F352216FF3DE416FF30E
:103CF000DF71002307F1A002174815F0D8FADBE6C0
:103D00001D4BC7F88C300023022262F307036FF3C8
:103D10000F236FF317436FF31F63C7F88830002139
:103D20006FF300016FF341016FF382016FF3C5017F
:103D3000012363F38811082363F352216FF3DE41FB
:103D40006FF3DF71002307F18802034815F0AFFA23
:103D5000B2E600BFDC13030070FC020000ED00E0DF
:103D6000F4130300081403001C14030038140300A8
:103D7000501403006C1403008414030000B5ABB0AE
:103D80009A4B05930023022262F307036FF30F237C
:103D90006FF317436FF31F63049300216FF3000168
:103DA0006FF341016FF382016FF3C501012363F3E8
:103DB0008811082363F352216FF3DE416FF3DF7143
:103DC000002304AA8A4815F072FA8A4B9B6A13F002
:103DD000007F26D1874B9B6A13F0807F47D1854BAC
:103DE0009B6A13F4002F68D1824B9B6A13F4802FD7
:103DF00040F089807F4B9B6A13F4003F40F0A9801C
:103E00007C4B9B6A13F4803F40F0C980794A936AE7
:103E10006FEA03436FEA1343936200202BB05DF80F
:103E200004FB754B0B930023022262F307036FF32D
:103E30000F236FF317436FF31F630A9300216FF390
:103E400000016FF341016FF382016FF3C50101239C
:103E500063F38811082363F352216FF3DE416FF39C
:103E6000DF7100230AAA624815F021FAB2E7634B1A
:103E700011930023022262F307036FF30F236FF302
:103E800017436FF31F63109300216FF300016FF36B
:103E900041016FF382016FF3C501012363F38811C0
:103EA000082363F352216FF3DE416FF3DF710023C8
:103EB00010AA4F4815F0FBF991E7514B17930023D7
:103EC000022262F307036FF30F236FF317436FF3BD
:103ED0001F63169300216FF300016FF341016FF32D
:103EE00082016FF3C501012363F38811082363F393
:103EF00052216FF3DE416FF3DF71002316AA3C48B5
:103F000015F0D5F970E73F4B1D930023022262F3B1
:103F100007036FF30F236FF317436FF31F631C93B4
:103F200000216FF300016FF341016FF382016FF322
:103F3000C501012363F38811082363F352216FF352
:103F4000DE416FF3DF7100231CAA294815F0AFF999
:103F500050E72D4B23930023022262F307036FF3F4
:103F60000F236FF317436FF31F63229300216FF347
:103F700000016FF341016FF382016FF3C50101236B
:103F800063F38811082363F352216FF3DE416FF36B
:103F9000DF71002322AA164815F089F930E71B4B80
:103FA00029930023022262F307036FF30F236FF3B9
:103FB00017436FF31F63289300216FF300016FF322
:103FC00041016FF382016FF3C501012363F388118F
:103FD000082363F352216FF3DE416FF3DF71002397
:103FE00028AA034815F063F910E700BFB4140300D2
:103FF00070FC020000ED00E0CC140300E0140300AC
:10400000FC1403001C150300441503006015030095
:1040100000B587B000230B70134A05921A4602219F
:1040200061F3070263F30F2263F3174263F31F6226
:104030000492194663F3000163F3410163F38201C3
:1040400063F3C501012262F38811082262F3522151
:1040500063F3DE4163F3DF7104AA044815F027F926
:1040600007B05DF804FB00BF8C15030070FC020074
:1040700090B583B000AF0F294FDC314C10390223CB
:104080003B718AB06B4613F1100248D04FF0110C0F
:1040900022B1BCF1040F01DD2A48586102203871B9
:1040A0001AB1BCF1080F00DD9C611AB1BCF10C0F14
:1040B00000DDD9611AB103F12001002090B3BCF1F9
:1040C000100F39DD11206AB100214FF0040C6CF3A0
:1040D00007016FF30F216FF317414FF0010C6CF3E1
:1040E0001F61196100216FF300016FF341016FF34C
:1040F00082016FF3C501012363F38811C0F3090343
:1041000063F352216FF3DE416FF3DF7100230E483A
:1041100015F0CDF80C37BD4690BD0C4CAEE76FF0F6
:10412000004CB5E707F1080404EB000E1EF804ECA0
:1041300001F801EB0130C1E76FF01B00C3E700BFDE
:10414000CC150300E415030070FC0200B015030059
:104150002DE9F043A5B000AF05460C461646C84B06
:104160007B610023022262F307036FF30F236FF3D7
:1041700017436FF31F633B6100216FF300016FF37F
:1041800041016FF382016FF3C501012363F38811CD
:10419000082363F352216FF3DE416FF3DF710023D5
:1041A00007F11002B74815F082F8B74B9B6A13F07D
:1041B000100F41D1B44B9B6A13F0080F63D1B24B7F
:1041C0009B6A13F0020F40F085806FF01508AE4B2C
:1041D0009B6A13F0010F40F0F680AB4B9B6A13F023
:1041E000200F40F01781A84B9B6A13F0100F04D1E9
:1041F000A54B9C6A14F0020405D0A34B5C6814F430
:10420000006440F03081A04B9B6A13F0200F04D073
:104210009D4A536A23F4005353629B4A936A43F0C6
:10422000FF0393620121284615F09AF93070204669
:104230009437BD46BDE8F083944BFB620023022215
:1042400062F307036FF30F236FF317436FF31F63DB
:10425000BB6200216FF300016FF341016FF3820134
:104260006FF3C501012363F38811082363F352211F
:104270006FF3DE416FF3DF71002307F128028148FD
:1042800015F015F896E7824B7B640023022262F357
:1042900007036FF30F236FF317436FF31F633B6441
:1042A00000216FF300016FF341016FF382016FF39F
:1042B000C501012363F38811082363F352216FF3CF
:1042C000DE416FF3DF71002307F140026D4814F007
:1042D000EEFF74E76F4BFB650023022262F30703D6
:1042E0006FF30F236FF317436FF31F63BB65002159
:1042F0006FF300016FF341016FF382016FF3C501AA
:10430000012363F38811082363F352216FF3DE4125
:104310006FF3DF71002307F158025A4814F0C7FF0A
:10432000594BD3F834809B6A13F0800F48D0E9468C
:1043300088B06B4613F110023CD00C211AB104294D
:1043400001DD554858611AB1082901DDC3F818800C
:104350000B2932DD0C205AB100214FF0030C6CF315
:1043600007016FF30F216FF317416FF31F6119619D
:1043700000216FF300016FF341016FF382016FF3CE
:10438000C501012363F3881100F47B7363F35221A9
:104390006FF3DE416FF3DF7100233A4814F087FFBB
:1043A000CD46002C3FF413AF374A936A23F08003C5
:1043B00093620CE76FF00041C0E76FF01B00CAE7A3
:1043C0006FF0150803E7354B7B670023022262F389
:1043D00007036FF30F236FF317436FF31F633B67FD
:1043E00000216FF300016FF341016FF382016FF35E
:1043F000C501012363F38811082363F352216FF38E
:10440000DE416FF3DF71002307F170021D4814F0E5
:104410004EFFE2E6224BC7F88C300023022262F303
:1044200007036FF30F236FF317436FF31F63C7F88F
:10443000883000216FF300016FF341016FF38201B7
:104440006FF3C501012363F38811082363F352213D
:104450006FF3DE416FF3DF71002307F18802094833
:1044600014F025FFBFE629464046FFF76BFA0446E5
:1044700000283FF4C8AE80F309880224C3E600BFD9
:10448000F815030070FC020000ED00E010160300B8
:1044900008140300441603005C160300741603009E
:1044A00084140300F0B599B000AF05460C468C4B60
:1044B0007B610023022262F307036FF30F236FF384
:1044C00017436FF31F633B6100216FF300016FF32C
:1044D00041016FF382016FF3C501012363F388117A
:1044E000082363F352216FF3DE416FF3DF71002382
:1044F00007F110027B4814F0DAFE002323707A4B98
:10450000DE6A16F002060BD1774BDB6A002B2FDB3D
:10451000754BD86A10F0804052D16437BD46F0BD6B
:10452000724BFB650023022262F307036FF30F2334
:104530006FF317436FF31F63BB6500216FF3000137
:104540006FF341016FF382016FF3C501012363F340
:104550008811082363F352216FF3DE416FF3DF719B
:10456000002307F158025F4814F0A1FE0020D4E7B1
:104570005F4B7B640023022262F307036FF30F2378
:104580006FF317436FF31F633B6400216FF3000168
:104590006FF341016FF382016FF3C501012363F3F0
:1045A0008811082363F352216FF3DE416FF3DF714B
:1045B000002307F140024B4814F079FE3046ACE787
:1045C0004C4BFB620023022262F307036FF30F23BD
:1045D0006FF317436FF31F63BB6200216FF300019A
:1045E0006FF341016FF382016FF3C501012363F3A0
:1045F0008811082363F352216FF3DE416FF3DF71FB
:10460000002307F12802374814F051FEAB6933F854
:10461000022C4DF602739A4210D0334B93F8283097
:10462000002B4CD1304B93F82930002B4DD12E4B21
:104630005B8D9BB2002B4ED130466EE728686C46EE
:1046400088B06B4613F1100233D00C211AB1042943
:1046500001DD294E5E6112B1082900DD98610B2948
:104660002ADD0C2052B10021032666F307016FF307
:104670000F216FF317416FF31F61196100216FF371
:1046800000016FF341016FF382016FF3C501012354
:1046900063F3881100F47B7363F352216FF3DE41FF
:1046A0006FF3DF7100230F4814F001FEA546286860
:1046B00033E76FF00041C9E76FF01B00D2E72246F5
:1046C00001212846FFF744FD27E72246012128461D
:1046D000FFF7A4F921E72846FFF750FB1DE700BFCD
:1046E0009416030070FC020000ED00E0AC1603001D
:1046F000D0160300E01603000017030070B590B059
:10470000354B5D68C5F30805002383F31188BFF3BB
:104710006F8F02F07F43B3F17F4F3FD102F00C0364
:10472000082B10D012F0080F35D00C4600260DF1E2
:1047300027022946204614F015FF05469DF827302C
:104740007BB310B070BD254B0F930023022262F3A0
:1047500007036FF30F236FF317436FF31F630E937A
:1047600000216FF300016FF341016FF382016FF3DA
:10477000C501012363F38811082363F352216FF30A
:10478000DE416FF3DF7100230EAA154814F08FFD90
:1047900000263446CBE704460126C8E70026344607
:1047A000C5E72022214601A814F0A0FF4EB1089BC6
:1047B000C3F308025AB96FEA53236FEA43230893FD
:1047C00005E0089B23F4FF7323F00103089301A97C
:1047D000284614F0A7FEB4E700ED00E01C17030024
:1047E00070FC0200024A536943F0100353617047A2
:1047F00000ED00E0EFF30880EFF3098101B57246A8
:10480000FFF77CFF01BD00BF002206E002F00F01B0
:10481000094B0B442021197601322F2A0ADC53B2AE
:10482000002BF3DB03F1604303F56143202183F8A0
:104830000013F1E7704700BFFCEC00E0002080F3BC
:104840001488BFF36F8F1AF0F9FF00200D4908603C
:10485000BFF34F8F0C4880F3088800F02DF820201C
:1048600080F3118809484FF40261401880F30988E9
:10487000EFF314800221084380F31488BFF36F8F95
:10488000FEF7CAFF94ED00E0C07B0020407D0020D1
:10489000084BD3F89000C0F30720002306E0054A38
:1048A000C2F898300021C2F8A01001338342F6DB31
:1048B000704700BF00ED00E010B572B6002484F32D
:1048C0001388FFF7E5FF234608E003F120010E4AB5
:1048D0004FF0FF3042F821000133DBB2072BF4D94F
:1048E000002308E003F16001074A4FF0FF3042F86F
:1048F00021000133DBB2072BF4D962B6BFF34F8F2F
:10490000BFF36F8F10BD00BF00E100E008B50A4B98
:104910009B68834202D00FF005FB08BDEFF30583CF
:10492000002BF8D0054B5A6842F080525A605A6A00
:1049300022F400425A62EEE7484F002000ED00E00A
:1049400008B5034B034A0121034814F060FE08BD7B
:1049500000000420000000204C17030008B5D0F828
:10496000A830203B0448036020234360034B83604E
:10497000012114F050FE08BD3C2A002000000B1558
:10498000084AC2F898000B6823F01F03034343F062
:104990001003C2F89C308B6843F00103C2F8A030CA
:1049A000704700BF00ED00E0B0B500AF0446072837
:1049B00004D8FFF7E5FF2046BD46B0BD6D4688B080
:1049C0006B4613F1100234D00C211AB1042901DD19
:1049D0001B48586112B1082900DD9C610B292BDDB1
:1049E0000C2052B10021032464F307016FF30F215F
:1049F0006FF317416FF31F61196100216FF300011D
:104A00006FF341016FF382016FF3C501012363F37B
:104A1000881100F47B7363F352216FF3DE416FF36F
:104A2000DF710023074814F042FCAD466FF015001B
:104A3000C2E76FF00041C8E76FF01B00D1E700BF8D
:104A40005817030060FC02002DE9F04700AF8146D3
:104A500088469A46164600250FE06FF0004124E094
:104A60006FF01B002DE02146F0B214F0B1FD0646B8
:104A700010F1160F4CD001360135454548DA05EBEB
:104A8000450409EB84046268002AF5D0BAF1000FEE
:104A9000E9D0204614F08BFD0028E4D16C4688B0A4
:104AA0006B4613F11002D8D00C211AB1042901DD94
:104AB0001948586112B1082900DD9D610B29CFDD2D
:104AC0000C2052B10021032565F307016FF30F217C
:104AD0006FF317416FF31F61196100216FF300013C
:104AE0006FF341016FF382016FF3C501012363F39B
:104AF000881100F47B7363F352216FF3DE416FF38F
:104B0000DF710023054814F0D2FBA5466FF01506AF
:104B10003046BD46BDE8F0878017030060FC020008
:104B200010B5034C01232278FFF78EFF207010BDD3
:104B30005C5A002008B50023094A1278FFF784FF69
:104B400010F1160F0AD0034606E0064AC2F8983064
:104B50000021C2F8A0100133072BF6DD08BD00BF0D
:104B60005C5A002000ED00E0044B0522C3F89420BD
:104B7000BFF34F8FBFF36F8F704700BF00ED00E0B2
:104B8000BFF35F8F024B0022C3F89420704700BF31
:104B900000ED00E038B50E4B1D68082D15D8FFF765
:104BA000EFFF002409E00A4B596804EB440293002C
:104BB00019442046FFF7E4FE0134A542F3D8054B23
:104BC0001D70FFF7D1FF002038BD4FF0FF30FBE72D
:104BD000B41703005C5A0020014B1860704700BFF7
:104BE000D00100200EB400B584B005AB53F8042BFF
:104BF00001906FF000410291039301A90548FDF770
:104C000063F8019B00221A7004B05DF804EB03B056
:104C1000704700BF8D9702004FF02002EFF3118321
:104C200082F31288BFF36F8F044A0121C2F8401546
:104C300083F31188BFF36F8F0020704700E00140BD
:104C4000C0B24FF08042C2F81C05BFF34F8F054938
:104C5000CA6802F4E062044B1343CB60BFF34F8F8A
:104C600000BFFDE700ED00E00400FA0530B108B533
:104C70008001034B43F00103984708BD704700BF14
:104C800040FD0200402928BF402100238B421CD256
:104C900030B410F803C04FEA1C1C5A000D4D15F833
:104CA0000CC00D4C04F813C010F803C00CF00F0C2E
:104CB000013215F80C50A55401338B42E9D3064854
:104CC000002200F8132030BC70470348002200F88F
:104CD00013207047D8170300482A002038B504462F
:104CE000054818F04DFB054620B10021083018F0AA
:104CF00069FB2C75284638BD3008002010B50246E7
:104D00000A4BD3F8B80058B118F094FB04460123BD
:104D1000037500218181083018F054FB204610BD36
:104D20000B460120FFF7DAFF0446F7E700000020FA
:104D300010B5A0F10E0CBCF1010F06D959B9012034
:104D4000FFF7CCFF0446204610BD10461946FFF77A
:104D5000D5FF0446F7E7064818F012FB0446002882
:104D6000F1D00021083018F02DFB01232375EAE76C
:104D7000D807002082685178074B83F824105188A7
:104D8000D984117983F82510B2F807101985B2F883
:104D900005205A85704700BF000000208368197AFB
:104DA000DA7942EA012198795A7942EA002242EA04
:104DB00001421879D97841EA002198785B7843EA72
:104DC000002343EA01430349C1F89830C1F89C200D
:104DD000704700BF0000002083681B7893B9BFF3C1
:104DE0005B8F094B53F8882FBFF35B8F02F00902EA
:104DF000BFF35B8F53E8001F43E800200028F9D180
:104E0000BFF35B8F704700BF0000002008B58168CA
:104E100008220131014814F069FC08BD2C00002073
:104E200008B5816840220131014814F05FFC08BDDB
:104E30003400002008B5816808220131014814F0CF
:104E400055FC08BD90000020F8B500AF05460E46A1
:104E50001446907909F03AFC884B834252D0A679E7
:104E6000304609F033FC6C468AB0694611F11002F5
:104E700042D018232AB1042B03DDDFF804C2C1F8A5
:104E800014C012B1082B00DD8D6112B10C2B00DDB6
:104E9000CE6112B1102B00DD08621AB1142B01DDB6
:104EA00076484862172B2ADD182052B100230625C8
:104EB00065F307036FF30F236FF317436FF31F635C
:104EC0000B6100216FF300016FF341016FF3820169
:104ED0006FF3C501022363F3881100F47F7060F360
:104EE00052216FF3DE416FF3DF710023654814F048
:104EF000DEF9A546BD46F8BD6FF00043BAE76FF096
:104F00001B00D2E7204618F08FF900EB40005E4B03
:104F100003EB800043889D4233D15C4BD3F8B8004B
:104F200028B118F061FA594B0022C3F8B820204686
:104F300018F07AF900EB4000534B03EB8000436814
:104F40000BB1002E69D0204618F06EF900EB40003E
:104F50004D4B03EB80008368002BCBD0204618F02C
:104F600063F9494D00EB400005F82060204618F039
:104F70005BF900EB400005EB8005A8680EF018FA1D
:104F8000B8E7204618F050F900EB40003E4B03EB29
:104F9000800040886C4688B06B4613F1100236D012
:104FA00010211AB1042901DD394E5E6112B10829C0
:104FB00000DD9D6112B10C2900DDD8610F2929DDCA
:104FC000102052B10021042565F307016FF30F2172
:104FD0006FF317416FF31F61196100216FF3000137
:104FE0006FF341016FF382016FF3C501022363F395
:104FF000881100F47D7363F352216FF3DE416FF388
:10500000DF7100231F4814F052F9A54672E76FF0D4
:105010000041C6E76FF01B00D3E7204618F004F903
:1050200000EB4000184B03EB8000426813685168A6
:10503000107A01F01F050122AA4070B1490903EB63
:105040008103BFF35B8F53E8001F114343E8001057
:105050000028F8D1BFF35B8F75E7490903EB8103A3
:10506000D243BFF35B8F53E8001F114043E80010A9
:105070000028F8D1BFF35B8F65E700BF040800206C
:105080001C18030008FC0200CC2A002000000020AD
:105090005418030038B504460421083018F0FBF911
:1050A0004578224601784088FFF7CEFE05B938BD25
:1050B00001480EF07DF9FAE7A000002038B504465B
:1050C0000321083018F0E7F90578A368224619781B
:1050D000B0F80100FFF7B8FE05B938BD01480EF081
:1050E00067F9FAE7A000002098B500AF0121083069
:1050F00018F0D1F9007888B06B4613F1100233D064
:105100000C211AB1042901DD1A4C5C6112B1082985
:1051100000DD98610B292ADD0C205AB100214FF0E7
:10512000030C6CF307016FF30F216FF317416FF35B
:105130001F61196100216FF300016FF341016FF3EB
:1051400082016FF3C501012363F3881100F47B73BF
:1051500063F352216FF3DE416FF3DF7100230648E2
:1051600014F0A5F8BD4698BD6FF00041C9E76FF097
:105170001B00D2E78818030008FC020080B582B04B
:1051800000AF81898068FFF77DFD02233B7188B005
:105190006B4613F1100241D04FF00D0C22B1BCF15F
:1051A000040F01DD25495961022139711AB1BCF1A1
:1051B000080F00DD98611AB103F11C01002080B3D3
:1051C000BCF10C0F36DD0D206AB100214FF0030C4D
:1051D0006CF307016FF30F216FF317414FF0010CD0
:1051E0006CF31F61196100216FF300016FF341013E
:1051F0006FF382016FF3C501022363F38811C0F3DB
:10520000090363F352216FF3DE416FF3DF71002373
:105210000B4814F04CF80837BD4680BD6FF0004CC9
:10522000BCE707F1080E86441EF804EC01F801EB18
:105230000130C4E76FF01B00C6E700BFAC180300E5
:1052400008FC0200F0B583B000AF0446012108302D
:1052500018F021F905780023012B55D85D4A02EB9F
:10526000C30112F83320954209D1A3894A789342A9
:1052700007D34B68204698470C37BD46F0BD013335
:10528000EAE76C4688B0694611F1100236D010206A
:105290001AB1042801DD504E4E6112B1082800DD1C
:1052A0008B6112B10C2800DDCD610F2829DD1020A3
:1052B00052B10023042565F307036FF30F236FF347
:1052C00017436FF31F630B6100216FF300016FF34E
:1052D00041016FF382016FF3C501012363F388116C
:1052E00000F47D7363F352216FF3DE416FF3DF71DE
:1052F00000233A4813F0DBFFA546BDE76FF00040FE
:10530000C6E76FF01B00D3E7A6893146A068FFF718
:10531000B9FC04233B716C468AB06B4613F1100252
:1053200048D04FF0150C22B1BCF1040F01DD2C491F
:1053300059611AB1BCF1080F00DD9D611AB1BCF1D1
:105340000C0F00DDDE61042139711AB1BCF1100FC0
:1053500000DD18621AB103F12401002068B3BCF12A
:10536000140F33DD15205AB10021052565F307011F
:105370006FF30F216FF31741012565F31F61196169
:1053800000216FF300016FF341016FF382016FF3AE
:10539000C501022363F38811C0F3090363F35221AB
:1053A0006FF3DE416FF3DF7100230C4813F07FFFD2
:1053B000A54661E76FF0004CB5E707F10805054425
:1053C00015F8045C01F8015B0130C7E76FF01B00C2
:1053D000C9E700BFE41B0300D018030008FC02006B
:1053E000F41803002DE9F04182B000AF0446838930
:1053F000012B2AD9022104F1080018F04CF80546C7
:105400000378052B31D032D30E3BDBB2012B2AD8E7
:10541000012313F0020F2CD02D780023022B7DD80E
:10542000724A02EBC30112F8332095422FD1A389AF
:105430004A7893422DD34B6820469847204617F070
:10544000D3FF0837BD46BDE8F08140F63713684A00
:105450006849694813F0D9FB404080F311884FF048
:10546000030002DFC6E70223D3E70323D1E70223C9
:10547000CFE740F63B135E4A60495F4813F0C5FB37
:10548000404080F311884FF0030002DFC4E701338E
:10549000C4E76E4688B0694611F1100238D010207A
:1054A0002AB1042803DDDFF858C1C1F814C012B1D5
:1054B000082800DD8B6112B10C2800DDCD610F28BA
:1054C00029DD102052B10023042565F307036FF393
:1054D0000F236FF317436FF31F630B6100216FF30B
:1054E00000016FF341016FF382016FF3C5010123E6
:1054F00063F3881100F47D7363F352216FF3DE418F
:105500006FF3DF7100233F4813F0D1FEB54695E7F6
:105510006FF00040C4E76FF01B00D3E7B4F80C80D5
:105520004146A068FFF7AEFB04233B716E468AB08C
:105530006B4613F1100249D04FF0150C22B1BCF1AB
:10554000040F01DD304959611AB1BCF1080F00DDCB
:105550009D6122B1BCF10C0F01DDC3F81C80042158
:1055600039711AB1BCF1100F00DD18621AB103F1E4
:105570002401002068B3BCF1140F33DD15205AB1AB
:105580000021052565F307016FF30F216FF3174124
:10559000012565F31F61196100216FF300016FF3AD
:1055A00041016FF382016FF3C501022363F3881198
:1055B000C0F3090363F352216FF3DE416FF3DF7130
:1055C0000023104813F073FEB54637E76FF0004C28
:1055D000B4E707F10805054415F8045C01F8015B20
:1055E0000130C7E76FF01B00C9E700BF041C0300D0
:1055F000181903004C1903006819030088190300E7
:10560000D018030008FC0200F418030010B50C4683
:105610000A604B609DF808300B7217F005FE00EB36
:105620004000024B03EB8000446010BDCC2A0020F8
:105630002DE9F84306460F464FF0FF324FF0FF3397
:10564000184817F09DFE044600F10809002148465D
:1056500017F0B8FE4FF0000884F81480204617F0C9
:10566000E3FD114D00EB400005EB80004680204635
:1056700017F0DAFD00EB400005EB8003C3F808806B
:10568000204617F0D1FD00EB400005EB8005C5F882
:1056900004800321484617F0DDFE0680877020460F
:1056A000BDE8F88304080020CC2A00202DE9F04151
:1056B00086B000AF064615460C4600296ED0012282
:1056C0000021384619F0B4FC204617F0ADFD00EB80
:1056D00040004A4B03EB80008760204617F0AAFE8B
:1056E0000146474817F072FE4FF4A02200233846C7
:1056F0000DF086FE8046002858D1204617F094FD14
:1057000000EB40003D4B13F82080B8F1000F68D04B
:105710006D4688B06B4613F1100259D010211AB1B2
:10572000042901DD3748586112B1082900DD9E6166
:105730001AB10C2901DDC3F81C800F294BDD1020A4
:1057400052B10021042666F307016FF30F216FF3B6
:1057500017416FF31F61196100216FF300016FF3AF
:1057600041016FF382016FF3C501022363F38811D6
:1057700000F47D7363F352216FF3DE416FF3DF7149
:105780000023214813F093FDAD46204617F02CFE70
:10579000B8F1090F22D06FF0040025E0FFF748FFB1
:1057A000044600288BD16FF068001DE040F23513ED
:1057B000164A1749174813F028FA4146164813F0BD
:1057C00024FA404080F311884FF0030002DF94E791
:1057D0006FF00041A3E76FF01B00B1E76FF06E00C0
:1057E00002E02DB12C6000201837BD46BDE8F081E5
:1057F000204617F0F9FD0020F6E700BFCC2A002074
:10580000BC000020E419030008FC02001819030082
:10581000B819030068190300C419030010B582B059
:10582000224BD3F8D4309B6813F0010F0DD101AA9D
:10583000002140F60340FFF739FF044668B901989C
:10584000FFF7CAFA019817F0CFFD01AA002141F233
:105850000300FFF72BFF044610B1204602B010BD35
:105860000198FFF7D3FA019817F0BEFD01AA0021B5
:1058700041F20100FFF71AFF04460028EDD101981C
:10588000FFF778FA019817F0AFFD01AA002141F265
:105890000200FFF70BFF04460028DED10198FFF756
:1058A000BFFA019817F0A0FDD7E700BF0000002065
:1058B00010B588B03C4B93F8303013F0400F0AD04D
:1058C00001AA002142F20300FFF7F0FE034650B3A5
:1058D000184608B010BD354B07930023022262F32F
:1058E00007036FF30F236FF317436FF31F630693E1
:1058F00000216FF300016FF341016FF382016FF339
:10590000C501012363F38811082363F352216FF368
:10591000DE416FF3DF71002306AA254813F0C7FCB0
:105920006FF01203D4E70198FFF784FA019817F09B
:105930005BFD1D4B93F8303013F0200F18D01A4B3D
:1059400093F8503013F0080F0ED001AA002142F254
